:020000040800F2
:10000000002000100D560308F94B02081198000853
:10001000F74B0208F54B0208F34B02080000000002
:10002000000000000000000000000000F14B02088A
:10003000EF4B020800000000ED4B0208355A0008A3
:100040007556030875560308755603087556030858
:1000500075560308755603080966000835670008D9
:10006000F9660008BD66000881660008A120000846
:1000700091200008812000087120000861200008FC
:100080004D200008392000087556030875560308EE
:1000900005500208755603087556030845660008A2
:1000A00069510008A951000859510008D1510008B0
:1000B00099510008895100087951000875560308C4
:1000C00075560308755603087556030875560308D8
:1000D00075560308615B0008E55A0008695A000874
:1000E000CD65000875560308DD4B020875560308F8
:1000F00075560308755603087556030875560308A8
:100100000000000000000000000000007556030819
:100110007556030875560308495D01082D5D0108F1
:100120002520000811200008FD1F0008E91F000815
:10013000D51F0008755603080000000000000000ED
:10014000755603087556030875560308000000002D
:10015000000000000000000000000000000000009F
:1001600000000000000000007556030875560308E3
:1001700075560308000000000000000000000000A9
:080180000000000075560308A1
:10018800002870B51EDB0928044620DD012303EB97
:1001980083035B00B0FBF3F2092AF8D87BB10E4E5B
:1001A800B4FBF3F00928CCBF57223022A6FB03E5A5
:1001B800024403FB1044EB0801F8012BF0D10023A3
:1001C8000B7070BD2D230B7040420131DBE73030DE
:1001D80001F8010BF3E700BFCDCCCCCC884230B49A
:1001E8004FF001042ED301FB04F4B0FBF4F58D426B
:1001F800F9D284B1AAB901E0B0FBF4F5092DCCBF5E
:10020800572230222A4404FB150003F8012BB4FBC3
:10021800F1F4002CF0D100221A7030BC7047B0FB0A
:10022800F4F5092DCCBF372230222A4404FB1500EF
:1002380003F8012BB4FBF1F4002CF0D100221A7062
:1002480030BC70470546002AEBD1D7E703685A1C33
:1002580002601970704700BF2DE9F047089C2578A7
:10026800002B804689460CBF4FF0200A4FF0300A19
:10027800661C35B3002A29DD334601E0024698B1F1
:1002880013F8011B501E0029F8D1971E60B13D4696
:10029800013D51464046C8476B1C002BF8DC2578C9
:1002A80027EAE770013055B1041B29464046C84784
:1002B800301916F8015B002DF7D1BDE8F087BDE8CD
:1002C800F087002A04DC2846BDE8F0870020EBE729
:1002D800571EDCE783684268D0ED037A00EB8301A0
:1002E8000133934281ED040A836004BF00238360D5
:1002F80000EB830393ED047A036870EE277A9A4241
:10030800C0ED037A77EEC77AC0ED037A0CDA0133D1
:1003180007EE103AF8EEC76AB7EE007A87EEA60A3B
:10032800036030EE070A704707EE102AB8EEC77A66
:1003380087EE870A704700BF90ED057A90ED004A76
:10034800D0ED066AD0ED014AD0ED047A90ED035A5B
:10035800D0ED025AA4EE007AB0EE406AB0EE470A39
:10036800B0EE667AA6EE247A67EEC07AA0EE457AF9
:10037800E6EE257A80ED057AC0ED067A704700BF73
:10038800D0ED057A90ED013AD0ED003AD0ED064A6D
:1003980090ED024A90ED077A90ED035A90ED086AC5
:1003A800D0ED045AC0ED067AF0EE406A27EE830AD3
:1003B800C0ED056AA3EEA60A80ED087AA4EE240A29
:1003C800A5EE470AA5EEC60A80ED070A704700BFEA
:1003D800D0ED007A90ED017A30EE670AE7EE007A08
:1003E800B0EE670AC0ED007A704700BF704700BFE3
:1003F8000A44914214D030B40139551E41F2210209
:1004080011F8014F082380EA042004044CBF82EA53
:1004180040004000013B80B2F7D18D42F0D130BCA2
:1004280070470378407840EA032010FB01F04FF44E
:10043800807190FBF1F000F30F0000B27047704735
:1004480070474378007840EA032010FB01F04FF42E
:10045800807190FBF1F000F30F0000B270472DE9B6
:10046800F74F6A4CDFF8A8E123880091DEF8001006
:10047800B4F90480C3EB21125B00C3EBE103B4F9C8
:10048800021052435943131308FB03F84FEAA838E4
:1004980008EBE12101EB8102B1F5FA3802F18002A3
:1004A8004FEAE1794FEA222349F1FF39B4F90820EC
:1004B8000193A8FB08AB08FB09F30BEB430BA16105
:1004C800D31702FB09F108FB0311A2FB08230B4415
:1004D8001F03160347EA1257B4F90A2002FB0BF16F
:1004E800D3170AFB03130546A2FB0A011944020AA3
:1004F80042EA016292194FEA2123E6887B410032E1
:1005080043F50043A2FB060106FB03114A10CB1773
:1005180052EA03016FD0B4F91060B4F90E00F7176E
:1005280006FB0BF10AFB0711A6FB0AAB8B4400FB89
:1005380009F6C11708FB0161A0FB08898944DEF8A8
:1005480004104FEA4846C1F5801E4FEA494747EA7A
:10055800D8371AEB060AB4F90C8076464BEB070B32
:10056800F71700264FEACE70F90716EB0A064FEA8E
:10057800C80741EA5E0147EB0B0740F6354E861B7C
:1005880061EB0707A6FB0E010EFB071134F066FEB0
:10059800B4F916204E13470B47EAC14702FB06FE83
:1005A800D31707FB03EEA2FB07237344564307FB4D
:1005B8000366A2FB07233344560E46EAC3163218D5
:1005C800B4F914604FEA636747EB01037143F71707
:1005D80000FB0717A6FB00013944C60C46EA413662
:1005E80092194FEAE147B4F912607B41100A40EAD8
:1005F8000360320112180DB1120A2A60009B13B170
:100608001A46019B136003B0BDE8F08F1C3C002024
:10061800281E002070473122F42106F087B900BF58
:10062800012380F8453070474FF400638382704798
:1006380037B500F10C04054600220A21204606F0D1
:1006480075F9142005F054F90F220A21204606F006
:100658006DF90A2005F04CF901AA03231021204660
:1006680006F0F0F80A2005F043F99DF804308033CD
:100678006B839DF805308033AB839DF8063080335B
:10068800EB8300220A21204606F050F90A2005F0E3
:100698002FF90DF1030201230221204606F0D2F8BA
:1006A80001230DF103020921204606F0CBF811229F
:1006B8000A21204606F03AF9012003B030BD37B5CB
:1006C80004466A460D460C3003212DF03FF90246D8
:1006D80090B1B4F91A106846FFF7A3FE2880B4F960
:1006E8001E100DF10200FFF79CFEA880B4F91C1043
:1006F80001A8FFF796FE6880104603B030BDF0B53C
:1007080000F10C0585B004460F4601230DF10702E0
:100718000221284606F096F818B90026304605B09A
:10072800F0BD9DF80730DB07F7D502AA032128465C
:100738002DF00CF901230DF107020921284606F0D6
:1007480081F806460028E8D011220A21284606F03A
:10075800EDF89DF8073013F00C0FDED1B4F91A103C
:1007680002A8FFF76EFE40423880B4F91C100DF164
:100778000A00FFF766FE40427880B4F91E1003A80D
:10078800FFF75FFE4042B880C8E707B5F7216A4621
:100798002DF0DCF89DF801309DF800100B4A1B0184
:1007A80043EA01339DF8021043EA111353609DF8A0
:1007B80004309DF803101B0143EA01339DF805102E
:1007C80043EA1113136003B05DF804FB281E0020F0
:1007D80070B40468037B2268022101FA03F31A4209
:1007E80013D042690A495C2000FB02124FF6FE76DC
:1007F80050685289C5680068296831402960C16815
:10080800D24392B20A40C260636070BC704700BFB6
:100818004459002030B40A4B1D7875B1094B0020AB
:1008280003EBC5051A6899885062D4682143D160E2
:10083800083323F8040CAB42F4D130BC704700BF36
:10084800245C0020285C002010B40268047B116836
:100858000223A340194209D00649406800240C70BD
:1008680001684FF6FE742140016053605DF8044B47
:10087800704700BFFA4900202DE9F3410569064693
:100888000F467DBBD0F80080C8F30A0323B30023CA
:10089800D6F8008001932EF09BF8042819D1224C39
:1008A800236943F001032361BBB2A8F800302EF09E
:1008B8008FF804282ED108F102030193019B3F0C05
:1008C8001F802EF085F82369042823F00103236193
:1008D80025D06FF0010505E02EF07AF8042805D040
:1008E8004FF0FF35284602B0BDE8F0810E4C236971
:1008F80043F002032361C4F81480236943F04003E2
:1009080023612EF065F82369042823F0020323618C
:10091800BDD0E5E7236923F001032361D9E73368F4
:1009280004333360DEE700BF00200240F8B5044618
:100938000D468E180027B54201D12069F8BDE3683D
:10094800591CE160234415F8012B1A720429F2D1CD
:10095800A1682046FFF790FFE7602061EBE700BF42
:10096800014B186805F0A6B9841F00202DE9F04F47
:100978004FF4807385B043838383C38300F10C05F0
:100988000446322004F0B4FF11220021284605F065
:10099800CDFF60220121284605F0C8FF642004F03D
:1009A800A7FF02A920460027FFF789FE0123B946C1
:1009B800B8463E460193012E14BF1122122200218F
:1009C800284605F0B3FF002E0CBF4FF0010B4FF087
:1009D800FF3B4FF00A0A01220221284605F0A6FF34
:1009E800142004F085FF02A92046FFF768FEBDF930
:1009F8000A20BDF90C00BDF90810364B82420BFBEA
:100A08000299A8BF02468A42A8BF0A469A4201FB39
:100A18000B880BFB00775ADB012005F04FF9BAF180
:100A2800010AD8D10136022EC5D12B4B93FBF8F819
:100A380093FBF9F97022A3F58423002193FBF7F7C0
:100A4800A4F81A80A4F81C90E783284605F06EFFE6
:100A580020220121284605F069FF00223146284658
:100A680005F064FF642004F043FF019B23B94FF4B1
:100A780080736383A383E383607E20B304F042FB27
:100A8800054605F095FDF0B11DB12223AB71002399
:100A9800EB710021284605F075FB21460F4B41F804
:100AA800083F28462DF036F835B1AD88B5FA85F5FA
:100AB800C5F11F056B1C06D0094A0123116803FA0A
:100AC80005F50D431560012005B0BDE8F08F002342
:100AD8000193A7E701F0FFFF00D03B00490400089D
:100AE8000004014010B490E80600047B406902232A
:100AF800A3404B6013685DF8044B4FF6FE710B4042
:100B0800136005F067B800BF98B10B4B012210B411
:100B180002FA01F103F1750402E00333A34209D09C
:100B28001A788242F9D15A780A42F6D001205DF843
:100B3800044B70470020FAE7206B030810B4002329
:100B4800094C01E0272B0AD003EB43020133A15CD7
:100B58008142F7D122445DF8044B90787047002019
:100B68005DF8044B704700BF206B030870B54488DC
:100B780006460D46C4F30B0422460021284635F0EC
:100B88005CFF3369094A934209D3094A934206D262
:100B9800224628461946BDE8704034F051BE23B1BC
:100BA80021462846BDE87040184770BD34CC03087C
:100BB80020CD0308064B07498B4202D30023184671
:100BC80070471A88C2F30B029042F8D01433F3E747
:100BD800C0C7030834CC0308024A136823EA00009C
:100BE800106070478C5E0020F8B5174D2B78A52B48
:100BF80028D16B78BE2B25D1022229464FF6FF70EB
:100C0800FFF7F6FB114FAC1C22884AB1A618BE426A
:100C180018D2052A16D92146FFF7EAFB3446F3E72E
:100C280021460222FFF7E4FB0222A118FFF7E0FBAE
:100C38000634074B641B1C8041F60F53C31A5842F5
:100C48005841F8BD0020F8BD00F003080000040872
:100C5800163200202DE9F04FDFF848914C4F8BB049
:100C68000326A7EB09071822002104A835F0E5FEA2
:100C7800484BCDF8109005971A69120604D5464AD4
:100C88005A6002F188325A6001228DF824203422F9
:100C9800DA60424B424C1B88ADF8003002226946AC
:100CA80004A8FFF743FE022269464FF6FF70FFF7DC
:100CB8009FFBDFF8F4A080464FF0000B544536D375
:100CC8000AAC002524F8245D0222214604A8FFF777
:100CD8002DFE022221464046FFF78AFB40BAC04358
:100CE800ADF80800022202A904A8FFF71FFE079822
:100CF80060B106ABC0F104022946184435F09DFEE8
:100D0800069904A8FFF7B8FD079508909DF82430C8
:100D1800089A23B11F490B6943F080030B61013E18
:100D28002DD0002A9FD1FFF75FFF50B32CE06588D4
:100D38008DF80DB0C5F30B05AB1DADF80830238851
:100D4800C3F30B02ADF80A201B0B062202A904A864
:100D58008DF80C30FFF7EAFD062202A94046FFF79E
:100D680047FB616880462A4604A8FFF7DFFD6168F3
:100D780040462A46FFF73CFB143480469EE7002A8B
:100D8800D1D0052003F080F80BB0BDE8F08F00BF8C
:100D9800000004080020024023016745956B030802
:100DA800C0C7030800F0030834CC03080378202BDD
:100DB800024600F10100F9D0092BF7D02D2B2CD0D9
:100DC8002B2B03BF5378B7EE000A0246B7EE000A92
:100DD800A3F13001C8B209289FED467A10D8F2EE87
:100DE800046A07EE901AF8EEE77A12F8013FE7EE88
:100DF800267AA3F13001C8B20928B0EE677AF0D993
:100E08002E2B4CD003F0DF03452B0BD0F7EE007AE6
:100E180067EE276A20EE260A70475378BFEE000A6D
:100E28000246D5E710B451782D2959D02B290ABF8D
:100E38009178501C901C0024A1F13003092B53D841
:100E4800002303EB830301EB430310F8011FA1F117
:100E58003002092AA3F13003F3D9B3F59A7F28BFEA
:100E68004FF49A73072B42D9DFED236A1A46F7EE3F
:100E7800007A083A072A67EEA67AFAD803F0070339
:100E88002BB1F2EE046A013B67EEA67AFBD124B3DC
:100E9800C7EE276A5DF8044B20EE260A70475378A0
:100EA800A3F13001C8B2092802F10102AAD8F2EE72
:100EB800046AF0EE665A07EE901AF8EEE77A12F82E
:100EC800013F87EEA66AA3F13001C8B2092866EE91
:100ED800A56A37EE067AEED994E767EE276AD9E76E
:100EE800901C91780124A7E7F7EE007ACFE7F7EE98
:100EF800007AC5E70000000020BCBE4CB5EEC00A71
:100F0800DFED317AF1EE10FACCBF30EE270A30EE81
:100F1800670ADFED2E7A20EE270A30B5FDEEC07A9B
:100F280087B017EE904A054684EAE470002303A9C7
:100F3800A0EBE47001930093029331F009FC002CBC
:100F4800ACBF20232D2303A88DF8003033F0DCFC40
:100F5800012803A924D002282DD0032805BF302357
:100F6800684668468DF8013035F06FFD684633F005
:100F7800CBFC0338C4B222466946284635F09CFDAE
:100F880000232B55284633F0BFFC2E22431C2A543D
:100F98000DEB0401E81835F075FD284607B030BDA3
:100FA800302368468DF801308DF802308DF8033013
:100FB80035F04BFDDAE7302368468DF801308DF8BF
:100FC800023035F042FDD1E76F12033A00007A444F
:100FD8002DE9F041064615460846B6FBF2F43CB941
:100FE80005FB1464124B1B5D00F8013BBDE8F08162
:100FF800B4FBF2F767B90E4B05FB174705FB146402
:10100800DA5D00F8012B1B5D00F8013BBDE8F081BB
:10101800B7FBF2F8B8F1000F02D04046FFF7D8FF4F
:1010280005FB1878024B13F8082000F8012BE3E7BA
:10103800589603082DE9F04714461D460646002336
:101048004FF47A722046294634F008F9DFF84881CF
:101058004B4A4C4F88FB00310144C31782FB002EDA
:10106800C3EB611188FB012887FB00278644464AA9
:10107800C3EBEE2EC1EB011C82FB0E29A0EB8C0CFE
:101088000744424A86F806C0C3EB27474FEAEE7C7E
:1010980008EB010ACCEBA90C82FB07824FEAE17846
:1010A8000CEB4C0CC8EB6A18AEEBCC0EC8EB08186E
:1010B800DFF8E8C086F804E0A1EB880171718CFBC9
:1010C8000010F917C1EBE21240F2B55101FB1272A0
:1010D800C3EBE050B2F5896F4FEA800740DA40F27F
:1010E800DA239A4244DCB2F5B77FB4BF4FF0000C64
:1010F8004FF0010C4FEA4C08254B08EB0C0103EBB1
:10110800C1031FFA8CFEB3F88E00224908EB0C03CA
:1011180001EBC30116310B2301E031F8020D8242C5
:101128001BDA013BF9D11A4BC44403EBCC0C012365
:10113800BCF87800B37007F2B2770132121ABE44D5
:10114800F270A6F800E0204629464FF47A72002390
:1011580034F084F83281BDE8F0870133DBB2E9E787
:101168004FF0030EF44640F296504FF00608CCE7D5
:101178004FF0020EF44640F229404FF00408C4E74D
:10118800C5B3A29107452EC2ABAAAA2A73B06D16A1
:10119800206B0308986B030889888888792D0311C8
:1011A800104B2DE93048D3E9004554EA05020BD12C
:1011B8000346012200201871587198719A70DA70EC
:1011C80018801881BDE83088074B1A6814EB020BA9
:1011D80045F1000C5A466346FFF72CFF0120BDE895
:1011E800308800BFE81F002090640020F0B4028817
:1011F8008578164FC37804794179A2F2B27202F069
:10120800030606EB4606013D05EB860507EB45059B
:10121800013BB5F878608579008940F2B5579208A6
:1012280007FB0232931903EB430304EBC303C3EB3D
:10123800031301EB8303C3EB031305EB83030021C3
:101248004FF47A72C2FB0301F0BC7047206B0308AD
:10125800FAB170B48E18044603E0101A14D1B142E2
:1012680014D014F8012BA2F14103192B11F8013BFA
:10127800A3F1410598BF2032192D03F12000ECD9C4
:10128800D01A01D1002BEAD170BC7047002070BC85
:1012980070471046704700BF4FF0FF32FFF7D8BFC6
:1012A800A0F16103192B98BF20387047A0F14103C2
:1012B800192B98BF20307047202805D009380428FA
:1012C8008CBF002001207047012070476138192821
:1012D8008CBF002001207047413819288CBF00209E
:1012E80001207047303809288CBF00200120704742
:1012F800A0F13003092B07D920F020004138192824
:101308008CBF0020012070470120704730B402686C
:101318001146531C036011F8024B0160D31C51782D
:1013280003609378151D05601B0443EA0123D078F8
:10133800234343EA006030BC704700BF0368591C70
:101348001A46016012F8021B0260587841EA002030
:10135800704700BF03685A1C02601878704700BFC6
:1013680038B504460068154634F06AFA22682A44FB
:10137800226038BD036810B40A0A5C1C04601A7045
:1013880003685A1C026019705DF8044B704700BF6F
:1013980003685A1C026010B4197003680A0A5C1CBE
:1013A80004601A7003680A0C5C1C04601A700368F5
:1013B800090E5A1C026019705DF8044B704700BF93
:1013C80003685A1C026019700368090A5A1C0260F3
:1013D800197070472DE9F047002488B080460F4601
:1013E8001E46A14605AD531C0393117839B3252930
:1013F80033D1931CCDF810900393507830284ED0F9
:101408004FF0000AA0F13003DBB2092B42D96C2857
:1014180019D0642800F0938024D825281CD063D9DB
:10142800582876D063281BD131784046B847039AAC
:10143800531C03931178043601340029D7D1204670
:1014480008B0BDE8F087039B5A1C03921B78642BF5
:101458007CD02AD8252B54D1252140460134B847C1
:10146800039AC0E7732833D044D975284FD106F1C1
:10147800040E30682B4600220A217646FEF7AEFE9F
:10148800049A0095534639464046FEF7E5FE039A0E
:101498000444A8E704AA03A931F0A2F8B7E7D31CCB
:1014A800039390784FF0010AACE7732B10D05BD907
:1014B800752B3AD0782B96D1A3F15802B2FA82F262
:1014C800306852092B4610210436FEF787FED7E70D
:1014D8003368049A0093394600234046FEF7BCFE61
:1014E80004360444039A7EE70028B9D1204608B0A0
:1014F800BDE8F0876E28B3D1039A336804361C60C0
:1015080071E72AD9582BD7D0632B8DD06BE7782871
:10151800A6D1A0F15802B2FA82F2306852092B46DD
:101528001021FEF75BFE0436AAE706F1040E3068C8
:101538002B4600220A217646FEF750FEA0E7331D0F
:10154800306829461E46FEF71BFE99E7331D3068B2
:1015580029461E46FEF714FE92E7002B7FF443AFA0
:10156800204608B0BDE8F0876E2BC6D03BE700BF29
:101578000EB400B584B005AB019053F8042B0649AE
:10158800039301A8FFF726FF019B00221A7004B0FD
:101598005DF804EB03B07047550200080FB430B58E
:1015A80083B006AB0A490B4853F8042B0968006856
:1015B8000193FFF70FFF084C0546206804F06AFB0B
:1015C8000028FAD0284603B0BDE8304004B0704780
:1015D800582E00205C2E0020841F0020DFED2B7A7F
:1015E800B4EEE70AF1EE10FA4ADDDFED296A9FED65
:1015F800297A01E0B0EE670AB4EEC70AF1EE10FAF4
:1016080070EE667AF6DC9FED247AF4EEC77AF1EE96
:1016180010FA38D5DFED1E6A9FED207A01E0F0EE72
:10162800407AF4EEC77AF1EE10FA37EEA60AF6D44D
:10163800DFED1B7AB4EEE70AF1EE10FA14DDDFED08
:10164800137A37EEC00A60EE006A9FED166A9FEDC6
:10165800167ADFED167AA6EE867A20EE266AE6EE90
:10166800877AA6EE270A7047DFED117AB4EEE70A0B
:10167800F1EE10FA44BFDFED087A37EEC00AE2E770
:10168800F0EE407ABFE7B0EE670AD1E7DB0F4940DA
:10169800DB0FC940E4CB1641DB0F49C0E4CB16C1D0
:1016A800DB0FC93F92E741B99730083C15A82ABE1D
:1016B800DB0FC9BF09B909E0194690FBF1F301FB3B
:1016C80013030846002BF7D1084670470146FBE78D
:1016D80007EE901AF8EE677A9FED837A27EE800A74
:1016E80020EE070AFDEEC07A17EE903A2033402B21
:1016F80000F28C80DFED7D7AB4EEE70AF1EE10FAA5
:1017080040F3E880B0EE407A9FED796ADFED796AC0
:1017180001E0B0EE677AB4EEE67AF1EE10FA77EE11
:10172800467AF6DC9FED747AF4EEC77AF1EE10FA99
:1017380040F1CD809FED6E6ADFED706A01E0F0EE5A
:10174800477AF4EEE67AF1EE10FA37EE867AF6D4B6
:10175800DFED6B7AB4EEE77AF1EE10FA51DCDFEDEB
:10176800697AB4EEE77AF1EE10FA44BFDFED627AF7
:1017780037EEC77A27EE076ADFED635ADFED637A43
:10178800DFED636A9FED635AE6EE257A67EE065A47
:10179800E6EE276AF7EE007AA5EEA67AF0EE675A2B
:1017A800E7EE055AE7EE457A87EEA55ADFED547A5B
:1017B80030EE277AFDEEC76A16EE903A2033402BBA
:1017C80029D99FED557AF6EE006AB7EE006AF7EE72
:1017D800004AC4EEA57A0023836143610362C361B2
:1017E80080ED045A67EEA66A27EE866A27EE877AA6
:1017F800C0ED006AC0ED026A80ED016A80ED037AEF
:101808007047DFED3A7A37EEC77AB3E7B7EE005A9A
:10181800F0EE455ACAE7B4EEE70AF1EE10FA5FDDDA
:101828009FED336ADFED336A01E0B0EE677AB4EE1C
:10183800E67AF1EE10FA77EE467AF6DC9FED2E7A2C
:10184800F4EEC77AF1EE10FA47D59FED296ADFED7D
:101858002B6A01E0F0EE477AF4EEE67AF1EE10FA40
:1018680037EE867AF6D4DFED267AB4EEE77AF1EE33
:1018780010FA27DCDFED237AB4EEE77AF1EE10FAFE
:1018880044BFDFED1D7A37EEC77A27EE076ADFED32
:101898001E4ADFED1E6ADFED1E7AE6EE246A67EE69
:1018A800064AE6EE267AB7EE006AA4EEA77AF6EEC6
:1018B800006A36EE476AF8EE007A27EE277A66EE77
:1018C800266A84E7DFED097A37EEC77ADDE7B0EEFE
:1018D800677A3DE7F0EE407A24E7B0EE677AC2E730
:1018E800F0EE477AAAE700BF27D4D236DB0F49408B
:1018F800DB0FC940E4CB1641DB0F49C0E4CB16C16E
:10190800DB0FC93FDB0FC9BF92E741B99730083CED
:1019180015A82ABEF304353F0000008070B406689D
:101928008E4217D90139751E002311F8014F08227C
:10193800634013F0800F4FEA430318BF83F0D503C9
:10194800013ADBB2F5D18D42EFD1721C02603370DF
:1019580070BC70470023F8E710B44C09012250F816
:10196800243001F01F0102FA01F10B4340F8243042
:101978005DF8044B704700BF4B0901F01F0150F898
:101988002320012303FA01F1114214BF1846002055
:10199800704700BF08B540F2E93300E09BB1028907
:1019A800013B12F0020F9BB2F8D0017340F2E93309
:1019B80000E043B10289013B12F0010F9BB2F8D05D
:1019C800007BC0B208BD04F02BFFC0B208BD00BF49
:1019D800F8B584894FF6FF764FF47A742BB311B3B8
:1019E8000F78013101E0B44217D00589013CAD07F9
:1019F800A4B2F8D507734FF47A7402E0BCB2B442CB
:101A08000BD00589ED0704F1FF37F7D5057BEDB25B
:101A18000AB115700132013BE0E704F001FF003024
:101A280018BF0120F8BDFF27DFE70120F8BD00BF80
:101A3800F0B55B4B5B4A97B01968914200AF00F074
:101A4800A3805949594A00234FF47000C1F888000F
:101A58003B607B60136843F48033136003E03B68AA
:101A6800B3F5A04F09D0136803F400337B603B68DB
:101A780001333B607B68002BF1D04C4B1B6813F49F
:101A8800003318BF01237B607B68012B52D0464C82
:101A9800464B474AE260474A596A11605A6A42F01F
:101AA80080725A625A6942F4FC025A610025032284
:101AB80007F10801012341F6FF764FF09040FD60E1
:101AC800BE603A73BB7328F051F94FF6FF7307F104
:101AD80008013948BB6028F049F907F1080137487F
:101AE800374E28F043F907F10801364828F03EF947
:101AF80007F10801344828F039F907F1080133489B
:101B080028F034F907F1080028F08AF9BB68304951
:101B1800304AA1FB031330499B0CF0204FF0070E0D
:101B28005C370B60566084F823009560C2F800E0CB
:101B3800BD46F0BD294A1D4B122111605A685A60F2
:101B48005A685A605A6842F480625A605A6822F4A5
:101B58007C125A605A6842F4E8125A601A6842F0D5
:101B680080721A601A689201FCD559680F4A21F0F0
:101B780003015960596841F002015960536803F044
:101B88000C03082BFAD182E700221A6062B6144BC4
:101B98001B6883F30888134B1B689847FEE700BF50
:101BA800FC9F0020EFBEADDE00ED00E0001002401B
:101BB8000005FA057C6A0020000400480008004877
:101BC8003F190100000C00480010004800140048AC
:101BD80083DE1B4310E000E09464002000200240F4
:101BE80000D8FF1F04D8FF1F064A0023516881420E
:101BF80002F11C0204D001330C2BF7D100207047EE
:101C0800D8B27047E400002070B50F4C0F4DC0EB00
:101C1800C00004EB8004686926693043686182B0BB
:101C28009209667BA1600025012101A863618DF8F6
:101C380004608DF805208DF806508DF8071028F0FF
:101C48005FF802B070BD00BFE40000200010024041
:101C5800074BC0EBC00030B403EB8000054C0569AE
:101C680063692B4363610176427630BC704700BFDD
:101C7800E4000020001002402DE9F04F554C54F8C4
:101C8800204083B0002C60D0A56D1F469046524B73
:101C98006A682265A160236004F15E014FF48073D5
:101CA80004F5AF726161A261E36023610646287E94
:101CB8002CF00CFFE86858B1FFF796FF721CD2B2FF
:101CC8000C21FFF7C5FF236DEA6862632433E364E0
:101CD800A86890B1FFF788FF721C8146D2B20B2129
:101CE800FFF7B6FF2346EA7E3C494846FFF78CFFDC
:101CF800236DAA68A2632833A36494F85D0003F0F7
:101D080001FA814694F85C0003F0FCF93A07824630
:101D180095F819B01DD5B9F1000F1AD017F0110FA9
:101D28004FF00B0306F1010614BF4E213E2189F83E
:101D3800063089F807605A46484602F043FEFB071A
:101D480043D5636B6BB3A36B5BB3204603B0BDE8AD
:101D5800F08F17F0010F0CBF2E274E2718F0020F37
:101D68000DD0B9F1000F0AD00B22731C89F8062098
:101D780089F8073048465A46394602F023FE18F0DB
:101D8800010FDED0BAF1000FDBD001360C238AF840
:101D980007605A4639468AF80630504602F012FE65
:101DA800CFE72B7FAA7E8DF804209B090021012212
:101DB80001A88DF805308DF806108DF8072027F05A
:101DC8009FFF204603B0BDE8F08F484604F096FB1D
:101DD800B7E700BF6C2E0020F86B0308ED0A000877
:101DE80000B97047F0B595B005462DF013FA6E4E60
:101DF800C368026832600446002B00F0C38028469E
:101E080003F080F9694B986018B129220023827188
:101E1800C371227A664D2E2102F0D4FD306803F09A
:101E280051FB2CF053FE3068624A038823F001030B
:101E38001B041B0C038014A91E232B8001270F23CE
:101E48000025138021F84C7D2D230293ADF80C500A
:101E5800ADF80650ADF80E502DF08AF9E379ADF8DB
:101E6800145060229907ADF816500695ADF81C502D
:101E7800ADF81E50ADF82050ADF82250049200F194
:101E8800838013F0010F14BF022200224FF48073E5
:101E9800ADF81470ADF81C20ADF82030002304AA6A
:101EA80061793068069302F091FB306861792DF012
:101EB8003FF93068436C43F40043436403889BB2A2
:101EC80043F080030380E3799B0768D56179026A50
:101ED80004238B4022EA03020262026A134303626C
:101EE8003268354F13889BB243F001031380207C7E
:101EF80000222921FFF7ACFE3049207C0023602214
:101F0800FFF782FEE068386027F066FE38680368ED
:101F18004FF6FE721340036027F05EFE09A827F013
:101F28002DFE33686279264938680A9134331344A0
:101F3800099380221023002509A940F22A3E0E9217
:101F48000B934FF400724FF400530D9510951395B1
:101F580011950F921293ADF830E027F01DFE6279CB
:101F680033680C2A98BF1749D86898BF31F81250BF
:101F78003A6815490543DD601368012043F0020300
:101F88001360087015B0F0BD13F0010F14BF0822DC
:101F98002A460423ADF81E20ADF816307EE701224C
:101FA800617927F029FD9BE7C05E0020281E0020EC
:101FB800B65E0020B45E0020BC5E00205108000818
:101FC8004C4B0020F88B0308B85E00200348D0F87B
:101FD8003C3113B100F59A7018477047E4000020AF
:101FE8000348D0F8203113B100F58C7018477047BA
:101FF800E40000200348D0F804310BB1FC30184746
:10200800704700BFE40000200348D0F8E8300BB167
:10201800E0301847704700BFE40000200348D0F8BC
:10202800CC300BB1C4301847704700BFE400002023
:102038000348D0F8B0300BB1A8301847704700BF3C
:10204800E40000200348D0F894300BB18C301847D6
:10205800704700BFE40000200248836F0BB1703066
:1020680018477047E40000200248C36D0BB1543094
:1020780018477047E40000200248036C0BB1383061
:1020880018477047E40000200248436A0BB11C302F
:1020980018477047E40000200248836803B11847D6
:1020A800704700BFE4000020F0B53E4C059D00EBF2
:1020B800800004EB80046468002C71D03A4E49001B
:1020C8004FF42040CFB2F060A169090454D460688D
:1020D800DFF8E0E047F4903100EA0E0001434FF4E6
:1020E80020406160F06003E0411E002848D00846A7
:1020F800A1698907F8D54FF42040A262F06003E097
:10210800421E00283CD01046A2695206F8D5274A3C
:102118006168DFF8A0E0F06042EA0342174301EA91
:102128000E0217436760C3B1013BDBB201332B4496
:10213800A0694FF4204210F0040002F1FF3207D1E9
:10214800511C26D0A06910F0040002F1FF32F7D02C
:10215800626A05F8012B9D42EAD14FF42040F060F5
:1021680002E0431E60B11846A3699B06F9D52023F7
:10217800F060E3610120F0BD411E08B10846A3E705
:102188000B4A138801339BB24FF0FF311380F16083
:10219800F0BD0749F2600B8801339BB20B80F0BD9C
:1021A8002046F0BD00640020281E00200024000204
:1021B80014320020009800FCF0B5037C012B85B098
:1021C800044663D0022B67D1836913B11A689B88D0
:1021D8001385606940F2E93301E0002B6CD0028975
:1021E800013B12F0020F9BB2F7D0C323037340F2F6
:1021F800E93301E0002B5FD00289013B12F0010FA7
:102208009BB2F7D0037B60694FF0060E838902AE5C
:102218004FF47A734FF6FF71FF2703E0013B9BB23F
:102228008B423CD002899507F8D507734FF47A732F
:1022380002E0ABB28B4232D00289D20703F1FF35FC
:10224800F7D5027BD2B20EB132700136BEF1010E63
:10225800E8D1A36913B11A689B8893619DF80C00B3
:102268009DF808609DF809109DF80A509DF80B200C
:102278009DF80D3041EA062143EA002342EA05228F
:10228800012021876287A38705B0F0BD90F914006B
:10229800431C01D0022805DD002005B0F0BD04F084
:1022A800BFFAD6E702AB617D009343220623FFF70E
:1022B800FBFE0028D2D1EFE704F0B2FAA3E700BF93
:1022C800F0B5037A012B85B0044663D0022B67D1A1
:1022D800036913B11A689B881385E06840F2E933F3
:1022E80001E0002B6CD00289013B12F0020F9BB277
:1022F800F7D0BB23037340F2E93301E0002B5FD032
:102308000289013B12F0010F9BB2F7D0037BE06812
:102318004FF0060E838902AE4FF47A734FF6FF71C1
:10232800FF2703E0013B9BB28B423CD00289950713
:10233800F8D507734FF47A7302E0ABB28B4232D010
:102348000289D20703F1FF35F7D5027BD2B20EB16D
:1023580032700136BEF1010EE8D1236913B11A6853
:102368009B8893619DF80C009DF808609DF8091002
:102378009DF80A509DF80B209DF80D3041EA062182
:1023880043EA002342EA05220120E1822283638393
:1023980005B0F0BD90F90C00431C01D0022805DD02
:1023A800002005B0F0BD04F03BFAD6E702AB617B34
:1023B80000933B220623FFF777FE0028D2D1EFE7F0
:1023C80004F02EFAA3E700BFB0F1FF3F56D0022871
:1023D80054DCF0B4324C00EB800004EB800044681D
:1023E800002C5BD02F4E49004FF42040CDB2F06056
:1023F800A169090444D460682B4F45F080713840C6
:1024080041F4903101434FF420406160F06003E0F3
:10241800411E002838D00846A1698F07F8D54FF427
:102428002040A262F06002E0421E68B31046A26932
:102438001106F9D562681C4945F0007545F48035E8
:102448000A4015434FF420406560F06002E0421EE8
:10245800D0B11046A2699207F9D54FF42040A36283
:10246800F06002E0431E78B11846A3699B06F9D5CF
:102478002023F060E3610120F0BC70470020704722
:10248800411E08B10846B3E7084A138801339BB2D6
:102498004FF0FF311380F160F0BC70472046FBE736
:1024A80000640020281E0020009800FC1432002040
:1024B8002DE9F04F85B090F855300190002B41F090
:1024C8005580019A137C012B01F0AC80022B44D17A
:1024D800936913B11A689B881385019B586940F268
:1024E800E93302E0002B01F00A810289013B12F076
:1024F800020F9BB2F6D06B23037340F2E93302E07C
:10250800002B01F0FC800289013B12F0010F9BB205
:10251800F6D0037B019B586940F2E93302E0002BB7
:1025280001F0E9800289013B12F0020F9BB2F6D05C
:102538008023037340F2E93302E0002B01F0DB80D3
:102548000289013B12F0010F9BB2F6D0037B019B7D
:102558009B6913B11A689B8893618F4C8F4DDFF884
:1025680044928F48DFF840E24FF0640A4FF0100CB5
:102578004FF47A76D9F80430C3F30803002B40F0FF
:102588006587EFF31183002B40F06087216882682C
:1025980000BF23689942F9D12F6806FB07F39B1AFD
:1025A800B3FBF7F306FB013101270091D9F804309A
:1025B800C3F30803002B40F08E85EFF31183002B43
:1025C80040F089852368816800BF22689342F9D169
:1025D800D5F800B006FB0BF2521AB2FBFBF206FB71
:1025E8000323009A9B1AB3F57A7FDFD3BAF1010A65
:1025F800C0D1019A137C012B01F01E80022B44D11B
:10260800936913B11A689B881385019B586940F236
:10261800E93302E0002B01F07A800289013B12F0D5
:10262800020F9BB2F6D06823037340F2E93302E04D
:10263800002B01F06C800289013B12F0010F9BB264
:10264800F6D0037B019B586940F2E93302E0002B86
:1026580001F059800289013B12F0020F9BB2F6D0BB
:102668000723037340F2E93302E0002B01F04B80AB
:102678000289013B12F0010F9BB2F6D0037B019B4C
:102688009B6913B11A689B889361DFF81891444ECF
:10269800DFF814C14FF0640A4FF010084FF47A774E
:1026A800D9F80430C3F30803002B40F0EC86EFF3AD
:1026B8001183002B40F0E7862168B26800BF2368C9
:1026C8009942F9D1286807FB00F39B1AB3FBF0F392
:1026D80007FB013101200091D9F80430C3F3080346
:1026E800002B40F01685EFF31183002B40F0118585
:1026F8002368B16800BF22689342F9D1D5F800B0C9
:1027080007FB0BF2521AB2FBFBF207FB0323009AFA
:102718009B1AB3F57A7FDFD3BAF1010AC0D1019AC7
:10272800137C012B00F0C087022B4FD1936913B1A2
:102738001A689B881385019B586940F2E93302E0C7
:10274800002B00F0EC870289013B12F0020F9BB2CC
:10275800F6D06B23037340F2E93302E0002B00F05C
:10276800DE870289013B12F0010F9BB2F6D0037B92
:10277800019B586940F2E93302E0002B00F0CB8757
:102788000289013B12F0020F9BB2F6D000230373BB
:1027980040F2E9330DE000BF90640020946400200B
:1027A80010E000E000ED00E08C640020002B00F059
:1027B800B2870289013B12F0010F9BB2F6D0037B6E
:1027C800019B9B6913B11A689B889361DFF8449257
:1027D8008F48DFF844E24FF0640A4FF0100C4FF4D2
:1027E8007A76D9F80430C3F30803002B40F0F48557
:1027F800EFF31183002B40F0EF852168826800BF5A
:1028080023689942F9D12F6806FB07F39B1AB3FB9B
:10281800F7F306FB013101270091D9F80430C3F31F
:102828000803002B40F09384EFF31183002B40F052
:102838008E842368816800BF22689342F9D1D5F855
:1028480000B006FB0BF2521AB2FBFBF206FB0323A5
:10285800009A9B1AB3F57A7FDFD3BAF1010AC0D187
:10286800019A137C012B00F01687022B44D193693F
:1028780013B11A689B881385019B586940F2E933A4
:1028880002E0002B00F053870289013B12F0020F8F
:102898009BB2F6D06B23037340F2E93302E0002BBE
:1028A80000F045870289013B12F0010F9BB2F6D078
:1028B800037B019B586940F2E93302E0002B00F0EA
:1028C80032870289013B12F0020F9BB2F6D0012336
:1028D800037340F2E93302E0002B00F024870289F9
:1028E800013B12F0010F9BB2F6D0037B019B9B6961
:1028F80013B11A689B889361DFF818914448DFF890
:1029080018E14FF00F0A4FF0100C4FF47A76D9F80F
:102918000430C3F30803002B40F07B85EFF31183E9
:10292800002B40F076852168826800BF23689942B1
:10293800F9D12F6806FB07F39B1AB3FBF7F306FBE5
:10294800013101270091D9F80430C3F30803002BA3
:1029580040F01B84EFF31183002B40F016842368AA
:10296800816800BF22689342F9D1D5F800B006FB10
:102978000BF2521AB2FBFBF206FB0323009A9B1AD6
:10298800B3F57A7FDFD3BAF1010AC0D1019991F882
:102998004F200B7C042A34BF18261A26012B00F07E
:1029A8009786022B4AD18B6913B11A689B881385C5
:1029B800019B40F2E932586902E0002A00F0BF8624
:1029C8000389013A13F0020F92B2F6D01B23037366
:1029D80040F2E93202E0002A00F0B1860389013AA8
:1029E80013F0010F92B2F6D0037B019B40F2E9325B
:1029F800586902E0002A00F09E860389013A13F024
:102A0800020F92B2F6D0067340F2E93309E000BF34
:102A180010E000E000ED00E08C640020002B00F0E6
:102A28008A860289013B12F0010F9BB2F6D0037B24
:102A3800019B9B6913B11A689B889361DFF83C92EC
:102A48008D48DFF83CE24FF00F0A4FF0100C4FF4BE
:102A58007A76D9F80430C3F30803002B40F0828457
:102A6800EFF31183002B40F07D842168826800BF5A
:102A780023689942F9D12F6806FB07F39B1AB3FB29
:102A8800F7F306FB013101270091D9F80430C3F3AD
:102A98000803002B40F09783EFF31183002B40F0DD
:102AA80092832368816800BF22689342F9D1D5F8E0
:102AB80000B006FB0BF2521AB2FBFBF206FB032333
:102AC800009A9B1AB3F57A7FDFD3BAF1010AC0D115
:102AD800019A137C012B00F0F185022B44D19369F4
:102AE80013B11A689B881385019B586940F2E93332
:102AF80002E0002B00F02B860289013B12F0020F46
:102B08009BB2F6D01C23037340F2E93302E0002B9A
:102B180000F01D860289013B12F0010F9BB2F6D02E
:102B2800037B019B586940F2E93302E0002B00F077
:102B38000A860289013B12F0020F9BB2F6D01823D5
:102B4800037340F2E93302E0002B00F0FC850289B0
:102B5800013B12F0010F9BB2F6D0037B019B9B69EE
:102B680013B11A689B889361DFF810914248DFF827
:102B780010E14FF00F0A4FF0100C4FF47A76D9F8A5
:102B88000430C3F30803002B40F00984EFF31183EA
:102B9800002B40F004842168826800BF23689942B2
:102BA800F9D12F6806FB07F39B1AB3FBF7F306FB73
:102BB800013101270091D9F80430C3F30803002B31
:102BC80040F02483EFF31183002B40F01F83236828
:102BD800816800BF22689342F9D1D5F800B006FB9E
:102BE8000BF2521AB2FBFBF206FB0323009A9B1A64
:102BF800B3F57A7FDFD3BAF1010AC0D101990B7C12
:102C080091F84E60012B00F02B85022B4AD18B697D
:102C180013B11A689B881385019B40F2E932586901
:102C280002E0002A00F09B850389013A13F0020FA5
:102C380092B2F6D01A23037340F2E93202E0002A76
:102C480000F08D850389013A13F0010F92B2F6D096
:102C5800037B019B40F2E932586902E0002A00F048
:102C68007A850389013A13F0020F92B2F6D00673FF
:102C780040F2E93309E000BF10E000E000ED00E0B9
:102C88008C640020002B00F066850289013B12F05D
:102C9800010F9BB2F6D0037B019B9B6913B11A68A5
:102CA8009B889361DFF83C928D48DFF83CE24FF057
:102CB8000F0A4FF0100C4FF47A76D9F80430C3F3AA
:102CC8000803002B40F03283EFF31183002B40F010
:102CD8002D832168826800BF23689942F9D12F6843
:102CE80006FB07F39B1AB3FBF7F306FB0131012739
:102CF8000091D9F80430C3F30803002B40F0A382F5
:102D0800EFF31183002B40F09E822368816800BF97
:102D180022689342F9D1D5F800B006FB0BF2521A9B
:102D2800B2FBFBF206FB0323009A9B1AB3F57A7FEA
:102D3800DFD3BAF1010AC0D101990B7C91F8506038
:102D4800012B00F08384022B43D18B6913B11A68DD
:102D58009B881385019B40F2E932586902E0002AFA
:102D680000F005850389013A13F0020F92B2F6D0FC
:102D78001923037340F2E93202E0002A00F0F784D5
:102D88000389013A13F0010F92B2F6D0037B019B3D
:102D980040F2E932586902E0002A00F0E48403892D
:102DA800013A13F0020F92B2F6D0067340F2E933FB
:102DB80002E0002B00F0D7840289013B12F0010FDA
:102DC8009BB2F6D0037B019B9B6913B11A689B8861
:102DD8009361DFF810914248DFF80CE14FF0640A84
:102DE8004FF0100C4FF47A76D9F80430C3F3080387
:102DF800002B40F06583EFF31183002B40F06083D4
:102E08002168826800BF23689942F9D12F6806FBC0
:102E180007F39B1AB3FBF7F306FB01310127009177
:102E2800D9F80430C3F30803002B40F02982EFF3EC
:102E38001183002B40F024822368816800BF226838
:102E48009342F9D1D5F800B006FB0BF2521AB2FB47
:102E5800FBF206FB0323009A9B1AB3F57A7FDFD3B4
:102E6800BAF1010AC0D1019A137C012B00F00A843F
:102E7800022B4BD1936913B11A689B881385019B68
:102E8800586940F2E93302E0002B00F078840289A7
:102E9800013B12F0020F9BB2F6D03723037340F2C6
:102EA800E93302E0002B00F06A840289013B12F04A
:102EB800010F9BB2F6D0037B019B586940F2E933BE
:102EC80002E0002B00F057840289013B12F0020F48
:102ED8009BB2F6D01223037340F2E93309E000BF36
:102EE80010E000E000ED00E08C640020002B00F012
:102EF80042840289013B12F0010F9BB2F6D0037B9A
:102F0800019B9B6913B11A689B889361DFF8F8925B
:102F1800BB48DFF8F0E24FF00F0A4FF0100C4FF407
:102F28007A76D9F80430C3F30803002B40F0E48222
:102F3800EFF31183002B40F0DF822168826800BF25
:102F480023689942F9D12F6806FB07F39B1AB3FB54
:102F5800F7F306FB013101270091D9F80430C3F3D8
:102F68000803002B40F0A981EFF31183002B40F0F8
:102F7800A4812368816800BF22689342F9D1D5F8FB
:102F880000B006FB0BF2521AB2FBFBF206FB03235E
:102F9800009A9B1AB3F57A7FDFD3BAF1010AC0D140
:102FA800019A137C012B00F06583022B44D19369AD
:102FB80013B11A689B881385019B586940F2E9335D
:102FC80002E0002B00F0E2830289013B12F0020FBD
:102FD8009BB2F6D03823037340F2E93302E0002BAA
:102FE80000F0D4830289013B12F0010F9BB2F6D0A6
:102FF800037B019B586940F2E93302E0002B00F0A3
:10300800C2830289013B12F0020F9BB2F6D0012362
:10301800037340F2E93302E0002B00F0B483028925
:10302800013B12F0010F9BB2F6D0037B019B9B6919
:1030380013B11A689B889361DFF8CC817049714F8E
:103048004FF00F094FF0100E4FF47A70D8F8043093
:10305800C3F30803002B40F06B82EFF31183002BBE
:1030680040F0668222688E6800BF23689A42F9D1D0
:10307800D5F800C000FB0CF39B1BB3FBFCF300FB73
:10308800023300930126D8F80430C3F30803002B59
:1030980040F03081EFF31183002B40F02B8123683F
:1030A800D1F808A000BF22689342F8D1D5F800B043
:1030B80000FB0BFCACEB0A0CBCFBFBFC00FB03C3EA
:1030C800009A9B1AB3F57A7FDDD3B9F10109BDD116
:1030D80005B0BDE8F08FEFF311888CF31288816892
:1030E8000368DB0344BFCEF8007081682368DEF80C
:1030F80000205FFA88F888F31188D5F800801A4410
:1031080006FB08F35B1AB3FBF8F306FB0233FFF781
:1031180068BAEFF3118E88F31288B1683368DB035D
:1031280044BFCCF80000B1682368DCF800205FFADF
:103138008EFE8EF31188D5F800E01A4407FB0EF3D3
:103148005B1AB3FBFEF307FB0233FFF7E0BAEFF3BA
:1031580011888CF3128881680368DB0344BFCEF8BA
:10316800007081682368DEF800205FFA88F888F329
:103178001188D5F800801A4406FB08F35B1AB3FBE4
:10318800F8F306FB0233FFF763BBEFF311888CF308
:10319800128881680368DB0344BFCEF80070816839
:1031A8002368DEF800205FFA88F888F31188D5F8DC
:1031B80000801A4406FB08F35B1AB3FBF8F306FB1E
:1031C8000233FFF7DBBBEFF311888CF312888168B9
:1031D8000368DB0344BFCEF8007081682368DEF81B
:1031E80000205FFA88F888F31188D5F800801A441F
:1031F80006FB08F35B1AB3FBF8F306FB02335FE444
:1032080010E000E08C64002000ED00E0EFF311888E
:103218008CF3128881680368DB0344BFCEF8007022
:1032280081682368DEF800205FFA88F888F311883F
:10323800D5F800801A4406FB08F35B1AB3FBF8F3D1
:1032480006FB0233D2E4EFF311888CF3128881680D
:103258000368DB0344BFCEF8007081682368DEF89A
:1032680000205FFA88F888F31188D5F800801A449E
:1032780006FB08F35B1AB3FBF8F306FB023353E5CE
:10328800EFF311888CF3128881680368DB0344BF6D
:10329800CEF8007081682368DEF800205FFA88F8AD
:1032A80088F31188D5F800801A4406FB08F35B1AE6
:1032B800B3FBF8F306FB0233CDE5EFF311888CF38B
:1032C800128881680368DB0344BFCEF80070816808
:1032D8002368DEF800205FFA88F888F31188D5F8AB
:1032E80000801A4406FB08F35B1AB3FBF8F306FBED
:1032F80002334DE6EFF3118A8EF312888A680B6861
:10330800DB0344BF3E608A682368D7F800C05FFAD1
:103318008AFA8AF31188D5F800A09C4400FB0AF3C6
:103328009B1AB3FBFAF300FB0C33C9E6EFF31182E7
:103338008CF3128887680368D90303D50123CEF874
:10334800003087682368DEF80010D2B282F3118853
:103358002A68194406FB02F3DB1BB3FBF2F306FBF6
:103368000131C4E4EFF311828CF312888768036893
:10337800D90303D50123CEF8003087682368DEF827
:103388000010D2B282F311882A68194406FB02F3AE
:10339800DB1BB3FBF2F306FB0131FFF774BBEFF362
:1033A80011828CF3128887680368D90303D5012337
:1033B800CEF8003087682368DEF80010D2B282F3B6
:1033C80011882A68194406FB02F3DB1BB3FBF2F3EE
:1033D80006FB0131FFF7EDBBEFF311828CF3128886
:1033E80087680368D90303D50123CEF800308768BE
:1033F8002368DEF80010D2B282F311882A681944D3
:1034080006FB02F3DB1BB3FBF2F306FB0131FFF70C
:1034180002BAEFF311828CF3128887680368D90324
:1034280003D50123CEF8003087682368DEF8001042
:10343800D2B282F311882A68194406FB02F3DB1B17
:10344800B3FBF2F306FB0131FFF77BBAEFF311820E
:103458008CF3128887680368D90303D50123CEF853
:10346800003087682368DEF80010D2B282F3118832
:103478002A68194406FB02F3DB1BB3FBF2F306FBD5
:103488000131FFF791B8EFF3118288F31288B06821
:103498003368D90303D50123CCF80030B06823681A
:1034A800DCF80010D2B282F311882A68194407FBAD
:1034B80002F31B1AB3FBF2F307FB0131FFF70AB95A
:1034C800EFF311828CF3128887680368D90303D558
:1034D8000123CEF8003087682368DEF80010D2B2E6
:1034E80082F311882A68194406FB02F3DB1BB3FB3D
:1034F800F2F306FB013191E4EFF311828CF31288A9
:1035080087680368D90303D50123CEF8003087689C
:103518002368DEF80010D2B282F311882A681944B1
:1035280006FB02F3DB1BB3FBF2F306FB013112E5EA
:10353800EFF311868EF31288D1F808C00B68DA030E
:1035480003D501233B60D1F808C023683A68F6B276
:1035580086F311882E681A4400FB06F3A3EB0C03CC
:10356800B3FBF6F300FB023300938BE51D09013D25
:10357800052D03F00F0300F2B5808D4A32F81500CF
:1035880040FA03F2D40740F1AD80012404FA03F3B2
:10359800013B184031F0B2FE864B874A5B5D184408
:1035A80012EBC00500F09E8052F83000AE88038A06
:1035B80033407EF486AF00F138428049EB71920ABD
:1035C8008A5C02F01F0352092021022A04FA03F33D
:1035D800A97100F0E880032A00F0E080012A00F0D9
:1035E800D880002302A90393029626F0BFFB019915
:1035F800734B41F80C3F28462AF08CFAAB88B3FA93
:1036080083F3C3F11F03581C3EF45BAF012202FA97
:1036180003F36C490A681343019A0B60137C012B6E
:103628007EF454AF10468023417D90F914006B223C
:10363800FEF7CAFEFEF791BF10460723417D90F9B9
:1036480014006822FEF7C0FEFFF71FB8084633468D
:103658001922497D90F91400FEF7B6FEFFF7B9BBB1
:10366800084633461A22497D90F91400FEF7ACFE4D
:10367800FFF718BB10463822417D90F91400FEF779
:10368800A3FED9E410461223417D90F91400372295
:10369800FEF79AFE3AE410466B22417D90F9140039
:1036A800FEF792FEFFF728B910465346417D90F980
:1036B80014006B22FEF788FEFFF788B8104618231F
:1036C800417D90F914001C22FEF77EFEFFF74CBAEC
:1036D800084633461B22497D90F91400FEF774FE14
:1036E800FFF7ACB90199364B41F80C3F00202AF09E
:1036F80011FA01238DE703F093F8FEF728BF03F0D2
:103708008FF8FEF707BF03F08BF8FEF7B8BF03F09A
:1037180087F8FEF797BF03F083F8FFF751B803F077
:103728007FF8FFF725B803F07BF8FFF7DFB803F061
:1037380077F8FFF7BEB803F073F8FFF779B903F02D
:103748006FF8FFF752B903F06BF8FFF707BA03F009
:1037580067F8FFF7E6B903F063F8FFF79DBA03F0DF
:103768005FF8FFF776BA03F05BF8FFF72CBB03F0BE
:1037780057F8FFF70CBB03F053F8FFF7C1BB03F092
:103788004FF8FFF799BB03F04BF84FE403F048F804
:103798002FE40D4A51690B43536122E70A4AD16964
:1037A8000B43D3611DE7084A91690B43936118E7FE
:1037B800D48B0308E08B030850530020548F030870
:1037C8002906000800040140001002401749184B60
:1037D800184A194810B4D1F8884044F47004C1F864
:1037E80088401C6844F001041C605C6822405A60F0
:1037F8001A6822F0847222F480321A601A6822F45D
:1038080080221A605A6822F4FE025A60DA6A22F0AC
:103818000F02DA621A6B002410404FF0006218633E
:103828009C608A605DF8044B704700BF00ED00E0C3
:10383800001002400CC07FF8CCFC00FF0B4B0022AC
:1038480010B4027203F1DC04012102E0072A09DC4A
:103858009979890702D51979815401329C4203F17B
:103868001403F3D15DF8044B704700BF5C8F030865
:1038780024230370704700BF30B4012302251424A9
:1038880015212222057244704171C27003700371C0
:10389800837030BC704700BF2DE9F0410B78057B81
:1038A800DB43DFB200F1130200F11D0302F8015FF0
:1038B8009342FBD1DFF890E000F12701002203F8E2
:1038C800012F9942FBD114210524002647FA04F35D
:1038D80003F00103002B1E4414BF4FF019084FF0EA
:1038E8000A0814F0010FF6B214BFAC464FF0000CF2
:1038F8000023CA1810FA82F20133434582F814C033
:10390800F7D15A1E92B20132013C8B18621C9BB24D
:1039180001D01946DAE716F0010F14BF19240A245A
:103928000022991810FA81F10132A2420D75F8D1DE
:1039380013449BB25A1C0344002192B21975AEF885
:1039480000200261BDE8F081701E00202DE9F04FD3
:10395800DFF890A0BAF802300B3383B01FFA83F96E
:1039680001F1060B4FF001084FF0000C002711F889
:1039780001EB3E464C460122A4F10B039BB2019198
:1039880005E001339BB2017B29759C4208D0C5181C
:10399800002AF6D1C51801339BB29C422A75F6D18C
:1039A80003190136092F019983F814C0F6B20CD017
:1039B800092E15D008FA07F313EA0E0F14BF0122D7
:1039C80000220C34A4B20137D6E709F17809594529
:1039D8001FFA89F9CAD1AAF802C003B0BDE8F08F6E
:1039E8000022EEE7701E00202DE9F047DFF85C802A
:1039F800B8F8043004331FFA83FC01F109094FF0C9
:103A0800010E11F8017B64460026231F0EFA06F208
:103A18009BB23A40C2B1B0F80CA0C51801339BB2B2
:103A28009C4285F814A0F5D101360434082EA4B2BE
:103A3800EBD10CF1200C49451FFA8CFCE1D1002395
:103A4800A8F80430BDE8F0879246E6E7701E00202B
:103A580010B50168047B0A680223A3401A420AD001
:103A6800054A406800241470026822F0010212041A
:103A7800120C02604B6010BDBF260020436A8269A9
:103A8800D154436A0169826B01338B4228BF0023FA
:103A98004362002A2FD0EFF31181502383F3128859
:103AA800836B1A68D2072CD470B45E686EB9456A05
:103AB800826A954217D084691444DC600ED9AA1A28
:103AC8005A608562002280F854201A6842F0010288
:103AD800C9B21A6081F3118870BC70470469A21AD0
:103AE8005A608662EEE7012380F85430C9B281F348
:103AF800118870BC7047026D136843F0800313602F
:103B08007047C9B281F31188704700BF426B10B487
:103B180062B1436CC2684469D11A013B615C5DF8CB
:103B2800044B08BF13464364C8B27047016A43692F
:103B3800C4685B5C0131A14228BF114601625DF88F
:103B4800044BD8B2704700BF836B13B190F8540090
:103B58007047836A406A181AB0FA80F040097047C3
:103B6800416A836A99420AD3CB1A816B026961B1AF
:103B78004968501E0B4483420AD2C01A7047026932
:103B88001144CB1A816B0029F2D1501EC01A70471C
:103B980000207047436B43B1426C5B6893422FBF70
:103BA800981AC0689B1AC0187047C269036A9A427B
:103BB8002FBFD01AC0688018C01A70470A4B30B59A
:103BC80003F1140493F900205D78072AC8BF143A5A
:103BD800811804330D7313F8025C855413F8012C13
:103BE8000A76A342EED130BD206C030803682DE9A4
:103BF800F041DF691FB13B46BDE8F0411847002A94
:103C0800164611DD04460D460E4400E023689B6805
:103C1800204698470028F9D0236815F8011B1B682F
:103C280020469847AE42F1D1BDE8F0810023232217
:103C3800027043708370C37070472D2343702E2326
:103C480003712F23C371704700232622036002707B
:103C5800272282700122436002718371704700BF7E
:103C68002DE9F0470569C3681D4028D00F46064670
:103C78004FF000484FF00009B5FA85F328FA03F22F
:103C8800D2431B3B32611540042B16D8DFE803F002
:103C98003129211903007B6A002B32D003F1FF3A46
:103CA8001FFA8AFAC7F824903C6A34B12368204680
:103CB800514698476468002CF8D1002DDCD1BDE846
:103CC800F0873868716B036889B29847002DD3D1A3
:103CD800F5E77868B16B036889B29847002DCBD1B6
:103CE800EDE7B868F16B036889B29847002DC3D136
:103CF800E5E7F868316C036889B29847002DBBD1B5
:103D0800DDE7F36A1FFA83FACEE700BF30B5044651
:103D1800006D61710368A26823F00103036087B036
:103D2800A379009213F004023DD04FF4805213F0AF
:103D38000203019244D102934FF48063002203935B
:103D480011F00103059237D1049308238D076946C2
:103D580048BF049326F054FA6079236DA17900F0E6
:103D68000202002A15BF4FF440324FF480324FF45C
:103D78000034002410F0010F586808BF2246CC0711
:103D88004CBF024320EA02025A609A6809074CBFF6
:103D980042F0080222F008029A601A6842F0010212
:103DA8001A6007B030BD13F0020301920BD04FF434
:103DB800005513460295C1E7042304930C23C5E775
:103DC8004FF40053B7E70293B8E700BF10B50446B5
:103DD800006DA160036823F001030360A37986B036
:103DE80013F00402009141D04FF4805213F0020303
:103DF800019244D102934FF4806362790393D1070F
:103E08004FF000030493059345BF0423049308234C
:103E18000C236946920748BF049326F0F1F96079AC
:103E2800236DA17900F00202002A15BF4FF4403239
:103E38004FF480324FF40034002410F0010F58681A
:103E480008BF2246CC074CBF024320EA02025A6050
:103E58009A6809074CBF42F0080222F008029A60EB
:103E68001A6842F001021A6006B010BD13F002038E
:103E7800019207D04FF4005113460291BDE74FF469
:103E88000053B7E70293B8E72DE9F04F013085B04A
:103E9800C3B203938E4D8F4F8F4C904E0A230293DB
:103EA8003220DFF8409229F091FA4FF4FA7A4FF075
:103EB800100C4FF47A70D9F80430C3F30803002BC0
:103EC80040F0C880EFF31183002B40F0C3802968CD
:103ED800A26800BF2B689942F9D1D7F800E000FB2F
:103EE8000EF39B1AB3FBFEF300FB01314FF0010EFA
:103EF8000191D9F80430C3F30803002B40F08E80F9
:103F0800EFF31183002B40F089802B68A16800BF74
:103F18002A689342F9D1D7F800B000FB0BF2521A85
:103F2800B2FBFBF200FB0323019A9B1AB3F57A7FDD
:103F3800DFD3BAF1010ABED1039B002B40F0C48045
:103F48004FF47A7ADFF89C9150464FF0100CD9F86C
:103F58000430C3F30803002B40F09980EFF311837A
:103F6800002B40F094802968A26800BF2B68994212
:103F7800F9D1D7F800E000FB0EF39B1AB3FBFEF370
:103F880000FB01314FF0010E0191D9F80430C3F361
:103F980008033BBBEFF3118323BB2B68A16800BF69
:103FA8002A689342F9D1D7F800B000FB0BF2521AF5
:103FB800B2FBFBF200FB0323019A9B1AB3F57A7F4D
:103FC800E3D3BAF1010AC2D1029B013B02937FF409
:103FD80067AF4349434B4448444A0860DA6005B038
:103FE800BDE8F08FEFF311888CF31288A16823687D
:103FF800DB0344BFC6F800E0A1682B6832685FFAAB
:1040080088F888F31188D7F800801A4400FB08F371
:104018005B1AB3FBF8F300FB0233CDE7EFF311882B
:104028008CF31288A1682368DB0344BFC6F800E05C
:10403800A1682B6832685FFA88F888F31188D7F886
:1040480000801A4400FB08F35B1AB3FBF8F300FB8B
:10405800023369E7EFF311828CF31288D4F808E091
:104068002368D90303D501233360D4F808E02B680B
:104078003168D2B282F311883A68194400FB02F31E
:10408800A3EB0E03B3FBF2F300FB01312EE7EFF3D2
:1040980011828CF31288D4F808E02368D90303D579
:1040A80001233360D4F808E02B683168D2B282F378
:1040B80011883A68194400FB02F3A3EB0E03B3FB23
:1040C800F2F300FB01315DE718462BF015F937E7ED
:1040D800906400209464002010E000E08C640020CC
:1040E800FC9F002000ED00E0EFBEADDE0400FA0505
:1040F80038B5434B5A899989914224BF00225A8185
:10410800198ADA89914224BF0022DA81DA788AB3DF
:10411800072A2FD03B493C4D91F853000124002138
:104128000A282C709C70D9713DD00C2865D0DFED21
:10413800377A8ABB364C9FED370AA278002918BF18
:10414800F0EE407A062A04D8334901EB820191ED5A
:10415800050A217959B3013A032A4DD8F7EE007AB6
:1041680087EE800A31F0ACFC2388984228BF1846B5
:10417800208038BDD97921B198780428B8BF0420A7
:104188009870204890F853000A280CD00C28CED1FB
:10419800DFED227A002ACDD0072ACBD00A282CD1ED
:1041A800DFED1F7AC6E70A20DFED1E7AC1E79B78AC
:1041B800154A07EE103A1178B8EEC77A27EE277A33
:1041C80007EE901AF8EEE77A67EE877AB4EEE70A18
:1041D800F1EE10FA10DDC0EE077AFDEEE77A17EE81
:1041E800903A102BA8BF1023012BB8BF0123DBB2D4
:1041F8008B4238BF0B46137038BDDFED0B7A99E759
:104208008054002094540020904100206F120339FC
:104218001C5900206F120338206C03080AD7A339F1
:104228000F506E3A5304E9386F12833A2DE9F0477C
:10423800A84FA94E17F0E4FCBE421ED2DFF8148343
:10424800DFF814934446258862197DB14A450DD29A
:10425800052D0BD933886188C3F30B03994200F00D
:10426800DE80144625886219002DEFD1716830462A
:104278001436FCF77BFCBE42E4D3984A1378A3F1CA
:10428800170102290FD9964911F83300002840F088
:10429800F280D8000144497829B1924911F83330A5
:1042A800002B00F01081904B5A78022A40F2DD80F2
:1042B80000228E495A701A788D48022A016000F24D
:1042C800D08002EB82018B4BC2EBC10203EB4203AD
:1042D800998C5A8C884C9142236001D300225A84CD
:1042E800864B9A78042A00F0E58032B91A88B2F52C
:1042F800F07F84BF4FF4F0721A80814DFFF7F8FE0B
:104308002B68804A1A40002A00F0E080D80700F1A4
:10431800CC80590400F1C4801A0700F1BC809B04CA
:1043280000F1B2802AF0C6F810B977482BF086F968
:104338008020FCF751FC4FF40070FCF74DFC4FF463
:104348008020FCF749FC4FF00070FCF745FC4FF06B
:104358008060FCF741FC4FF00060FCF73DFC24F066
:104368002DFF00213022694832F067FB206823F0D6
:1043780035FE674B276803F1500102E00433994288
:104388006DD01A78002AF9D19C78D8788442F5D271
:104398006049614B0D79614961480A70614E624C10
:1043A8000460C822642111FB0521002259609A602B
:1043B800DA601A615A619A61DA6183F8202083F819
:1043C800212037601AF0C6FB584B9FED595A1B88BD
:1043D800584A9FED596A5079584906EE903AF8EED6
:1043E800E66A1388C5EE265A07EE103A5388127902
:1043F800C1ED005A07EE903AB8EEC77A504BF8EE86
:10440800E77A18725A7227EE067A67EE867ABDE85E
:10441800F04783ED017AC3ED007A17F0D9BB6379D1
:104428009B077FF41EAF716894F804A03046FCF730
:104438009DFB3388BAEB133F04D01436BE42FFF419
:1044480001AF1AE773887068AA1FC3F30B039A4277
:1044580004F10601A8BF1A4631F0F2F9EDE701228E
:1044680096E700221A70234B32E7204902EB4202FA
:1044780001EB82011FE7D8000C186468002C7FF458
:1044880009AF1724147005E72E48FCF7A5FB402058
:10449800FCF7A2FB46E72C48FCF79EFB2B683EE79F
:1044A8002A48FCF799FB2B6836E72948FCF794FB68
:1044B8002B682EE79A8AB2F57A7FBFF41EAF4FF4C5
:1044C8007A729A8219E718231370ECE643F0010315
:1044D8002B601BE734CC0308C0C70308E83B002067
:1044E80030930308606F03083442002040420020E4
:1044F800B0470020525D0020AC4700201C59002026
:104508008C5E00200960000240600020181F002017
:10451800D8340020DC510020D44900204C1C002055
:104528005C1F00204C1F0020A2410020A821002071
:10453800C0C9FB48DC1F002017B7D138AC210020C8
:10454800DC4F00200940000201600002092000023F
:104558000860000202F003080000040838B50C4C9B
:104568000C4DAC4206D2616820461434FCF7FEFAC2
:10457800AC42F8D3084A094B094C14600022094997
:104588001A705A7008480860BDE8384022F0F0BA3E
:10459800C0C7030834CC0308AC47002034420020CD
:1045A800525D0020B047002040420020054B10B566
:1045B8009A68054C2178501C09B99A6010BD0246CA
:1045C800F8E700BF701E0020BF260020F0B50C29B8
:1045D8002BD8DFE801F06F2A2A2A4C2A2A2A2B2A0C
:1045E8002A2A0700046AB2F80CE097881668674D13
:1045F80024F480540462036A4468C16923F40053B4
:1046080043EA0E3321F4E641A84243EA073341EA7C
:10461800062100F0B58005F50065A84200F0B080DD
:1046280092684460C16102640362F0BD046A9689BD
:104638009588D2F800E0554F24F480740462036A28
:104648004468C16923F4007343EA062321F0730127
:10465800B84243EA052341EA0E017ED04C4DA842F8
:104668007BD092684460C161C2630362F0BD046A92
:1046780096899588D2F800E0444F24F0100404622B
:10468800036A4468816923F0200321F0807143EABA
:10469800061321F4E641B84243EA051341EA0E2124
:1046A80048D03B4DA84245D09268446081618263FE
:1046B8000362F0BD046A9389B2F804E01768334EC8
:1046C80024F001040462056A4468816943EA0E0320
:1046D80021F4803125F002059BB221F07301B0422C
:1046E80043EA050341EA070114D0294DA84211D035
:1046F80005F54065A8420DD005F58065A84209D0AA
:1047080005F58065A84205D09268446081614263DE
:104718000362F0BDD689158A578A23F0080333430C
:104728003D43D68824F4407423F00403ADB23343E8
:104738002C43E9E7D589178AD68823F0800343EA12
:10474800051324F44064558A23F0400344EA87049F
:1047580043EA061344EA8504A6E7D589178AD6886A
:1047680023F4006343EA052324F44054558A23F4D0
:10477800806344EA071443EA062344EA051470E711
:10478800158A24F4804444EA851449E7002C014042
:10479800003401402DE9F04F4FF48C72002183B0B2
:1047A8007848794CDFF80492784D794E794FDFF8E4
:1047B800008232F042F978487849DFF8F8E1DFF80A
:1047C800F8C100221359834200F0C180B3F1804F31
:1047D80000F0BF80AB4200F0C880B34200F0C78051
:1047E800BB4200F0C680734500F0C580634500F009
:1047F800C480434500F0C380DFF8C0A153457ED094
:104808000AF5806A534508BF092379D01432F02A83
:10481800D8D15D4C624D634E604F04F1F00802E060
:104828001434A04568D0A379002BF9D023794FEA36
:10483800131909F1FF39B9F1050F03F00F03EFD888
:1048480035F8190040FA03F2D207E9D54FF0010A0A
:104858000AFA03F3013B184030F050FD16F809300E
:104868005149184411EBC002DAD051F83000DFF892
:1048780050E1217A00F138439B0A1EF8033003F017
:104888001F0E5B09022B0AFA0EFA69D0032B62D0BD
:10489800012B03D17B694AEA03037B619388009368
:1048A800B3FA83F3C3F11F039BB2DA0800EB820269
:1048B80003F00703D2F820E09B004FF00F0C0CFA2E
:1048C80003FC2EEA0C0EC2F820E0D2F820E001FA30
:1048D80003F343EA0E0313626946002302221434E9
:1048E8008DF804208DF805308DF806308DF80730E6
:1048F80025F03CFAA04596D103B0BDE8F08F082317
:1049080009EBC3034FF0010B93F834A00AF01F031F
:104918004FEA5A1ABAF1020F0BFA03F30BD0BAF1A5
:10492800030F0ED0DA457FF471AFD1F814A043EA33
:104938000A034B616AE7D1F818A043EA0A038B61BE
:1049480064E7D1F81CA043EA0A03CB615EE70023C1
:10495800D6E70123D4E7FB694AEA0303FB619DE735
:10496800BB694AEA0303BB6198E70223C8E703234C
:10497800C6E70423C4E70523C2E70623C0E70723E5
:10498800BEE700BFE42400205C8F03080004004059
:104998000008004000100040002C014000100240B8
:1049A800D48B0308E08B030850530020206C0308C5
:1049B8000040014000140040003401400044014020
:1049C800548F0308002867D003682DE9F04F03F1DE
:1049D80038445C4EA40A0125345D04F01F066409BE
:1049E800022C05FA06F558D0032C00F0A580012CFE
:1049F80058D08088B0FA80F4C4F11F04A4B2E50846
:104A080003EB850504F007042E6AA4000F27A740CE
:104A180026EA07062E622E6A01F00307A2407C1ED2
:104A28003243012CC1F3810CC1F300182A62C1F38F
:104A380041113CD9C60700F18980850700F19580AE
:104A4800440700F1A380020700F1B180C60600F117
:104A5800BF80850600F1CD80440600F1DB800206A8
:104A680000F1E980C60500F1F780850500F10581B0
:104A7800440500F11381020500F12181C60400F10B
:104A88002F81850400F13D81440400F14B8102042B
:104A980000F15981BDE8F08F70472B4CA66935436A
:104AA800A561A6E7284C666935436561A1E700243E
:104AB80022464FF0010E4FF0030904E00132102A9C
:104AC80004F10204E6D00EFA02F636EA0005F5D142
:104AD800D3F808A009FA04F5ED430AEA050AC3F871
:104AE80008A0D3F808B00CFA04FA4AEA0B0AC3F88B
:104AF80008A0B3F804A01FFA8AFA2AEA06069E80DC
:104B0800B3F804A008FA02F646EA0A06B6B29E808E
:104B18001E682E401E60D3F800A007FA04F646EA85
:104B28000A061E60D3F80CA001FA04F605EA0A0A80
:104B380046EA0A05DD60C1E7034CE6693543E561ED
:104B480057E700BF548F0308001002401A6822F08C
:104B580003021A601A683A431A60DA6822F00302FC
:104B68000A438507DA607FF56BAF1A6822F00C02FA
:104B78001A601A6842EA87021A60DA6822F00C02A0
:104B880042EA81024407DA607FF55DAF1A6822F0D5
:104B980030021A601A6842EA07121A60DA6822F0CC
:104BA800300242EA0112DA6002077FF54FAF1A6855
:104BB80022F0C0021A601A6842EA87121A60DA689C
:104BC80022F0C00242EA8112C606DA607FF541AFE0
:104BD8001A6822F440721A601A6842EA07221A60B8
:104BE800DA6822F4407242EA01228506DA607FF52B
:104BF80033AF1A6822F440621A601A6842EA8722C0
:104C08001A60DA6822F4406242EA81224406DA60D5
:104C18007FF525AF1A6822F440521A601A6842EAF2
:104C280007321A60DA6822F4405242EA0132DA6046
:104C380002067FF517AF1A6822F440421A601A6814
:104C480042EA87321A60DA6822F4404242EA813244
:104C5800C605DA607FF509AF1A6822F440321A6097
:104C68001A6842EA07421A60DA6822F4403242EAD5
:104C780001428505DA607FF5FBAE1A6822F440220E
:104C88001A601A6842EA87421A60DA6822F44022F7
:104C980042EA81424405DA607FF5EDAE1A6822F4F3
:104CA80040121A601A6842EA07521A60DA6822F457
:104CB800401242EA0152DA6002057FF5DFAE1A6857
:104CC80022F440021A601A6842EA87521A60DA68C7
:104CD80022F4400242EA8152C604DA607FF5D1AE7E
:104CE8001A6822F040721A601A6842EA07621A606B
:104CF800DA6822F0407242EA01628504DA607FF5E0
:104D0800C3AE1A6822F040621A601A6842EA8762E3
:104D18001A60DA6822F0406242EA81624404DA608A
:104D28007FF5B5AE1A6822F040521A601A6842EA56
:104D380007721A60DA6822F0405242EA0172DA60B9
:104D480002047FF5A7AE1A6822F040421A601A687A
:104D580042EA87771F60DA6822F0404242EA8171AE
:104D6800D960BDE8F08F00BF03682DE9F04F03F16B
:104D78003845644EAD0A0124755D05F01F066D09BE
:104D8800022D04FA06F400F0A280032D00F0A4809E
:104D9800012D52D08088B0FA80F4C4F11F04A4B267
:104DA800E50803EB850504F007042E6AA4000F2725
:104DB800A74026EA07062E622E6A01F0030702FAC8
:104DC80004F47A1E3443012AC1F3810CC1F300189C
:104DD8002C62C1F3411135D9C60700F197808507C8
:104DE80000F1A380440700F1B180020700F1BF8001
:104DF800C60600F1CD80850600F1DB80440600F18F
:104E0800E980020600F1F780C60500F105818505F5
:104E180000F11381440500F12181020500F12F8181
:104E2800C60400F13D81850400F14B81440400F182
:104E38005981020455D4BDE8F08F334D6E6934436F
:104E48006C61A7E7002422464FF0010E4FF00309DA
:104E580004E00132102A04F10204ECD00EFA02F642
:104E680036EA0005F5D1D3F808A009FA04F5ED43B0
:104E78000AEA050AC3F808A0D3F808B00CFA04FA3D
:104E88004AEA0B0AC3F808A0B3F804A01FFA8AFA82
:104E98002AEA06069E80B3F804A008FA02F646EA53
:104EA8000A06B6B29E801E682E401E60D3F800A087
:104EB80007FA04F646EA0A061E60D3F80CA001FABF
:104EC80004F605EA0A0A46EA0A05DD60C1E70E4D5E
:104ED800AE693443AC615DE70B4DEE693443EC6178
:104EE80058E71A6822F040421A601A6842EA87773F
:104EF8001F60DA6822F0404242EA8171D960BDE859
:104F0800F08F00BF548F0308001002401A6822F087
:104F180003021A601A683A431A60DA6822F0030238
:104F28000A438507DA607FF55DAF1A6822F00C0244
:104F38001A601A6842EA87021A60DA6822F00C02DC
:104F480042EA81024407DA607FF54FAF1A6822F01F
:104F580030021A601A6842EA07121A60DA6822F008
:104F6800300242EA0112DA6002077FF541AF1A689F
:104F780022F0C0021A601A6842EA87121A60DA68D8
:104F880022F0C00242EA8112C606DA607FF533AF2A
:104F98001A6822F440721A601A6842EA07221A60F4
:104FA800DA6822F4407242EA01228506DA607FF567
:104FB80025AF1A6822F440621A601A6842EA87220A
:104FC8001A60DA6822F4406242EA81224406DA6012
:104FD8007FF517AF1A6822F440521A601A6842EA3D
:104FE80007321A60DA6822F4405242EA0132DA6083
:104FF80002067FF509AF1A6822F440421A601A685F
:1050080042EA87321A60DA6822F4404242EA813280
:10501800C605DA607FF5FBAE1A6822F440321A60E2
:105028001A6842EA07421A60DA6822F4403242EA11
:1050380001428505DA607FF5EDAE1A6822F4402258
:105048001A601A6842EA87421A60DA6822F4402233
:1050580042EA81424405DA607FF5DFAE1A6822F43D
:1050680040121A601A6842EA07521A60DA6822F493
:10507800401242EA0152DA6002057FF5D1AE1A68A1
:1050880022F440021A601A6842EA87521A60DA6803
:1050980022F4400242EA8152C604DA607FF5C3AEC8
:1050A8001A6822F040721A601A6842EA07621A60A7
:1050B800DA6822F0407242EA01628504DA607FF51C
:1050C800B5AE1A6822F040621A601A6842EA87622E
:1050D8001A60DA6822F0406242EA81624404DA60C7
:1050E8007FF5A7AE1A6822F040521A601A6842EAA1
:1050F80007721A60DA6822F0405242EA0172DA60F6
:1051080097E600BF10B50409013C052C17D80D4BD4
:1051180033F8142000F00F0042FA00F313F00103F3
:105128000DD0012303FA00F00138104030F0E6F802
:10513800054A064B125D104403EBC00010BD002069
:1051480010BD00BFD48B0308E08B03085053002028
:1051580001490248FEF784BDD425002000480140DB
:1051680001490248FEF77CBD84250020004001402B
:1051780001490248FEF774BD5C2500200008004084
:1051880001490248FEF76CBD3425002000040040A8
:1051980002494FF08040FEF763BD00BF0C25002098
:1051A80010B5064C06482146FEF75AFD04F1C80121
:1051B8000448BDE81040FEF753BD00BFE4240020BA
:1051C800002C01400044014001490248FEF748BD57
:1051D800E4240020002C01402DE9F0410468514DE1
:1051E800A30AAB4200F084800AD94F4DAB4277D076
:1051F8000135AB425FD0023DAB426DD0BDE8F081D6
:105208004A3DAB4270D00135AB4258D0B3F5801F50
:10521800F4D14FF0480E012647794FEA970C002940
:105228006AD0B000634685190227D4F80C809F40E5
:105238000CEB4503BFB23D4D03F1040C47EA0807E8
:1052480045F8231045F82C20E760EFF31181502230
:1052580082F31288821905EBC2021369002B32D03F
:1052680013620433821905EBC202576917B11F6034
:1052780053690433821905EBC202976917B11F609D
:1052880093690433821905EBC202D76917B11F600D
:10529800D36904330027CAB21F6082F311883044EF
:1052A80005EBC000036A8BB9E3684FF6FE72134042
:1052B800E360BDE8F0814FF4887E0626ACE74FF046
:1052C800980E0326A8E705EB0E03CBE7E36843F047
:1052D8000103E360BDE8F0814FF0C00E04269BE7B0
:1052E8004FF0E80E052697E74FF0700E022693E779
:1052F8004FF0200E00268FE7BF08022306FA03F0BE
:10530800BB40DB43E768094D9BB23B4087190CEB78
:10531800470CE3600CF1040345F82C1045F82320F2
:1053280093E700BF4B00100051001000E424002058
:1053380030B503685C4D18885C4CB4FBF2F2013957
:10534800013AAB4294B283B089B282B266D058486F
:10535800834263D0B3F1804F60D0A0F59830834288
:105368005CD000F58060834258D0524883425BD0BD
:1053780000F5806083427DD022F4407200F58C30C5
:1053880092B283421A80D9621C850ED0484A934251
:105398000BD002F54062934207D002F58062934237
:1053A80003D002F58062934201D100221A860122BD
:1053B8005A611A883C4992B242F001028B421A8023
:1053C80062D0B3F1804F61D03B4A934260D002F57E
:1053D800806293425ED002F5006293425CD002F58F
:1053E800806293425AD002F59032934258D002F527
:1053F8004062934256D002F5806293421ED002F575
:105408008062934208BF092219D002A84FF00123F5
:1054180040F8043D24F074FC03B030BD254822F068
:105428007002834292B2A3D101201A80D9621C85EE
:1054380058611A8892B202431A80C5E708221F4BA6
:1054480003EBC20301A893F835408DF8044001230B
:1054580000228DF805308DF807308DF8062024F0ED
:105468004FFC1B2CD8D1164B019301A824F048FC03
:1054780003B030BD01201A80D9621C8558611A8892
:1054880092B202431A809CE70022D8E70122D6E7AD
:105498000222D4E70322D2E70422D0E70522CEE78E
:1054A8000622CCE70722CAE7002C014000A24A04E2
:1054B800003401400010004000040040206C030844
:1054C80019010001204B98422DD0B0F1804F2CD00B
:1054D800A3F5943398422AD003F58063984228D0E4
:1054E80003F50063984226D003F58063984224D0E0
:1054F80003F59033984222D003F54063984220D0B8
:1055080003F58063984207D003F58063984208BF8B
:10551800092202D00020704708220C4B03EBC2037B
:1055280093F8340070470022F7E70122F5E70222DA
:10553800F3E70322F1E70422EFE70522EDE706226D
:10554800EBE70722E9E700BF002C0140206C0308C5
:105558002DE9F04F013085B0C3B203930B46029199
:105568008B4C8C4E002B00F09A8032208A4D8B4F4A
:10557800DFF82C9227F02AFF4FF4FA7A4FF0100C3C
:105588004FF47A70D9F80430C3F30803002B40F0C5
:10559800DE80EFF31183002B40F0D9802968A268E0
:1055A80000BF2B689942F9D1D7F800E000FB0EF351
:1055B8009B1AB3FBFEF300FB01314FF0010E019182
:1055C800D9F80430C3F30803002B40F08780EFF3C9
:1055D8001183002B40F082802B68A16800BF2A68E5
:1055E8009342F9D1D7F800B000FB0BF2521AB2FB84
:1055F800FBF200FB0323019A9B1AB3F57A7FDFD3F2
:10560800BAF1010ABED1039B002B40F0BD804FF4D4
:105618007A7ADFF88C9150464FF0100CD9F80430A4
:10562800C3F30803002B75D1EFF31183002B71D15D
:105638002968A26800BF2B689942F9D1D7F800E021
:1056480000FB0EF39B1AB3FBFEF300FB01314FF096
:10565800010E0191D9F80430C3F3080313BBEFF32B
:105668001183FBB92B68A16800BF2A689342F9D15E
:10567800D7F800B000FB0BF2521AB2FBFBF200FBAA
:105688000323019A9B1AB3F57A7FE3D3BAF1010A8F
:10569800C4D1029B013B0293002B7FF466AF05B097
:1056A800BDE8F08FEFF311888CF31288A1682368A6
:1056B800DB0344BFC6F800E0A1682B6832685FFAD4
:1056C80088F888F31188D7F800801A4400FB08F39B
:1056D8005B1AB3FBF8F300FB0233D2E7EFF3118850
:1056E8008CF31288A1682368DB0344BFC6F800E086
:1056F800A1682B6832685FFA88F888F31188D7F8B0
:1057080000801A4400FB08F35B1AB3FBF8F300FBB4
:10571800023370E7EFF311828CF31288D4F808E0B3
:105728002368D90303D501233360D4F808E02B6834
:105738003168D2B282F311883A68194400FB02F347
:10574800A3EB0E03B3FBF2F300FB01317FE7EFF3AA
:1057580011828CF31288D4F808E02368D90303D5A2
:1057680001233360D4F808E02B683168D2B282F3A1
:1057780011883A68194400FB02F3A3EB0E03B3FB4C
:10578800F2F300FB013118E7184629F0B5FD3EE7B2
:1057980010E000E08C6400209064002094640020F5
:1057A80000ED00E0204B5B68C3F3080330B4BBB9DD
:1057B800EFF31183A3B91D4B1D4C1868A16800BFF6
:1057C8001A689042F9D11B4B1C684FF47A7202FB9D
:1057D80004F3591AB1FBF4F130BC02FB0010704716
:1057E800EFF31182102383F3128811498C680B6838
:1057F80013F4803F104B02D0012018608C680B49CD
:10580800D2B20D68186882F311880A4B19684FF4F0
:105818007A72284402FB01F31B1B30BCB3FBF1F383
:1058280002FB0030704700BF00ED00E090640020EC
:1058380010E000E0946400208C6400202DE9F84F0B
:105848008046FFF7AFFF254E2549DFF8A0E0254A3F
:10585800254D844610274FF47A740120DEF8043071
:10586800C3F30803D3B9EFF31183BBB90B68D2F8BC
:1058780008A000BFD1F800904B45F7D1D6F800B08A
:1058880004FB0BF9A9EB0A09B9FBFBF904FB039329
:10589800A3EB0C034345E1D3BDE8F88FEFF3118A7E
:1058A80087F31288D2F808B01368DB0344BF286076
:1058B800D2F808B00B68D5F800905FFA8AFA8AF334
:1058C8001188D6F800A0994404FB0AF3A3EB0B0354
:1058D800B3FBFAF304FB0933DAE700BF9464002052
:1058E8009064002010E000E08C64002000ED00E0EF
:1058F8002DE9F04FDFF830C1474A4849484E494D35
:105908008046102718F1FF38C0F08480DCF8043096
:10591800C3F30803002B5CD1EFF31183002B58D19C
:105928000B68946800BF08688342F9D1D6F80090E4
:105938004FF47A7000FB09FEAEEB040EBEFBF9FED5
:1059480000FB03EEDCF80430C3F308034FF47A7469
:105958000120FBB9EFF31183E3B90B68D2F808A073
:1059680000BFD1F800904B45F7D1D6F800B004FB42
:105978000BF9A9EB0A09B9FBFBF904FB0393A3EBA9
:105988000E03B3F57A7FBDD2DCF80430C3F3080305
:10599800002BDFD0EFF3118A87F31288D2F808B012
:1059A8001368DB0344BF2860D2F808B00B68D5F849
:1059B80000905FFA8AFA8AF31188D6F800A0994411
:1059C80004FB0AF3A3EB0B03B3FBFAF304FB093361
:1059D800D5E7EFF3118487F31288D2F8089013689B
:1059E800D80303D501232B60D2F808900B682868E8
:1059F800E4B284F31188D6F800A04FF47A7400EB6F
:105A0800030E04FB0AF3A3EB0903B3FBFAF304FB4D
:105A18000E3E97E7BDE8F08F10E000E090640020AC
:105A2800946400208C64002000ED00E030B4EFF3B3
:105A38001183102282F312880649074C0A68074826
:105A4800013200250A602560DBB2026883F3118801
:105A580030BC7047906400208C64002010E000E0A7
:105A68001D4B70B59C68236D626BDD69C2B1A36B79
:105A78002BB12B0702D5236D08221A6270BD2A06A6
:105A8800F7D5A26A616A8A4220D0511CA069A16236
:105A9800825C2069266D81423285EAD3A362E8E7F9
:105AA800A906E4D5E26A22B1988C216B80B29047AE
:105AB800DDE7E1699B8C6069DBB24E1CE66143540B
:105AC800E169E368994228BFE261D0E7226D136873
:105AD80023F080031360CCE76C2E00201D4B70B5BB
:105AE8005C68236D626BDD69C2B1A36B2BB12B07B8
:105AF80002D5236D08221A6270BD2A06F7D5A26A5C
:105B0800616A8A4220D0511CA069A162825C206926
:105B1800266D81423285EAD3A362E8E7A906E4D577
:105B2800E26A22B1988C216B80B29047DDE7E16987
:105B38009B8C6069DBB24E1CE6614354E169E36803
:105B4800994228BFE261D0E7226D136823F08003F1
:105B58001360CCE76C2E00201D4B70B51C68236DBC
:105B6800626BDD69C2B1A36B2BB12B0702D5236D24
:105B780008221A6270BD2A06F7D5A26A616A8A42AB
:105B880020D0511CA069A162825C2069266D8142E7
:105B98003285EAD3A362E8E7A906E4D5E26A22B12E
:105BA800988C216B80B29047DDE7E1699B8C606936
:105BB800DBB24E1CE6614354E169E368994228BFB1
:105BC800E261D0E7226D136823F080031360CCE70D
:105BD8006C2E002070B4EFF31186502383F31288E3
:105BE800836B1A68D20720D45D686DB9446A826AEB
:105BF800944217D081691144D9600ED9A21A5A600B
:105C08008462002280F854201A6842F00102F1B23E
:105C18001A6081F3118870BC704701698A1A5A604A
:105C28008562EEE7012380F85430F1B281F31188E0
:105C380070BC704703685B6A03B11847704700BFC0
:105C480003681B6A03B11847704700BF03682DE952
:105C5800F041DF691FB13B46BDE8F0411847002A13
:105C6800164611DD04460D460E4400E023689B6885
:105C7800204698470028F9D0236815F8011B1B68AF
:105C880020469847AE42F1D1BDE8F08103689B6990
:105C9800184700BF03685B69184700BF0368DB68E3
:105CA800184700BF03689B68184700BF03685B6814
:105CB800184700BF03681B68184700BF054B53F817
:105CC800203033B11A689B88918A0B4218BF1B0495
:105CD800936170475C640020036803F138422DE942
:105CE800F04F920A584DAA5C02F01F055209012490
:105CF800022A04FA05F400F08C80032A00F08E8052
:105D0800012A3CD001F003077A1E012AC1F3810C55
:105D1800C1F300188088C1F3411135D9C60700F1D5
:105D28009780850700F1A380440700F1B18002073E
:105D380000F1BF80C60600F1CD80850600F1DB804A
:105D4800440600F1E980020600F1F780C60500F17B
:105D58000581850500F11381440500F121810205C3
:105D680000F12F81C60400F13D81850400F14B81CB
:105D7800440400F15981020455D4BDE8F08F334A38
:105D880055692C435461BDE7002422464FF0010EAB
:105D98004FF0030904E00132102A04F10204ECD0A8
:105DA8000EFA02F636EA0005F5D1D3F808A009FA8A
:105DB80004F5ED430AEA050AC3F808A0D3F808B0C9
:105DC8000CFA04FA4AEA0B0AC3F808A0B3F804A0CC
:105DD8001FFA8AFA2AEA06069E80B3F804A008FA8F
:105DE80002F646EA0A06B6B29E801E682E401E607B
:105DF800D3F800A007FA04F646EA0A061E60D3F8AC
:105E08000CA001FA04F605EA0A0A46EA0A05DD606A
:105E1800C1E70E4A95692C43946173E70B4AD5692B
:105E28002C43D4616EE71A6822F040421A601A685F
:105E380042EA87771F60DA6822F0404242EA8171BD
:105E4800D960BDE8F08F00BF548F030800100240EE
:105E58001A6822F003021A601A683A431A60DA686C
:105E680022F003020A438507DA607FF55DAF1A68FE
:105E780022F00C021A601A6842EA87021A60DA688D
:105E880022F00C0242EA81024407DA607FF54FAF44
:105E98001A6822F030021A601A6842EA07121A6079
:105EA800DA6822F0300242EA0112DA6002077FF56E
:105EB80041AF1A6822F0C0021A601A6842EA8712D3
:105EC8001A60DA6822F0C00242EA8112C606DA6075
:105ED8007FF533AF1A6822F440721A601A6842EAF2
:105EE80007221A60DA6822F4407242EA0122850623
:105EF800DA607FF525AF1A6822F440621A601A68E2
:105F080042EA87221A60DA6822F4406242EA812271
:105F18004406DA607FF517AF1A6822F440521A6017
:105F28001A6842EA07321A60DA6822F4405242EAF2
:105F38000132DA6002067FF509AF1A6822F440429E
:105F48001A601A6842EA87321A60DA6822F4404214
:105F580042EA8132C605DA607FF5FBAE1A6822F4A0
:105F680040321A601A6842EA07421A60DA6822F474
:105F7800403242EA01428505DA607FF5EDAE1A68E3
:105F880022F440221A601A6842EA87421A60DA68E4
:105F980022F4402242EA81424405DA607FF5DFAE0E
:105FA8001A6822F440121A601A6842EA07521A6004
:105FB800DA6822F4401242EA0152DA6002057FF5FB
:105FC800D1AE1A6822F440021A601A6842EA87526F
:105FD8001A60DA6822F4400242EA8152C604DA60A2
:105FE8007FF5C3AE1A6822F040721A601A6842EA56
:105FF80007621A60DA6822F0407242EA0162850498
:10600800DA607FF5B5AE1A6822F040621A601A6845
:1060180042EA87621A60DA6822F0406242EA8162E4
:106028004404DA607FF5A7AE1A6822F040521A607D
:106038001A6842EA07721A60DA6822F0405242EAA5
:106048000172DA6097E600BF2DE9F04F4A484B4BE2
:106058004B4C4FF090414FF0010A4FF002094FF0BE
:1060680004084FF0080C4FF0100E2027402680251A
:1060780030F8022B12F0010F03D01960A3F804A026
:10608800083312F0020F03D01960A3F80490083304
:1060980012F0040F03D01960A3F80480083312F03B
:1060A800080F03D01960A3F804C0083312F0100FCA
:1060B80003D01960A3F804E0083312F0200F02D0CF
:1060C80019609F80083312F0400F02D019609E803B
:1060D800083312F0800F02D019609D80083312F443
:1060E800807F05D04FF4807B1960A3F804B0083393
:1060F80012F4007F05D04FF4007B1960A3F804B0B8
:10610800083312F4806F05D04FF4806B1960A3F840
:1061180004B0083312F4006F05D04FF4006B196017
:10612800A3F804B0083312F4805F05D04FF4805B05
:106138001960A3F804B0083312F4005F05D04FF4D7
:10614800005B1960A3F804B0083312F4804F05D03F
:106158004FF4804B1960A3F804B00833D20B04D075
:106168004FF4004219609A80083301F58061A1421A
:106178007FF47EAFBDE8F08FD48B03085053002026
:1061880000180048002852D0036803F138422DE96E
:10619800F04F920A504DAA5C02F01F0552090124E3
:1061A800022A04FA05F443D0032A00F09080012A59
:1061B80043D001F003077A1E012AC1F3810CC1F311
:1061C80000188088C1F341113CD9C60700F18880C6
:1061D800850700F19480440700F1A280020700F1CE
:1061E800B080C60600F1BE80850600F1CC8044066A
:1061F80000F1DA80020600F1E880C60500F1F680B9
:10620800850500F10481440500F11281020500F1C1
:106218002081C60400F12E81850400F13C814404EC
:1062280000F14A81020400F15881BDE8F08F7047FF
:106238002A4A95692C439461BBE7284A55692C433F
:106248005461B6E7002422464FF0010E4FF00309CF
:1062580004E00132102A04F10204E6D00EFA02F634
:1062680036EA0005F5D1D3F808A009FA04F5ED439C
:106278000AEA050AC3F808A0D3F808B00CFA04FA29
:106288004AEA0B0AC3F808A0B3F804A01FFA8AFA6E
:106298002AEA06069E80B3F804A008FA02F646EA3F
:1062A8000A06B6B29E801E682E401E60D3F800A073
:1062B80007FA04F646EA0A061E60D3F80CA001FAAB
:1062C80004F605EA0A0A46EA0A05DD60C1E7034A58
:1062D800D5692C43D4616CE7548F03080010024041
:1062E8001A6822F003021A601A683A431A60DA68D8
:1062F80022F003020A438507DA607FF56CAF1A685B
:1063080022F00C021A601A6842EA87021A60DA68F8
:1063180022F00C0242EA81024407DA607FF55EAFA0
:106328001A6822F030021A601A6842EA07121A60E4
:10633800DA6822F0300242EA0112DA6002077FF5D9
:1063480050AF1A6822F0C0021A601A6842EA87122F
:106358001A60DA6822F0C00242EA8112C606DA60E0
:106368007FF542AF1A6822F440721A601A6842EA4E
:1063780007221A60DA6822F4407242EA012285068E
:10638800DA607FF534AF1A6822F440621A601A683E
:1063980042EA87221A60DA6822F4406242EA8122DD
:1063A8004406DA607FF526AF1A6822F440521A6074
:1063B8001A6842EA07321A60DA6822F4405242EA5E
:1063C8000132DA6002067FF518AF1A6822F44042FB
:1063D8001A601A6842EA87321A60DA6822F4404280
:1063E80042EA8132C605DA607FF50AAF1A6822F4FC
:1063F80040321A601A6842EA07421A60DA6822F4E0
:10640800403242EA01428505DA607FF5FCAE1A683F
:1064180022F440221A601A6842EA87421A60DA684F
:1064280022F4402242EA81424405DA607FF5EEAE6A
:106438001A6822F440121A601A6842EA07521A606F
:10644800DA6822F4401242EA0152DA6002057FF566
:10645800E0AE1A6822F440021A601A6842EA8752CB
:106468001A60DA6822F4400242EA8152C604DA600D
:106478007FF5D2AE1A6822F040721A601A6842EAB2
:1064880007621A60DA6822F0407242EA0162850403
:10649800DA607FF5C4AE1A6822F040621A601A68A2
:1064A80042EA87621A60DA6822F0406242EA816250
:1064B8004404DA607FF5B6AE1A6822F040521A60DA
:1064C8001A6842EA07721A60DA6822F0405242EA11
:1064D8000172DA6002047FF5A8AE1A6822F0404221
:1064E8001A601A6842EA87771F60DA6822F0404229
:1064F80042EA8171D960BDE8F08F00BF10B103682E
:1065080082881A85704700BF10B1036882889A6133
:10651800704700BF38B100298388026814BF002182
:1065280010218B40936170470E4B1B8801463BB985
:106538000D4B0E4A1B7810680BB981F00101E9E791
:106548000B4B5A691AB118B91A6810605874704719
:10655800084A18681188084A92FBF1F20121026082
:1065680059747047686400206A6400206C640020D5
:10657800706400208864002020A1070010B40A4B32
:106588000A4A1C7801238340234052F8200029B985
:10659800B3FA83F149095DF8044BBBE7191C18BF2E
:1065A80001215DF8044BB5E7586400205C640020C5
:1065B80030B1036882881B8A1A4214BF0120002068
:1065C800704700BF2DE9F0410B4E346873691C40D9
:1065D8000FD0DFF828800127B4FA84F3C3F11F0332
:1065E80007FA03F558F8230003689847AC43756128
:1065F800F2D1BDE8F08100BF00040140CC5F00206B
:106608002DE9F0410B4E346873691C400FD0DFF858
:1066180028800127B4FA84F3C3F11F0307FA03F5AE
:1066280058F8230003689847AC437561F2D1BDE878
:10663800F08100BF00040140CC5F00202DE9F0414B
:106648000B4E346873691C400FD0DFF8288001278F
:10665800B4FA84F3C3F11F0307FA03F558F82300CB
:1066680003689847AC437561F2D1BDE8F08100BF7B
:1066780000040140CC5F00202DE9F0410B4E346846
:1066880073691C400FD0DFF828800127B4FA84F31F
:10669800C3F11F0307FA03F558F823000368984766
:1066A800AC437561F2D1BDE8F08100BF0004014040
:1066B800CC5F00202DE9F0410B4E346873691C4013
:1066C8000FD0DFF828800127B4FA84F3C3F11F0341
:1066D80007FA03F558F8230003689847AC43756137
:1066E800F2D1BDE8F08100BF00040140CC5F00207A
:1066F8002DE9F0410B4E346873691C400FD0DFF868
:1067080028800127B4FA84F3C3F11F0307FA03F5BD
:1067180058F8230003689847AC437561F2D1BDE887
:10672800F08100BF00040140CC5F00202DE9F0415A
:106738000B4E346873691C400FD0DFF8288001279E
:10674800B4FA84F3C3F11F0307FA03F558F82300DA
:1067580003689847AC437561F2D1BDE8F08100BF8A
:1067680000040140CC5F0020084A094808B5936935
:1067780043F0010393610021402230F05EF9054B9C
:106788004FF0FF321A60C3F8032008BD0010024022
:10679800CC5F00200C6000202DE9F041044618462B
:1067A8000D46164698462EF0AFF82768E67228443C
:1067B800A07229467D69434632462046AC46BDE86C
:1067C800F0416047036810B504461B689847236882
:1067D80020469B689847A37B0133A37310BD00BF75
:1067E80008B52120FEF78EFC0B4B186018B111225A
:1067F80000238271C3712021FFF7C4FC2020FEF71B
:1068080081FC064B186018B1112200238271C371F4
:106818002021BDE80840B5E4642E0020682E002041
:10682800064B984202D04FF0FF307047044A538B12
:1068380001339BB25383508B80B2704700380040BD
:1068480028640020F0B50E460178012985B0044679
:106858004BD002294FD11D46836846F0800113B101
:1068680018689B880385606840F2E93301E0002BD3
:1068780055D00689013B16F0020F9BB2F7D0017381
:1068880040F2E93301E0002B49D00189013B11F0C6
:10689800010F9BB2F7D0037B60684FF0000C83892F
:1068A8004FF6FF764FF47A734FF0FF0E654502D12D
:1068B80026E0B34222D00189013B8F079BB2F8D56D
:1068C80080F80CE04FF47A7302E0BBB2B34215D003
:1068D8000189C90703F1FF37F7D5017BC9B20AB1AE
:1068E800117001320CF1010CE0E790F90400411C31
:1068F80001D002280CDD002005B0F0BDFFF790FFA5
:10690800A3688BB11A689B889361012005B0F0BD1C
:10691800617900923246FBF7C7FB05B0F0BD0392E0
:10692800FFF77EFF039AB7E70120E5E70378012B1D
:1069380043D0022B3FD170B5836801F07F0113B1BA
:106948001C689B88238505461646406840F2E93452
:1069580001E0002C38D00389013C13F0020FA4B2E7
:10696800F7D0017340F2E93100E069B303890139D6
:1069780013F0010F89B2F8D0037B686840F2E9315F
:1069880000E021B30489013914F0020F89B2F8D06C
:10699800067340F2E93300E0CBB10289013B12F003
:1069A800010F9BB2F8D0037BAB689BB11A689B8838
:1069B8009361012070BD0020704713460A46417953
:1069C80090F90400FBF700BDFFF72AFFD5E7FFF7B2
:1069D80027FFE9E7012070BD427A02B9704710B578
:1069E80004460368406804F10A019847002363726B
:1069F80010BD00BF437A5A1C0344D2B24272997246
:106A0800037A934200D802B9704710B50446036868
:106A1800406804F10A0198470023637210BD00BF63
:106A280038B50B4C23688BB15A68821A002A054680
:106A380004DA0CE05A68AA1A002A07DB9A6822606E
:106A480018461A6890472368002BF3D138BD38BD23
:106A5800743400202DE9F04F2DED068BAB4BAC4A7A
:106A68001C7897B000F59C41203181460B9111604C
:106A7800002C00F0EC86A74A1268904240F283800E
:106A8800A54A06921668A549A54A0591013C1C70BD
:106A9800A44B049206F480560893002E40F081809F
:106AA800A14B1B78022B01F08081042B01F06F8130
:106AB800012B01F023819D4B9945089B9B7800F29F
:106AC8009985002B40F09A85994B0793069B1E6881
:106AD80016F4805740F08986DFF894A2049BB3F936
:106AE8000610059B5D8BA942B4BF00250125914B7B
:106AF8001B6813F080535ED0079A127812F00102D7
:106B08005FD00598408C884241F3A282002D5ED167
:106B1800894C94F88C10002959D188488849006814
:106B280090F82D0000240C604C608C60854900288A
:106B38004ED10870002A4FD0F1064DD5824A1278FE
:106B4800D20649D4002F47D1002B45D1740243D433
:106B58007E4B1B78002B02F02C827D4B9B78002DFE
:106B680042F069823BB17B4A7B4B12681B689B1AD7
:106B7800002BC2F26B8210206F4C29F01FFA012300
:106B880084F88D3028E0644B06931E68644B634A92
:106B9800049306F48056634B05920893002E3FF445
:106BA8007FAF00216348FAF7E7FE00287FF478AF4B
:106BB8000DF03CFE74E770029ED4079A127802F03A
:106BC80001025D4C002184F88C10002DA5D05D4990
:106BD80001200870002AAFD1604B1A78002A79D1B9
:106BE8000599049C488BB4F90070898BB4F902406C
:106BF800B842B4BF8026002646F04003B942D8BF49
:106C080033469B0843F08006A042B8BF3346049F32
:106C180043F04006A142C8BF33469B08B7F9044079
:106C2800B7F9066043F08007A042B8BF3B4643F07F
:106C38004007A142C8BF3B469B0843F080073E4C33
:106C48008642C8BF3B4643F0400794F88EE08E4228
:106C5800B8BF3B469E4501F05384A4F8902084F8C1
:106C680092203A4984F88E300E78002E01F04A833B
:106C78005F2B01F0C7836F2B01F00984079B1B78FA
:106C8800DA0727D494F8921021BBB4F99030322B4C
:106C980020DD94F88E200120572A84F8920001F014
:106CA8007E87069B1B685F0741F198825A2A41F04C
:106CB800958294F89430002B42F0A28194F8963093
:106CC80083F0010384F89630002B42F0A7810C2052
:106CD80029F074F9224B0993224B234D0A93069B02
:106CE8001B685C0700F1E5860DF150091F4E0B95F6
:106CF8000022C9F804203446149240F6330B4FF0B2
:106D0800190840F28337049D37E000BF7034002033
:106D18003C3300206C3400201C57002014600020F5
:106D28008E880020D4490020EA3A0020404B4C00CD
:106D38001B520020644100207C1E0020AC4700202C
:106D48005C3B002078210020F43B00204C1C0020F4
:106D5800BC41002090640020FC250020BF42002098
:106D68004C470020B0470020A8470020D834002016
:106D7800283500200434544522D0A178E37899427C
:106D880018FB0170F6D294F801E00EF1040E18FB1E
:106D9800037135F91E305B45A8BF5B46B3F5617FCB
:106DA800B8BF4FF461739842E4DA9942E2DB217884
:106DB8002729DFD848460434FAF7CEFD5445DCD1FC
:106DC800674A0B9D1378674A99E8030082E8030035
:106DD800002B40F0BE85644B1A78002A00F0E88545
:106DE80001216048FAF7C8FD002840F0E682089BB8
:106DF800DB78002B40F0E1822B881FB227F00107D7
:106E08001FFA87F84345A5F8008000F0FD87574F23
:106E18004FF002090E204FF0140B4FF0FF0A87F8CD
:106E2800009087F801B087F802A029F0C7F8494612
:106E38004C48B5F80080FAF79FFD002800F0D8828A
:106E480028F001039BB243452B800AD00E2087F817
:106E5800009087F801B087F802A029F0AFF8B5F8DC
:106E6800008018F0020F01F0A581414B414A1978C2
:106E780050680B9318F0030F08BF81F00201C1F3AB
:106E880040010C92FFF746FB24213648FAF774FDBF
:106E980030B9079A1378590744BF23F004031370D5
:106EA800099B1B6813F00A0F1BD005212D48FAF720
:106EB80063FD002801F0A2802F887B0741F137820B
:106EC80028480621FAF758FD002801F08480780642
:106ED80041F1258207212348FAF74EFD002840F0AA
:106EE800A0870C211F48FAF747FD2A88002800F0E0
:106EF800938242F480739A422B8009D01B4B022262
:106F080014211A700E20FF2259709A7029F056F831
:106F1800194B1B78082B00F08B820E2B00F088820F
:106F2800069BD3F8008018F4806F5FD0134B1B7951
:106F3800002B00F0248214210A48FAF71DFD0028CE
:106F480040F022821FF0F2FA012028F079FF002891
:106F580049D0DFF82CA000274FF0CC0BA14614E055
:106F680040590020644100202F4200207C3F00202F
:106F7800586400205C640020E83B00207045002035
:106F880048850020DFB2022F2CD80BFB07F87B1CAA
:106F98005AF80840002CF5D1032290F902300294E7
:106FA8000192C278E24951F82220009218462246FE
:106FB8002346012128F080FB034607EB470000EB3E
:106FC8000010099353B121460AEB8000CC222FF020
:106FD80034FD099B4AF808300137FFB227F01CFD41
:106FE8000028D0D14C46069BD3F80080079B93F825
:106FF80000A0D04B1AF0010A00F06D8201221A702D
:107008000A9B04991B68B1F906105A89CA480127D6
:107018009142077080F24582C84B4FF07E521A6049
:10702800059BC74FB3F81890049B97F90420B3F950
:107038000030387897F801C0002AA3EB090714BF7D
:1070480001224FF0FF32002FB8BF7F42B7F5FA7F19
:10705800A8BF4FF4FA77B84280F2BC823F1A07EE15
:10706800907AF8EEE77AB74F4B45C7ED007A03DA26
:10707800F1EE677AC7ED007A049BB3F902E0AEEB54
:107088000903002BB8BF5B42B3F5FA7FA8BF4FF4E2
:10709800FA73984280F202821B1A07EE903AF8EED1
:1070A800E77AF145C7ED017A03DDF1EE677AC7EDBE
:1070B800017A049BB3F90400A0EB0903002BB8BFC5
:1070C8005B42B3F5FA7FA8BF4FF4FA736345CCBFB0
:1070D800A3EB0C03002302FB03F207EE902AF8EE61
:1070E800E77A4845C7ED027ABCBFF1EE677AC7ED8B
:1070F800027A18F4805800F0AE81B1F5FA6F924B1D
:10710800A8BF4FF4FA61B1F57A7F1A78B8BF4FF487
:107118007A71A1F57A71002A41F046818B4ADFF82D
:1071280044E282FB0130CB17C3EB6013581C6FF0AD
:10713800630C3EF910003EF913E00CFB0313A0EBBF
:107148000E0003FB00F382FB0312DB17C3EB621391
:107158009E440FFA8EFE07EE90EAB8EEE78A87EDB6
:10716800038AB8F1000F40F0B4832B885A0640F127
:10717800FB807749774A91ED018AD2ED019A92ED29
:10718800026A91ED034A92ED030A91ED029A92ED9B
:10719800007AD1ED005AD7ED011A97ED002A6E4A10
:1071A8006E4938EE445A79EEC63A77EE007A65EEC3
:1071B800233A75EEC96A75EE890A37EE401A66EE0B
:1071C800A76AB0EE633AA0EE813A13F00303B0EE7B
:1071D800665A78EE044A79EE867AA0EE815AF0EE85
:1071E800638AA4EEA73AD4EEA78AA4EEE75A33EE50
:1071F800263AF0EE687AF0EE674AF6EE008A35EE47
:1072080088AAE0EEC14A28EEC33A35EE635A77EE13
:10721800293A77EEE67AAAEE233A25EE285A76EE50
:10722800403A34EE49AAE0EE817A74EEA64AAAEE14
:10723800235A34EE094A37EE697A64EEA84A63EEB7
:10724800036AE4EE074A75EEC85A36EE006A67EE3E
:10725800A87AB0EE667A95EE057AE5EE056AE5EE6F
:10726800867AB1EE648AF0EE665AF0EE476AB1EEBD
:10727800674AE8EE246A63EE270A67EEA43AE4EE6A
:10728800275AB1EE450AB0EE609AB0EE631AA4EE42
:10729800277A23EE244AE7EEA76AA5EE249AA0EE01
:1072A800031AE8EE245AB0EE448A31EEA16AE0EE01
:1072B800240AA5EE278A66EEA16A72EE028AE5EE36
:1072C800033A61EE211A26EE096AA4EEA47AA0EE2A
:1072D800274A0CBFD7ED022ADFED212A82ED005A9A
:1072E800A2EE256AE8EEA06AE2EE081A73EEA33A67
:1072F80027EE227A34EE044AF0EE005AE3EEA26A50
:10730800A2EE846AA1EEA57AC7ED016AC1ED366ADC
:1073180081ED356A87ED006A81ED377A82ED013AB1
:10732800C2ED027AC2ED034AF3B987ED027A1BE097
:10733800708A03081C520020B02100202C21002054
:107348009441002080450020B42600201F85EB5181
:107358008400002058070020900700207C1E002091
:1073680000000000E4510020BAF1000F40F0358120
:107378002CF024FE17B0BDEC068BBDE8F08F079B00
:107388001B78D9077FF5DEAD4FF40F702BF06CFB3F
:1073980000283FF428AE0FF009FB4FF40F702BF0D4
:1073A8000DFB00283FF41FAE0FF000FB4FF40F70E9
:1073B8002BF004FB0028EED115E6099B1B68980703
:1073C8007FF51AADB5F8008018F0010F10D148F01C
:1073D800010398452B800BD09B4B022214211A7075
:1073E8000E20FF2259709A7028F0E8FDB5F8008049
:1073F80028F002039BB243452B803FF436AD924BF5
:1074080002201421FF2218700E2059709A7028F05B
:10741800D5FDB5F8008028E522F480739BB29A4226
:107428002B807FF46BAD894B1B78082B7FF475ADEF
:107438002A8822F040039BB29A422B803FF470AD19
:10744800814B022214211A700E20FF2259709A7063
:1074580028F0B4FD64E5059B5A8B9142C0F2D184B3
:10746800B1F5FA6FD4BFC2EB0101C2F5FA614FF46E
:107478007A7303FB01F176480378C2F5FA62B1FB2F
:10748800F2F1002B3FF44AAE4378724A01FB03F154
:1074980082FB0123C917C1EB63113FE6DFED6E7A6A
:1074A800FFE5B1F5FA6F80F2A584187A8B1A03FB11
:1074B80000F3C2F5FA6293FBF2F3C3F1640307EE3B
:1074C800903AF8EEE77A9FED657A654B67EE877A32
:1074D800C3ED007AA4E51B780693002B7FF490ADEA
:1074E800604A1268002A3FF48BAD5F4A079212F88F
:1074F800030CDFF8A8B11146D71E21F0D1FD9BF887
:107508000090079A002800F0FC85069BB9F1000F4F
:1075180041F07C8407F10801787921F0C1FD002849
:1075280041F0D7845149B87A21F0BAFD002800F01B
:10753800FB85B9F1020F41F0D4844D49F87B21F065
:10754800AFFD002841F0C9844A49387D21F0A8FDE3
:10755800002800F0FB85B9F1040F41F0D2844649B8
:10756800787E21F09DFD002841F0C7844349B87F0B
:1075780021F096FD002800F0FB85B9F1060F41F0D7
:10758800B8843F4997F8230021F08AFD002841F08C
:10759800AC843C4997F8280021F082FD002800F0CF
:1075A800FB85B9F1080F41F0B084374997F82D00F1
:1075B80021F076FD00283FF423AD0922134602EBA3
:1075C80082021744314A7878B9788BF80030107005
:1075D800517015E5DFED207A45E50B9B19780C9B7A
:1075E80001F001011868FEF795FF17B0BDEC068B96
:1075F800BDE8F08F13B9089A01239370244B089AB9
:107608001D7892F8214007931B2021F073FD012C6F
:1076180005F00108814600F0378705F00205089A51
:107628001C4E92F82030DFF878A01B4F099593463E
:10763800052B00F2A387DFE813F0BD00B300350087
:10764800FB00FD00F00000BF7C3F0020E83B00206D
:10765800B42600201F85EB51000000000AD7233C08
:107668002C210020205200203A3F0020443F0020D7
:10767800493F00204E3F0020533F0020583F002044
:107688005D3F0020623F0020673F00202452002019
:107698001B520020DC510020A447002000000020DD
:1076A8004C1C0020012C04BF05238BF82030B8F1B6
:1076B800000F12D0059B3088B3F91810002213462A
:1076C80061F30F0260F31F4261F30F03049861F343
:1076D8001F430360032342600993AA4DDBF814108B
:1076E8002A68914280F0FE8547F230510322CBF898
:1076F8001C108BF8202002200CF05EFA0DF096F892
:107708002968DBF81C200A440421CBF818208BF8E0
:107718002010012C40F078872A68DBF81810914275
:1077280080F02C879AF8000020B921F0E3FC0028AB
:1077380040F024873A6822F002023A602A68738887
:10774800642101FB03234FF480600022CBF8103042
:107758008BF820208BF803200CF0FEF99BF82030E2
:1077680066E721F0CDFC012807D1864D72882B6889
:10777800642101FB0233CBF81030B9F1000F02D0BD
:10778800B379002B4BD1012C00F0F8867D4DDBF846
:1077980010102A689142C0F0448701238BF82030EA
:1077A800012C3AD0F379012B46D021F037FC9BF815
:1077B80020303DE7B8F1000FD3D1099D4FF4806028
:1077C800B9F1000F00F02A830CF0DEF9089A0023C3
:1077D8001361002D3FF47AA9284628F0EFFB069B99
:1077E8001E6816F480573FF477A91D216648FAF7FA
:1077F800C3F800287FF470A9644B03F1500A03E032
:1078080004339A4500F0C0861A78262AF8D1997868
:10781800DA789142F4D2FFF761B95A4D8EE721F038
:10782800FDFB03224FF47A738BF82020CBF81C3031
:10783800544D60E7534D6CE721F0F0FB032240F60E
:10784800B8338BF82020CBF81C304E4D53E7504FFF
:107858003B78002B01F03B824E4BDFF84881DFF884
:1078680048B1DFF848A1059345465E46049099461D
:107878000EE019F804109847032C28DC88B93B78E7
:107888002AF8020F01349C4205F1040580F2368182
:10789800072CE1B23046DBF80430EADD984700B245
:1078A800EDE738F824206B88801A4FF47A719B1A18
:1078B80001FB00F040F6CA0290FBF3F00844904246
:1078C80040F2EE23A8BF10469842B8BF184600B24F
:1078D800D5E71D212C48FAF74FF828B100F028BE4B
:1078E8000436A6423FF441AC31782629F8D1B27863
:1078F800F3789A42F4D2089BDB78002B7FF435ACFE
:107908002148FAF739F8DFED247A002801F0FA81E6
:1079180038EE678A214A2249FDEEC87ACDED047A0D
:10792800BDF910301B0382FB0302DB17C3EBA21265
:10793800C9F57A731BB203FB02F343F30F334B44CD
:1079480007EE903AF8EEE77A0123C7ED037A0B7059
:107958000BE40E4B03E00433A3423FF43CAA19782E
:107968002329F8D19878DA789042F4D20648FAF7C1
:1079780003F800283FF42FAA142028F01FFBFFF774
:107988002ABA00BF9064002064410020D834002047
:107998009C3500201460002000007A44D34D62100A
:1079A800A4210020BC350020E04200207A1E0020DF
:1079B800DFF8F092DFF8F0A2AB4F0B9209F15A080A
:1079C8004FF0010B494619F8010C21F069FB00B38F
:1079D80099F8040099F8023099F803E000EB4001A7
:1079E80007EB8101013BD1F8A02003EB430353448B
:1079F80093420ED097F8CC20C1F8A0300BFA00F0D3
:107A080022EA00000B9B81F89CE0C1F8A43087F8BB
:107A1800CC0009F10609C145D4D1944B944A1B788E
:107A28000B930A9BDFF884A212681B680C93AAF1D7
:107A38009C094FF0000B9046DAF8043083B31F78A6
:107A480077B3DAF80820A8EB0202002A0CDB99F8D1
:107A5800CC20012101FA0BF122EA010208F5FA71A2
:107A680089F8CC20CAF808100B9ACAB19AF80020F5
:107A780059780432D2B2002940F02E83059904982F
:107A8800098B30F9122001F1C800824240F38E853B
:107A980099F8CC109A7841FA0BF3D90740F1198676
:107AA8000BF1010BBBF1040F0AF10C0AC4D1FFF76B
:107AB80097B96D4C94F896305BB1079B1B78D80743
:107AC80007D5049BB3F90620059B5B8B9A4200F30C
:107AD800F28511216748F9F74FFF002800F0A682C8
:107AE80094F89A302BB994F8943013B93223A4F847
:107AF8009830012384F89A30FFF7F6B8DDF8109033
:107B08005D4A06925D49126842F2010AA1FB091B0F
:107B180012EA0A0A4FEA9B1B00F08582584D594821
:107B2800524C59492E780078267008701EB1564973
:107B38000E7886F001064C4C0F2184F82410002B97
:107B480000F01284059D514BB5F826C0B5F824E025
:107B5800059D109318462D8B00784D4B129594F87F
:107B6800255009954B4D0495A3FB00535B0803EB87
:107B78004303C31ADBB20F90CDF834C002F480522D
:107B88000C9304F128000BF59673CDF8449097F800
:107B98000080DDF82490DFF818C109943D4C0E915F
:107BA800139200210A930896CDF81CE0089B002B3D
:107BB80000F03A83099B079D33F911201FFA82FED2
:107BC800AE454FEA410303D30D9DAE4540F27183A4
:107BD8005CF82120934580F03183E25EBAF1000F12
:107BE80040F0468301314145E25200F10600DDDBF9
:107BF8000E9A099C284B84F824200F2A49460CBF6A
:107C080001220022DDF8449084F825101A7000F053
:107C1800B283224B1B491C4ADFF854B008931C4618
:107C2800042001230B7013700BF0C6FFDBF8003043
:107C3800A1686268E3605B1A934284BF002384F8FA
:107C48002130069B3C781E68002C01F05780059A6D
:107C5800134DB2F824E0178B0E4916F480562846C7
:107C680040F0B283324634E07C1E0020C549002033
:107C780090640020644100201C570020D34D6210FE
:107C880018330020CC000020CD0000208D340020C7
:107C9800ABAAAAAA8E880020DE420020D449002080
:107CA800F0350020513E0020A06C0308181F00206A
:107CB80090340020437803EB830303EB830303F240
:107CC800EE239BB20132A24221F8023B00F10200EE
:107CD8000ED015F81230002B00F0EF82022BE9D0FD
:107CE80001320B8821F8023BA24200F10200F0D1D8
:107CF800109A137801331370FEF7CFBED74CD4F81F
:107D08008830A9EB0303002BFEF6D5AED44AD54B39
:107D1800527C059933F812308A7DDFEDD36A9FEDE6
:107D2800D36AC97D9BB207EE102A07EE903AB8EEE7
:107D3800C77AF8EEE77A27EE267A67EE867A0B9A04
:107D4800C4F88820C7EE876A40F2FF32FCEEE67A74
:107D5800CDED077ABDF81C30934228BF134609B110
:107D6800D31A9BB2C248C34D0178C34C35F8116091
:107D7800226825F81130921B13440131BF4D23604E
:107D880001F00F021B0902702B80FEF794BEFDF76D
:107D980009FDBB4BBB4A1B68C31A93427EF78BAEE7
:107DA800B64B00221A80FEF786BE059A0499537DC9
:107DB800D27D013B31F913301AB1C3F53B63083367
:107DC8001BB2A3F57A7307EE903A9FEDAF7AAB4AF0
:107DD800F8EEE77A40F2FF3167EE877AFCEEE77A51
:107DE800CDED077ABDF81C308B4228BF0B461380B7
:107DF800FEF761BE1B7AC3F1640307EE903AFFF702
:107E080060BB4146FFF737BB0221A048F9F7B4FD34
:107E180000283FF4EDAA2F80FFF723B80BF09CFE53
:107E2800D4E49B4AB2F90030002BB8BF5B42B3F5EB
:107E3800E17FBFF656A8B2F90230002BB8BF5B420B
:107E4800B3F5E17FBFF64DA8924B93ED096AD3EDE8
:107E5800076A93ED057AD3ED037A76EE866A77EEB4
:107E6800877A76EEA66AB7EE007A37EE666A77EE1C
:107E7800A77AB0EEC66AF0EEE75AB4EEE56AF1EE1C
:107E880010FAB4BFB0EE655AB0EE465AB5EE405A95
:107E9800F1EE10FA40F0DF839FED7F7AB4EEE56AE9
:107EA800F1EE10FA44BF9FED7D6A36EE477AB7EEE1
:107EB800006AF4EEC66AF1EE10FAC8BFDFED786A20
:107EC800F5EEC07AC8BF36EEC77AF1EE10FA48BFB1
:107ED800B1EE477AF6EE007A27EE677ADFED6F7A31
:107EE80077EE276ABDEEE66A16EE103A2033402B8D
:107EF80040F27E86DFED6B6A6B4ADFED6A7AC2ED8F
:107F0800006AFDEEC76AC2ED017A16EE903A203398
:107F1800402BC2ED027A49D8DFED617AB4EEE77AF8
:107F2800F1EE10FA41F368809FED606ADFED606A58
:107F380001E0B0EE677AB4EEE67AF1EE10FA77EE89
:107F4800467AF6DC9FED5B7AF4EEC77AF1EE10FA2A
:107F580041F12B809FED556ADFED576A01E0F0EEA5
:107F6800477AF4EEE67AF1EE10FA37EE867AF6D42E
:107F7800DFED4A7AB4EEE77AF1EE10FA40F3918633
:107F8800DFED477A37EEC77A27EE076ADFED4B5AFF
:107F9800DFED4B6ADFED4B7AE6EE256A67EE065AAF
:107FA800E6EE267AA5EEA77AF0EE477A464BC2EDC2
:107FB800037A1B6813F4003340F0628643491A467B
:107FC800C85C0A2803F10C0300F08E850132182AD8
:107FD800F6D1FEF786BF27F040039BB2BB422B8049
:107FE8003EF478AF3A4B022214211A700E20FF2279
:107FF80059709A7027F0E2FFFEF76CBF2B8823F0C8
:108008000407BFB2BB422F803EF45AAF304B022266
:1080180014211A700E20FF2259709A7027F0CEFF93
:108028002F88FEF74DBF2B490E787FE594F89430E2
:10803800002B3EF459AE079B1B7813F001037EF426
:1080480053AE012284F8943084F89520FEF74CBE94
:10805800024C012184F88C10FEF7B9BD7C1E00206B
:10806800D8630020F86300200000C8420000804464
:10807800EB3A0020F03A0020EC3A0020CC490020EE
:10808800F01F002060E316006F12833F6441002058
:108098005847002068070020A7DFA834DB0FC93F36
:1080A800DB0F49400000000084000020DB0FC940BE
:1080B800E4CB1641DB0F49C0E4CB16C192E741B9C6
:1080C8009730083C15A82ABE443E0020A483030824
:1080D8007C3F0020C5490020012900F0238599F83C
:1080E800CC20012303FA0BF30BF1010B1343BBF173
:1080F800040F89F8CC300AF10C0A7FF49DACFEF726
:108108006FBE511D787920F0CBFF00283FF40AAAF2
:10811800B9F1010F40F0DD8607F10D01B87A20F0C2
:10812800BFFF002840F0DD86C149F87B20F0B8FF8A
:1081380000283FF409AAB9F1030F40F0CE86BD49E3
:10814800387D20F0ADFF002840F0DB86BA49787E04
:1081580020F0A6FF00283FF409AAB9F1050F40F066
:10816800CC86B649B87F20F09BFF002840F0C18636
:10817800B34997F8230020F093FF00283FF409AA99
:10818800B9F1070F40F0B186AE4997F8280020F002
:1081980087FF002840F0B986AB4997F82D0020F0FA
:1081A8007FFF00283EF42CAFB9F1090F3EF428AF49
:1081B800FFF703BA48F0020343452B803EF455AE5F
:1081C800A24B022214211A700E20FF2259709A70B5
:1081D80027F0F4FEB5F80080FEF747BE5D2A00F0F0
:1081E8007D825B2A00F086855E2A00F0E885562AA3
:1081F80000F04E86972A00F05D86A72A00F0E385F6
:10820800934D2B889E0740F09E85A2F1B703072B5C
:1082180000F29E82DFE813F080029C029C029C021E
:108228008E029C0272027202079B002B3FD05CF800
:10823800212093454FEA4103FFF4CFAC854A854D91
:10824800D25C05EB030E002A00F0B180022A47D168
:108258009EF8012002EB820202EB820202F2EE2279
:1082680092B2032933DD12B2BAF1000F3FF4BAAC6F
:108278000C9D20F81520B9F1000F03D10F9D022D98
:108288007FF6B0ACB0F802900288B0F804E04A4437
:108298009644714A0FFA8EFE82FB0E526F4DA2EB86
:1082A800EE7225F803E012B24FF001099AE41A467B
:1082B8004B000A9D4CF8215090E4D3B2022B04D90C
:1082C800032B7FF40DAD7346FCE43B46FAE401252D
:1082D80005FA01FE0E9D25EA0E0512B20E957DE403
:1082E800E25ABEE75E4A1278002A7FF4FDA9B8F187
:1082F800000F3FF4F9A9012C40F040819BF8203091
:10830800FFF796B931465748F9F736FB002800F0D1
:10831800D38084F893600CF0ABFEFEF7AFBC47F057
:108328004003BB422B807FF45DAEFEF7D3BD47F020
:1083380004039F422B800AD0444B022214211A7056
:108348000E20FF2259709A7027F038FE2F88464B6E
:10835800464AB3F90430464982FB0302DB17C3EBF4
:10836800A2030B80FEF7ACBD424B434A1092012298
:108378001A70424B04931B213A48F9F7FDFA00287A
:108388007FF447AC3E4BDFF8FCB008931946DBF8A6
:108398000030CA688B609B1AC82B00F29C84069B2D
:1083A8001E6806F48056A3E45B78FFF76EB8CAB27D
:1083B800022A40F2B483032A92D1129A139D079E8F
:1083C800002D08BF32464CE700220FE0437803EB4C
:1083D800830303EB830303F2EE239BB20132A24231
:1083E80021F8023B00F102003FF482AC15F812308C
:1083F8001BB1022BEAD00B88F0E7D3B2032BFAD8D3
:108408003B46EBE7B2F5FA7FFEF664AC94F892309F
:10841800002B7EF45FAC079B1B78012213EA020550
:1084280084F8922000F0D8830CF000FAFEF752BCD2
:10843800493F00204E3F0020533F0020583F002076
:108448005D3F0020623F0020673F00207C3F002006
:10845800A8470020F035002056555555EC1E002041
:10846800682100206441002058470020676666663E
:10847800A6210020DE4200208D3400208E880020B6
:10848800D4490020906400200025FFF7C8B8B2F551
:10849800FA7FFEF61FAC94F89230002B7EF41AACEB
:1084A800079A1278012184F89210D10700F1F0831D
:1084B8000CF0DEFDFEF70EBC079BBA4A1B78106075
:1084C800D8077EF5DFABB84B1B78002B3EF402AC27
:1084D800089BDB78002B7EF4FDAB94F893300133D6
:1084E800DBB2032B84F893307EF6F4ABAF4B5B78AA
:1084F80013B9002D7EF4EEAB0CF098F9FEF7BEBB75
:10850800AB4AAC491068B4F99020C66981FB0601F2
:108518008911F617701A00F5FF407F3082423EF746
:10852800A0AB891B0A4412B2A4F89020FEF799BBAD
:10853800089BDB78002B7FF4D7A9DFED9F7A9D4954
:1085480038EE678AC9F5FA63FDEEC87A1BB2CDED3D
:10855800047ABDF91020120381FB0201D217C2EB85
:10856800A11203FB02F343F30F334B4407EE903A97
:10857800B8EEE78A87ED038AFFF7B6B9099D002DA3
:108588003EF4A4AAFFF728B98C4A059BD588049A1B
:108598001B8BB2F906105A1B914240F389802B4479
:1085A8009942B4BF00250125FEF7A1BAC8398A420D
:1085B80042DA99F8CC109A7841FA0BF3DB073FF5C9
:1085C8006FAA524201200D9227F0DEFD7B1E0D9A04
:1085D800162B00F25181DFE813F0230237020A025A
:1085E8005C024B027002F501E001CB01B601A1016A
:1085F8004F015C028E017002F501E0017A0166010B
:1086080052013F0129011501AB460899DBF800200A
:10861800CB69099D13448B61002D3EF457AAFFF7DF
:10862800DBB820F0FBFC032140F6B8328BF82010B1
:10863800CBF81C20FFF75FB899F8CC30012202FA7A
:108648000BF223EA020308F5FA7289F8CC30CAF86B
:108658000820FFF725BAB4EEE56AF1EE10FA8CBFF0
:10866800B0EE654AB0EE464AC4EE054A9FED542A7C
:108678009FED545ADFED541ADFED542A9FED543A1A
:10868800DFED543A9FED544AA4EE825AE4EEE12A13
:10869800A4EE857AA4EEA23AB0EE475AB0EE637A19
:1086A800A4EE837AA4EE874A84EE057AFFF7F6BB38
:1086B8000125FEF71CBA00214848F9F75DF90028A2
:1086C8007FF407AA322384F89600A4F89830FFF7BD
:1086D80000BA002A0CBF0120022074E7404B002298
:1086E80001204049404C0B60404B0993404B22709D
:1086F800404D0A9327F048FDFEF7F1BA3C4A3A4B41
:108708000A9211463C4A0A6002225A70374B099372
:1087180020F054FDFEF7E3BA354A334B0A9211466E
:10872800364A0A6001225A70304B099320F046FD00
:10873800FEF7D5BA2E4A2C4B0A921146304A0A60E7
:1087480000225A70294B099320F038FDFEF7C7BA6A
:10875800792A00F01F847A2A00F011849E2A00F0FA
:1087680006849D2A00F0FB83AE2A00F0F183AD2A2F
:1087780000F0E783EF2A00F0E183FD2A00F0CC83C4
:10878800FB2A00F05184FE2A00F04B84F72A00F0FF
:1087980042847B2A00F02684144B0993144B0A93D5
:1087A800FEF79DBA00260020C5490020BC410020E4
:1087B8008C4F0020D34D621000007A44C051002035
:1087C80099FB243F69A2163E39094E3DE3B59E3E0A
:1087D80088FA163E45FE7F3FA7DFA8346441002093
:1087E800525D0020AC470020344200204C47002056
:1087F800B0470020A8470020584200204C420020E3
:1088080040420020D9F8D000B64B90F836109B783B
:1088180011446429A8BF642121EAE17180F8361067
:10882800002B40F004841FF02FFD58E4D9F8D00045
:10883800AC4B90F837109B781144FE29A8BFFE2155
:1088480021EAE17180F83710002BECD0162020F0D7
:108858009BFCD9F8D000E6E70C98A24B417811446C
:10886800B1F5967FA8BF4FF4967121EAE171417086
:108878009B78002B40F00E84D9F8D000D3E7D9F8C4
:10888800D000984B81781144C829A8BFC82121EA93
:10889800E17181709B78002BC5D0142020F074FC06
:1088A800D9F8D000BFE7D9F8D0008E4B41781144F1
:1088B800C829A8BFC82121EAE17141709B78002B23
:1088C800B1D0132020F060FCD9F8D000ABE7D9F87C
:1088D800D000844B01781144C829A8BFC82121EAD7
:1088E800E17101709B78002B9DD0122020F04CFC88
:1088F800D9F8D00097E77B4B0C989B7841791144C5
:108908006429A8BF642121EAE1714171002BB3D029
:108918000E2020F039FCD9F8D00084E7D9F8D0002F
:10892800704B017A9B781144C829A8BFC82121EA55
:10893800E1710172002B3FF476AF0B2020F024FC8C
:10894800D9F8D0006FE7D9F8D000664BC1799B7889
:108958001144C829A8BFC82121EAE171C171002BBF
:108968003FF461AF0A2020F00FFCD9F8D0005AE795
:10897800D9F8D0005B4B81799B781144C829A8BFEE
:10898800C82121EAE1718171002B3FF44CAF092025
:1089980020F0FAFBD9F8D00045E7D9F8D000514BC0
:1089A800417993F802E01144C829A8BFC82121EAF7
:1089B800E1714171BEF1000F40F05A83112F7FF42D
:1089C80061AF30E7D9F8D000464B017993F802E05F
:1089D8001144C829A8BFC82121EAE1710171BEF17B
:1089E800000F40F05E83102F7FF460AF1BE70C99F7
:1089F8003C4B0F790D931744642FA8BF642727EACF
:108A0800E7770F7120F0DAFB0D9B9B78002B3FF482
:108A180033AF0320394620F0B7FBD9F8D00002E77E
:108A28000C98304B01781144FA29A8BFFA2121EAA1
:108A3800E17101709B78002B3FF41EAF012020F0FC
:108A4800A3FBD9F8D000EEE60C98264B81781144A8
:108A58006429A8BF642121EAE17181709B78002B09
:108A68003FF40AAF022020F08FFBD9F8D000DAE6F5
:108A78000C981C4BC1799B78114481F30801C17192
:108A8800002B3FF4F9AE052020F07EFBD9F8D0008A
:108A9800C9E60C98134B817993F802E011446429D4
:108AA800A8BF642121EAE1718171BEF1000F40F095
:108AB800E9820D2F7FF420AFDEE6D9F8D000094B0C
:108AC800C17893F802E01144C829A8BFC82121EA57
:108AD800E171C170BEF1000F40F0C0820F2F7FF42A
:108AE800F9AEA0E6725E0020CA48D0F800E0530054
:108AF800BEF1000F08D09F1801EB87079EF801E030
:108B08007F787745BEF4EDA91A44C34FC34B01EBF8
:108B18008201002201603A801A60FEF7E2B9129AD7
:108B2800FFF79FBB04999B7831F91220B2F5617F5A
:108B38004FF4966191FBF3F3C0F2C08040F6330125
:108B48009142A8BF11460C2FA1F5617191FBF3F179
:108B580000F04581182F7FF4C2AAC9B2C8290B4674
:108B6800A8BFC823D9F8D020D77DD8B2B8423FF4DF
:108B7800B6AADF1BAA4BD07548BF0737FF109B78F2
:108B88000137FFB23BB9002F3FF4A9AA384627F0B6
:108B9800FBFAFFF7A4BA182020F0F6FAF3E7A14A87
:108BA800A14B099210461A68A0494FF47A73B3FB97
:108BB800F2F3C3EB431203EB82030268DB00A1F874
:108BC800A83053077EF588A8994B9A4D0A221A8037
:108BD800994B0A93FEF783B80F2027F0EFF9B4F802
:108BE800903084F89250FA3BA4F89030FEF772B8AF
:108BF800B4EEE77AF1EE10FA40F38B81DFED8F5A8D
:108C08009FED8F6A01E0F0EE676AF4EEC66AF1EE56
:108C180010FA76EEE57AF6DCDFED8A6AF4EEE67AAB
:108C2800F1EE10FA40F1E581DFED845A9FED866A96
:108C380001E0F0EE667AF4EEC67AF1EE10FA77EE1D
:108C4800A56AF6D4DFED817AF4EEE76AF1EE10FA60
:108C580040F3A980DFED7E7A77EEE66A66EEA65AE3
:108C68009FED7C5A9FED7C6ADFED7C7AA5EE856AE4
:108C780026EEA55AE5EE867AE5EE276AFFF73CB9B7
:108C8800774B1B78032B00F020810023FFF796B960
:108C9800744A64491360684B0991664D0A93FEF75C
:108CA8001EB8DFED717AB4EEE77AF1EE10FA44BF40
:108CB800DFED647A37EEC77AFFF766B90C2F00F05C
:108CC800F680182F7FF40BAA00210B464AE7674A63
:108CD8000592FEF715BF664A069B1E68136823F0C7
:108CE80004031360089A012306F4805682F82130A1
:108CF800FEF7FEBF5F4B01220220F2E406F4805625
:108D0800FEF7F6BF38EE678A5B4B5C491870FDEEDC
:108D1800C87AC9F5FA63CDED047ABDF910201203BB
:108D280081FB0201D217C2EBA1121BB203FB02F3B3
:108D380043F30F334B4407EE903AF8EEE77AC7ED6A
:108D4800037AFEF712BA0023BB2A149300F0478176
:108D5800B72A00F04081BE2A00F03B81BD2A7FF48B
:108D6800F7AC4FF6FE71464A2E48D689099090898D
:108D780033440144D381918112F042FFF7F76AFF2F
:108D880012F026FFFBF752FA012027F0FDF9B4F89C
:108D98009030294A0A92FA3B0022A4F8903084F8CD
:108DA8009220FDF79CBFDFED307AF4EEE76AF1EE32
:108DB80010FA44BFDFED237A77EEE66A4EE7314BCF
:108DC800022203208DE4304A164B09931378194D7B
:108DD80043F004031370184B0A93FDF780BFCFB21A
:108DE8002A4B0E915B78BB423FF479A90C4B0D934B
:108DF80038460DF021FA0D9B0E999B781BB1C9B22C
:108E08000C2020F0C1F90137FFB2BCE61A46FEF784
:108E1800D6BB00BF242100200C22002010220020F5
:108E2800725E00204C4700200C570020945400200C
:108E3800C2890020A8470020B0470020DB0FC940A6
:108E4800E4CB1641DB0F49C0E4CB16C1DB0FC93FA9
:108E5800DB0F494092E741B99730083C15A82ABE74
:108E6800CF49002000260020DB0FC9BF1460002076
:108E7800A4470020A05D0020A4210020D34D62104B
:108E88009C410020EE5D0020F43B0020344200208D
:108E980012F0B6FEF7F7DEFE12F09AFEFBF7C6F9FF
:108EA800012027F071F994F88E20FFF7A3B9002765
:108EB800394695E7804B814A09924FF4C8721A8067
:108EC8007F4B804D0A93FDF70ABF27F05BF8FEF74A
:108ED80008B801221346FEF772BB03221346FEF7B9
:108EE8006EBB02221346FEF76ABB07221346FEF743
:108EF80066BB06221346FEF762BB05221346FEF741
:108F08005EBB04221346FEF75ABB08221346FEF73F
:108F180056BBF0EE667A7FE6002101200CF062FE77
:108F2800B4F89030654A0992963B654AA4F89030A7
:108F380000230A9284F89230FDF7D1BE002108463A
:108F4800ECE7FF21002021F0B7F994F88E2011E416
:108F58000121002021F0B0F994F88E2007E40021C7
:108F6800FF2021F0A9F994F88E20FFF7FDBB00211E
:108F7800012021F0A1F994F88E20FFF7F2BB524AA4
:108F88004E4B0993137A43F0010313724C4B0A9327
:108F9800FDF7A5BE4C4A494B0993137A23F0010308
:108FA8001372474B0A93FDF79ABEB0EE677AFEF745
:108FB800DFBF002D3DF4DFAD444C94F88D30002B1D
:108FC8003DF40AAE26F0DEFF002384F88D30FDF76D
:108FD80003BE0221C7E619464FF6FE73C3E61946DB
:108FE8000223C0E64FF4FA6102200CF0FBFDFFF704
:108FF800D3BBF0EE676A25E6F0EE477AFEF7A2BF2C
:109008002E4B09932E4B84F8941084F895002D4D1F
:109018000A93FEF74FBD002104207FE70B20FDF7E0
:1090280057BE0021032079E70021022076E71720A8
:1090380020F0AAF820E4002BBED02549254A09686B
:109048004FF47A7000FB03131360B5E71F4C0BF065
:10905800EDFB002384F88D30FDF7BEBD0F200E9385
:109068000D9220F091F8D9F8D0000E9B0D9A35E5B5
:1090780011200E930D9220F087F8D9F8D0000E9B9E
:109088000D9A9BE40D200E930D9220F07DF80E9B17
:109098000D9A0EE5152020F077F8D9F8D000FFF7E3
:1090A800C2BB10200E930D9220F06EF8D9F8D000B4
:1090B8000E9B0D9A97E400BFC48900204C470020FE
:1090C800B0470020A8470020C44200207C1E002092
:1090D80090640020FC2500202DE9F047C74C636808
:1090E80020469847002800F0C380C54B1B78012212
:1090F800042B84F83C2000F0BD80B4F91610B4F9B4
:109108001820B4F91A3021636263A363BD4B1B882E
:10911800002B69D0BC4DD4ED0C7AD5ED004A95ED05
:10912800050A95ED015A95ED067AD5ED035A95EDA8
:10913800026AF8EEE76AD5ED047AA4EEA60AA5EE6F
:10914800267A67EEC07AA5EEC07AE6EE267A85ED35
:10915800057AC5ED067A2CF0B3FCD4ED0D6AD5ED91
:10916800094A95ED0E0A95ED0A5A95ED0F7AD5ED57
:109178000D7AD5ED0C5A95ED0B6A2063F8EEE66A88
:10918800A4EEA60AA5EE267A67EEC07AA5EEC07A06
:10919800E6EE267A85ED0E7AC5ED0F7A2CF090FC76
:1091A800D4ED0E6AD5ED124A95ED170A95ED135ACE
:1091B80095ED187AD5ED167AD5ED155A95ED146A10
:1091C8006063F8EEE66AA6EEA40AA6EE857A67EE74
:1091D800C07AA0EE657AE6EE867A85ED177AC5ED57
:1091E800187A2CF06DFCA063884FA17F884815F091
:1091F80033FC3B88002B40F08480864ED6F8E05044
:10920800854B1B685B0743D4B5F90070216B636B12
:10921800A06B824A824E92ED026AD2ED006AD2EDCC
:10922800015AC91B2163B5F90270DB1B6363B5F9E9
:1092380004703568C01B07EE900AB8EEE75A07EECF
:10924800901AB8EEE77A07EE903AF8EEE77A36EE3B
:10925800056A36EE877A77EEA57A0135A06382ED46
:10926800026A82ED007AC2ED017A3560BDE8F087C6
:10927800BDE8F0876B4BB4F91600B4F91810B4F9CF
:109288001A2018802063598061639A80A2633DE7A1
:10929800B6F89820322A00F08880002A66D196F81D
:1092A8009530002BB0D06048D6F8FC205F4980FB91
:1092B8000273D217C2EB23122A80D6F8002180FB52
:1092C8000273D217C2EB23126A80D6F80431A78A38
:1092D80080FB0302DB17C3EB2213DB1BAB800023ED
:1092E800CB6086F8953012F08BFCF7F7B3FC12F0E0
:1092F8006FFCFAF79BFF012026F046FFD6F8E050F6
:1093080082E7444E226BD6F8E050B3F5C87F4FF0A1
:10931800000323632B80398818BFD6F8E400B7F818
:10932800008008BF0020B1F5C87F18BFD6F8E83024
:10933800616B02440B440020B8F5C87F6063C6F82F
:10934800E420C6F8E830688052D0D4F838E0D6F87F
:10935800EC10A0637144B8F1010FA880C6F8EC10B6
:1093680068D008F1FF38A7F8008049E7D6F8FC0074
:10937800236B00210344C6F8FC3021632980D6F80A
:109388000001636B61630344C6F800316980A36B15
:10939800D6F80401A1630344012AC6F80431A98060
:1093A80075D0013AA6F8982079E72B8820491F48FC
:1093B800276BA6F8F0300023B5F802E0B5F804C032
:1093C800C0684B608B602363C6F8FC702B80616BB0
:1093D800C6F8001163636B80A16BC6F80411A36320
:1093E800A6F8F2E0A6F8F4C0C6F8F800AB80D8E713
:1093F800A36BC6F8EC30A063A880B2E760470020F2
:10940800604500200437002008370020C489002068
:10941800904700207C1E00201C570020D04F0020C1
:10942800CC4F0020644500201F85EB519C41002053
:10943800781F0020DFF804C1DFF8F0E0C8328CFBA9
:1094480002A9C833D217C2EBE9128CFB03A9DB17B8
:10945800C3EBE913C8316B802A808CFB013CA28ADC
:10946800CB17C3EBEC139B1AAB80CEF80C0012F0B1
:10947800C7FBF7F7EFFB12F0ABFBFAF7D7FE404656
:1094880026F082FEB7F80080D6F8E05069E7254B51
:1094980086F89A101B6886F8942013F4003334D1A8
:1094A80019462148475C0B2F01F10C0110D00133FC
:1094B800182BF7D1B6F8F0101C4B2980B6F8F270CB
:1094C800B6F8F400D6F8F8106F80A880D96068E77D
:1094D800174FD7F800C05900BCF1000F09D001EBB5
:1094E800030E00EB8E0E9CF801C09EF801E0E645E5
:1094F800E0D20B44DFF848E00E4900EB830000237C
:109508003860AEF800300B60D4E70B4B1B78032BA8
:1095180001D00B46C5E726F035FDD6F8E050B6F881
:109528009820C7E7443E0020A48303089C410020FC
:109538002421002010220020CF4900201F85EB5154
:109548000C2200202DE9F0478C4B1B78DB070746DF
:1095580044D58B4B8B4D1C788B4E012C59D01CD38A
:10956800022C07D189498A4A09881288914201D96F
:1095780001241C70EB7AE3B12B89D3B1854B1B789E
:10958800BBB10CF07BFE002800F09B802B7B834254
:109598002CBF0121002131700CE07C497E4A0988EA
:1095A80010886A7B801A8842E2DAEB7A0024002B62
:1095B800E2D131782A79632A06D8022C774E00F056
:1095C800BA803378002B5DD1754AAB7A8C4238BFAC
:1095D8000C461470002B4CD1BDE8F0876B4B694DDD
:1095E80019885B88E878CB1A83EAE3728142A2EB98
:1095F800E3721DD32B788B421AD3614B1C78E01E83
:10960800012861D96749097802294FD0012C5E4E9B
:10961800A5D15F4A5D491288687B0988121A914270
:1096280039DD5D4A12888A42A4D200241C70A1E761
:10963800B1EB400FE1DC524B1C78E11E012940F2EE
:109648009480022ADEDC57494F4E0878DFF84481BF
:10965800DFF844C1DFF838E1002103240228347020
:109668001C7088F80010ACF80010AEF8001081D11A
:109678001FE0012C71D0022C0BD10720BDE8F04768
:1096880026F09CBC7068381A474B984258DD7270B7
:109698009AE7BDE8F08702241C706BE7022AD2DD46
:1096A8004049097802294FF0040464D13949364EFB
:1096B80009783E48022ACCBF00220122C28081805C
:1096C8004BE70221317075E7022A9BDC95F800C050
:1096D80091FBFCFC0CF1010CBCF1080FDFF8B4A005
:1096E800304EA87895F801E096F800802A4CDFF80B
:1096F800A090254EA8BF4FF0080C8AF800C01FFAAA
:109708008CFA10FB0AF01EFB0AFE80B2DFF88CA070
:109718002080A9F800E000244FF0640EB8F1020F91
:1097280034701C70CAF804408AF801E07FF439AF3D
:109738000FFA8CF1BDE73078A0B901237760337058
:10974800C2F164021A4B00FB02F083FB0023C0172E
:10975800A0EBA3506430707036E70820BDE8F047EE
:1097680026F02CBC7368F81A8EE7032C96D10D49A5
:10977800097802299AD0044EFCE600BF1B5200204B
:10978800AC2600203C470020BC2600208444002052
:10979800B02600207E450020AE260020B4260020FA
:1097A800CF490020604500207F969800644500203E
:1097B8006BCA5F6B022828BF022010B4084C094B03
:1097C800207000EB8002C0EBC20207495DF8044B31
:1097D800013003EB4203C0B20B6026F0D5BC00BFDA
:1097E80034420020525D0020AC47002008B512F03A
:1097F80007FAF7F72FFA12F0EBF9FAF717FD01203D
:10980800BDE8084026F0C0BC1C4C08B50121022068
:10981800FCF7B4FE237803F00502052A2AD003F0EA
:109828000903092B08D000210120FCF7A7FE00211D
:109838000846FCF7A3FEFEE7114A124B11681A68A6
:109848000B68114C4FF6FE7003400B6013882068BC
:1098580023F001031B041B0C138018B12A220023D8
:109868008271C37102224E21FBF7ACF82068FCF725
:1098780045FED8E71EF04CFF2378D0E7602E002085
:10988800C8260020CC260020E42E002008B5FAF7D0
:1098980065FE12F0B5F9F7F7DDF9BDE8084012F0FA
:1098A80097B900BF08B512F0ABF9F7F7D3F9BDE8DF
:1098B800084012F08DB900BF2DE9F04FBF4B1E785C
:1098C8008BB0002E40F0BC80BD4BBE4C1D78DFF83D
:1098D80014A3DFF81493DFF8148305F00105A4F14D
:1098E8000A0B54F80A3CBBB1CC2707FB06B718464D
:1098F800FCF7DCF980B154F80A0CFCF7CFF914F83E
:10990800023C8BB9242831D0F5B154F80A3C1846EA
:10991800FCF7CCF90028EED10136032E04F1CC0473
:10992800DFD10BB0BDE8F08F012B23D0022B2BD059
:10993800032B37D0042B67D0052B40D0062B4FD0F4
:1099480054F80A2C1346D2E754F80A3C23281A463E
:1099580000F087819C4991F832108142C7D19B4B16
:10996800CAF80090C3F80C801346C0E7012304F836
:10997800023CCAE74D2854F80A2C0CBF02230023E6
:1099880004F8023C1346B2E700233C2804F8023CE2
:1099980045D03E28D4D10122032304F8012C04F831
:1099A800023CB2E7C02814D80022042304F8050CAE
:1099B80004F8040C04F8062C04F8023CA5E714F893
:1099C800063C14F8052C9A422FD814F8043C83421C
:1099D80003D0002304F8023C97E7062304F8023C6E
:1099E80014F801ECBEF1000F00F08481BEF1010F04
:1099F80000F0C88101360023032E04F8023C04F16C
:109A0800CC047FF46EAF8CE714F8043C04F8030C24
:109A18005840052304F8040C04F8023C75E70322B7
:109A280004F8013C04F8022C6FE714F8042CF91828
:109A38004240013304F8042C04F8063C887264E7B9
:109A4800634B186800283FF46CAFFCF7C5FFDFF8DC
:109A5800A0A1604DDFF89C91DAF80000FCF726F928
:109A680000283FF45EAFDAF80000FCF717F9092880
:109A78001BD03F2819D02B68002B66D1042800F092
:109A8800AC810C2800F0E6807F28E5D0A0F1200208
:109A9800D2B25E2AE0D80BB92028DDD05A1C09F8CA
:109AA80003002A600DF0BCFED6E72C68002C5AD1C2
:109AB800494B264603F59478002E08BF1E46083306
:109AC8004345F9D1002E00F07C81A3F1080B3068E2
:109AD800DBF80020075D135D9F42204402EB040180
:109AE80040F06D81671E4F4422460BB9FD2A5CD9B0
:109AF80007F8013F01322A6010F8013F11F801EF21
:109B08009E45F2D00AB1B34512D034480DF090FE0C
:109B1800B34508D356F8080B0DF08AFE09200DF05E
:109B28007FFE5E45F6D92E480DF082FE2A68002495
:109B3800944291D2661E4E4416F8010F0DF070FE45
:109B48002B6801349C42F7D386E70C2800F082800A
:109B58000A2851D00D284FD07F2800F00081FF2B14
:109B68003FF67AAF92E71C4F4FF0000B07F5947859
:109B78005E4602E0083747450DD022463968484618
:109B8800F7F766FB0028F5D1BB46002EF2D13E461A
:109B980008374745F1D1002E99D1BBF1000F3FF4AA
:109BA8005BAF0E480DF044FEB4E7511C202009F8C5
:109BB8000200296009F801300A46A4E72F42002074
:109BC8001B520020528500204060002000ED00E07C
:109BD8000831002010320020048003088096030812
:109BE80088960308FC9F0020EFBEADDE0400FA054E
:109BF8000C310020103100200DF09BFE23217F48FE
:109C08002CF032FF002800F0E680A0EB0900286065
:109C180088B1431E19F80310202940F0EC8009EBA5
:109C2800030204E012F8011D20294CD10346581EF6
:109C3800002BF7D12B604FF48072002148462CF09E
:109C4800FCFE6F4B1B78002B3FF46BAE6D480DF09C
:109C5800EFFD01E76C480DF0EBFD6A480DF0E8FDFB
:109C6800FAE66A496A48C9786A4ADFF8D8E1C2F868
:109C78000831003118BF012101706749C2F80C1181
:109C88004021C2F8103182F8141182F81551634945
:109C980063480B6002F58672CEF80020584A01230B
:109CA80013700EF015FA57480DF0C2FD4FF400601E
:109CB80009F082FF5B4B93F83230232B00F093803E
:109CC80014F8023C3AE62B60574C002204F59478CD
:109CD80009F8032002E00834444578D02168484652
:109CE80010F0BCFD0028F6D0444570D26368984750
:109CF80000239FE74D4BADF822E00FCB0DF1280C68
:109D080002AF87E80F004CF824ED14F8051C14F88E
:109D1800033C069404EB010E624639464FF0010CF1
:109D280006A8CDF81CE0ADF820308DF824C000F06E
:109D38008BF8E8B9019F002304F8023C002F3FF498
:109D4800EBAD54F80A0C0CF067FD013654F80A0C18
:109D5800B847032E04F1CC047FF4C3ADE1E5013B21
:109D6800002233482B6009F803200DF061FD73E6EB
:109D7800029A304B03923946A4F10A0002930CF080
:109D88008BFCD7E714F8053C14F8032C06942344FD
:109D980007936E2A4FF0000308930993ADF820202B
:109DA8007FF428AE06A8F7F7D5FA06A8F7F7C6FA9B
:109DB80006A8F7F7C3FA06A8F7F7C0FA1AE6224684
:109DC800A0E61D48A3F1080B0DF032FDA2E61B48E2
:109DD8000DF02EFD8CE728681AE708480FF041FCC3
:109DE8000BB0BDE8F08F164A14F8023CC2F80C809C
:109DF800CAF80090A2E5034666E700BF10310020CC
:109E08002F420020889603089096030834420020C9
:109E1800302700207C1E0020F53B00080C31002074
:109E2800BC9603084060002004800308E86C03081F
:109E3800B8960308F48A0020809603089C960308C5
:109E480000ED00E0083100202DE9F04FB0F908508E
:109E58000D81EDB2442D8DB00C46164600F00782F8
:109E680007462FD9812D00F0458200F28180542DBC
:109E780000F0AE8040F296816E2D00F0C681802DF4
:109E880040F0B280B44B1D780B3D15F0FF0512D0A1
:109E9800B24F00220A2621683B88481C20600E70B9
:109EA8002168FF2B02F10102A8BFFF23481CAA4228
:109EB80020600B70EFDB01252B46284663810DB02F
:109EC800BDE8F08F052D00F0C0811ED8022D77D097
:109ED80040F22F81032D00F08D81042D40F0848005
:109EE8002A469F492046F7F73BFA00212046F7F714
:109EF80067FA22680021531C0125236028462B4657
:109F0800117063810DB0BDE8F08F242D56D040F25A
:109F1800C880282D00F0B381382D65D10A68914B8F
:109F28000125511C216015702268052150192060F7
:109F3800117022680A2150192060117022680021CE
:109F4800501920601170226819785019206011701A
:109F5800226859785019206011702268997853192D
:109F680023602B461170284663810DB0BDE8F08F41
:109F7800A02D11D040F2B380B82D00F0B981FE2D8C
:109F880032D1794D05F1080635F8021B2046F7F75E
:109F980017FAAE42F8D18EE7744B08461968F7F7FE
:109FA800F7F9734B20461968F7F7F2F9714B1968FE
:109FB80020460125F7F7ECF92B467EE76E4BF6E7CE
:109FC80004226E4920460125F7F7CAF92B46CAE74D
:109FD8000B6800215A1C2260197022680125531948
:109FE80023602B461170BEE72146284608F096FDEF
:109FF800014600287FF45FAF742D00F0F180772DC3
:10A0080009D13B687A689A4240F0D1815C4A20467F
:10A0180026F072F94FE7F52D00F0CD817A683E6899
:10A02800292DA2EB060300F0708240F24D82392DF3
:10A0380001F04E82532D40F08182721C3A603178D3
:10A04800032900F208854A1E4E4D4F48D2B202EB52
:10A05800420205EB42020170557800293FF42BAF0C
:10A06800013BDBB2AB4240F0F684821C0023136054
:10A07800536013725DB101353B682844013A0133DE
:10A088003B6013F8011C02F8011F9042F7D13F4BC7
:10A098001B78002B3FF40FAF012524F0AEFC2B46B4
:10A0A80061E7202DA0D10B68394D591C6A782160D1
:10A0B8001A7023682A78591C21601A702368AA78B4
:10A0C800591C21601A7029892046F7F779F9236805
:10A0D8006A79591C21601A702268A9790BE7822DC8
:10A0E80082D10B682B4A2C4D1178294A581C2060C4
:10A0F800197011892046F7F763F9284B22681B88E5
:10A10800FF2B02F10101A8BFFF2321601370A9688A
:10A1180081F3100189B22046F7F752F9296801F353
:10A128000F0189B22046F7F74BF91D4B22681978C1
:10A13800E1E6012D7FF458AF0B680022591C21601D
:10A148001A7023685A1C22601D7022682521531C2E
:10A1580023602B46117006E70E4500208426002058
:10A168003A4200203D5D002064450020ACF7FF1F07
:10A17800B0F7FF1FB4F7FF1F8C5E0020C4960308DA
:10A1880039F602089C6D030874600020BD26002083
:10A198003C4700207E450020704400208444002075
:10A1A800CF490020522D7FF41FAF0A68B04E531CD0
:10A1B8000321236006F10C071170334606200121A4
:10A1C8002268551C256011702268BB4202F101010A
:10A1D8002160107000F0C8809979D8790633EFE7CC
:10A1E8003B687A689A4240F0DE80A24A204626F010
:10A1F80083F860E60B685A1C0A601D700B685A1CCD
:10A208000A601D700A68002175E69B4B0A681B8866
:10A218009A4DFF2BA8BFFF23511C21601370A9681A
:10A2280081F3100189B22046F7F7CAF8944B20460B
:10A238001988F7F7C5F8296801F30F0189B2204694
:10A248000125F7F7BDF82B468DE60B228D492046F0
:10A25800F7F786F808228C492046F7F781F8012598
:10A2680007228A492046F7F77BF82B467BE6002A27
:10A278003FF421AE864B136001252B4673E60B682D
:10A28800DFF83C82834E591C022221601A70236831
:10A2980006275A1C22601F7023680A22591C216055
:10A2A8001A70236801255A1922601D70B8F8001029
:10A2B8002046F7F785F8B8F802102046F7F780F837
:10A2C80023685A1922601F70236850225919216087
:10A2D8001A7023680022591921601A7031882046A3
:10A2E800F7F76EF871882046F7F76AF82B463AE6D2
:10A2F800694B5CE6694B1E780A3E16F0FF063FF490
:10A30800DAAD674B674F1E4403F101080A2314E0D6
:10A31800502B00F0AA80002529462268501C206096
:10A3280020461370F7F74CF829462046F7F748F807
:10A3380046453FF4C0AD18F8013B0A2BE8D15A4A0C
:10A348009568116805EB85054FF6FF726D0095421B
:10A35800A8BF15469142A8BF114625EAE57521EA2E
:10A36800E171ADB289B2D8E7504B21681A78481C20
:10A3780020600A70002A3FF49EAD013AD2B202EB87
:10A38800420206EB42025578002D3FF494AD0135A8
:10A398001D440133226813F8011F501C9D422060A0
:10A3A8001170F7D187E55A1C3A6019781DE75A1CD5
:10A3B8003A6019782AE63B687A689A4241F09880B0
:10A3C8003B4BFF221A704FF000093A4D0AF0F2F9A0
:10A3D80049462022384885F800902CF02EFB8DF84D
:10A3E8000C909DF80C30072B01F20B81DFF8D4801C
:10A3F800314F4A469DF80C3003EB430308EBC30387
:10A408005B7CE3B19DF80C3003EB430308EBC3031B
:10A4180020215B699BB19DF80C3003EB430308EBEB
:10A42800C303586947F82200FBF7ACFE2B7857F8AE
:10A438002300FCF769F82A780132D2B22A709DF815
:10A448000C300133DBB28DF80C309DF80C30072B43
:10A45800D0D92368591C21601A70002E3FF42BAD07
:10A46800164B336001252B467DE5BD68396869E7E1
:10A478009C6D030899F6020884440020704400206B
:10A48800CC490020CC960308D8960308E496030824
:10A498005D28010874260020443E00200E45002057
:10A4A800F86C0308782600204026002074600020FD
:10A4B800D81F00207A3F0020643C0020ADFC010832
:10A4C8008C4100205C580020212D37D13346721C66
:10A4D8003A60184D13F8022B6A703B6073782B7042
:10A4E800F31C3B60B378AB703846F6F727FF3B6840
:10A4F8002881591C1A46396012F8021B69713A60A2
:10A508005B78AB7101252B462DE5731C3B603378D6
:10A518000A2B01F01580502B40F041873846F6F79A
:10A528000DFF054E30803846F6F708FF012570808C
:10A538002B4618E53C470020742600200B3DEF2DE4
:10A5480000F2898201A050F825F000BF49B2000846
:10A558005FAA00085FAA00085FAA00085FAA0008AF
:10A568005FAA00085FAA00085FAA00085FAA00089F
:10A578005FAA00085FAA00085FAA00085FAA00088F
:10A588005FAA00085FAA00085FAA00085FAA00087F
:10A598005FAA00085FAA00085FAA00085FAA00086F
:10A5A8005FAA00085FAA00085FAA000813B10008A4
:10A5B8005FAA0008A1B200085FAA00087FB20008DD
:10A5C8005FAA00085FAA00085FAA000821B2000875
:10A5D8005FAA000883B100085FAA0008E1B000087C
:10A5E8005FAA0008BBB000085FAA0008A9B000086D
:10A5F8005FAA000855B000085FAA000871B40008F7
:10A608005FAA00085FAA00085FAA00085FAA0008FE
:10A61800BF9E00085FAA000845B400085FAA0008AA
:10A628005FAA0008BFB400085FAA00085DB300086D
:10A638005FAA00085FAA00085FAA00085FAA0008CE
:10A648005FAA00085FAA00085FAA00085FAA0008BE
:10A6580005B400085FAA0008B7B300085FAA00089D
:10A668005FAA00081FB300085FAA00085FAA0008D5
:10A678005FAA00085FAA00085FAA00085FAA00088E
:10A688005FAA0008BBB200085FAA0008D3AF0008A1
:10A698005FAA000829AF00085FAA00083DAE0008BD
:10A6A8005FAA000815AE0008F7AD0008DBAD00088A
:10A6B8005FAA00085FAA00085FAA00085FAA00084E
:10A6C8005FAA00085FAA00085FAA00085FAA00083E
:10A6D8005FAA00085FAA00085FAA00085FAA00082E
:10A6E8005FAA00085FAA00085FAA00085FAA00081E
:10A6F8005FAA00085FAA00085FAA00085FAA00080E
:10A708005FAA00085FAA00085FAA00085FAA0008FD
:10A718005FAA00085FAA00085FAA00085FAA0008ED
:10A728005FAA00085FAA00085FAA00085FAA0008DD
:10A738005FAA00085FAA00085FAA00085FAA0008CD
:10A748005FAA00085FAA00085FAA00085FAA0008BD
:10A758005FAA00085FAA00085FAA00085FAA0008AD
:10A768005FAA00085FAA00085FAA00085FAA00089D
:10A778005FAA00085FAA00085FAA00085FAA00088D
:10A788005FAA00085FAA00085FAA00085FAA00087D
:10A798005FAA00085FAA00085FAA00085FAA00086D
:10A7A8005FAA00085FAA00085FAA00085FAA00085D
:10A7B8005FAA00085FAA00085FAA00085FAA00084D
:10A7C8005FAA00085FAA00085FAA00085FAA00083D
:10A7D8005FAA00085FAA00085FAA00085FAA00082D
:10A7E8005FAA00085FAA00085FAA00085FAA00081D
:10A7F8005FAA00085FAA00085FAA0008B1AD0008B8
:10A808005FAA00089BAD000889AC00085FAA000891
:10A818005FAA00085FAA00085FAA00085FAA0008EC
:10A828005FAA00085FAA00085FAA00085FAA0008DC
:10A838005FAA00085FAA00085FAA00085FAA0008CC
:10A848002DAC00085FAA0008BDAB00085FAA00088D
:10A8580023AB000809AB0008EDAA00085FAA0008AE
:10A86800D3AA00085FAA0008ABAA00085BAD0008DD
:10A87800FDAC00085FAA00086DAD00085FAA0008DB
:10A888005FAA0008B3AC00087DAA000869AA0008FE
:10A89800D5AC000841AA00081FAA00085FAA000852
:10A8A80007AA00085FAA00085FAA00085FAA0008B4
:10A8B8005FAA00085FAA00085FAA00085FAA00084C
:10A8C8005FAA00085FAA00085FAA00085FAA00083C
:10A8D8005FAA00085FAA00085FAA0008EDA900089F
:10A8E8005FAA00085FAA000895A900085FAA0008E7
:10A8F8005FAA00085FAA00082FA900085FAA00083D
:10A908005FAA00085FAA000815A90008B74B1B78C2
:10A91800DB0700F1A0800125FEF7C4FFF9F786FCEC
:10A928002B46FFF720BB3846F6F708FD3B68ADF825
:10A938000C001A46591C396012F8021B3A608DF84F
:10A948000E105A788DF80F20DA1C3A609A788DF834
:10A9580010201A1D3A60DA788DF811205A1D3A60D5
:10A968001B798DF8123003A80023ADF81430F6F7E0
:10A978003DFC9F4A9F4B1268801A4FF0010561F118
:10A988000001C3E904012B46FFF7EDBA731C3B60D5
:10A9980033780F2B5FD8B21C3A60C3EBC303964AD7
:10A9A8007178D154F11C39601344B2785A70321D51
:10A9B8003A60F2789A70721D3A603279DA70B21D94
:10A9C8003A6072791A71F21D3A60B2795A7106F1D9
:10A9D80008023A60F2799A7101250EF0BFF92B4608
:10A9E800FFF7C1BA3846F6F7A9FC844EF08138461D
:10A9F800F6F7A4FC0125B0812B46FFF7B4BA384618
:10AA0800F6F79CFC7E4A00EB80004300012513808A
:10AA18002B46FFF7A8BA3846F6F790FC794E3082F5
:10AA28003846F6F78BFC70823846F6F787FC012526
:10AA3800B0822B46FFF797BA3346721C3A6013F878
:10AA4800020B3B60F31C71783B60B2781CF01EF877
:10AA580000287FF430AA4FF0FF352B46FFF783BA62
:10AA6800694B6A4918684E2201252AF0E9FE2B46EF
:10AA7800FFF779BA3246731C3B60654B12F8021B2C
:10AA880019703A6072785A70F21C3A60B2789A700B
:10AA98003846F6F753FC5F4B0125D8802B46FFF765
:10AAA80062BA731C3B603078060600F1F2854F4BA2
:10AAB8001B78DD073FF5FFA9032828BF00200125E3
:10AAC800FEF778FE2B46FFF74EBA484B1B78D8079F
:10AAD8003FF5F1A90125FEF7D9FEF9F7A7FB2B46AB
:10AAE800FFF741BA414B1B78DA073FF5E4A94A4A18
:10AAF8001378012543F0040313702B46FFF733BA8C
:10AB08003A4B1B78D9073FF5D6A9444B4FF4C87286
:10AB180001251A802B46FFF726BA092B9BDDDFF8A3
:10AB280000813346721CD8F800503A6013F8022BA3
:10AB38002A703B607378AB70F31C3B60B378642B6E
:10AB4800A8BF6423321D6B713A60F378642BA8BFE9
:10AB58006423721DAB713A603379EB71B31D3B60AE
:10AB68007379642BA8BF6423F21D2B723A60B37902
:10AB7800EB7006F108033B60F3792B713846F6F762
:10AB8800DDFB7A683B686881D11A00290CDD591C05
:10AB9800D8F800003960521A002A1978417203DD8A
:10ABA8009A1C3A605B78437001251EF007FB2B4620
:10ABB800FFF7D9B9144B1868F31C02462136991EC1
:10ABC800396013F8031C1170591E396013F8021C00
:10ABD80051703B6013F8011C91700333B34202F1CA
:10ABE8000302ECD11DF050FBFFF765B91B520020A2
:10ABF80090640020D81F0020583D00209C41002070
:10AC0800AC4100201C590020AC470020DC8A030816
:10AC180094410020C0510020F43B0020C48900204A
:10AC2800B0470020C3F34705122D3FF614AFBDB15E
:10AC38000CAB0DF10A0803EB45094646A9F12609B4
:10AC48003846F6F77BFB26F8020F4E45F8D1A24BA3
:10AC580038F8022F23F8022FB045F9D1112D09D861
:10AC68009E4A6B00023B13440021223223F8021F44
:10AC78009342FBD19A4A01231D461370FFF773B91B
:10AC8800731C98493B600A783378002A40F0E484C2
:10AC980004220A70944A9B001380FAF783FD934BB1
:10ACA800012598612B46FFF75EB93846F6F746FB53
:10ACB8008F4E30803846F6F741FB70803846F6F7FD
:10ACC8003DFB0125B0802B46FFF74DB93346721C7A
:10ACD8003A60884A13F8021B11703B60864A737801
:10ACE8009370F31C3B60854BB2789A7001252B4614
:10ACF800FFF739B90D2B7FF4AEAE731C3B60357886
:10AD0800072D3FF6A8AEDFF8108238460C26F6F776
:10AD180015FB06FB05F608EB0605A8803846F6F78E
:10AD28000DFBE8803846F6F709FB3B6828811A4690
:10AD3800591C396012F8021BA9723A605B78EB72F1
:10AD48003846F6F7E3FA012548F806002B46FFF7E0
:10AD58000AB93846F6F7F2FA694B012518802B46EE
:10AD6800FFF701B9DFF8B48198F80030002B3FF401
:10AD7800A2A8644E00253846F6F7E0FA1DF0B4FBA9
:10AD880098F80030A6EC010A01359D42F3DBFFF785
:10AD980092B85D4E002338463360F6F7B7FA0125BE
:10ADA80030602B46FFF7DFB83346721C3A6013F861
:10ADB800025B3B60F31C70783B60B178002D00F0BB
:10ADC8008084012D7FF477A80BF01AFA2B46FFF741
:10ADD800CAB8731C3B603378002B00F034844FF4FE
:10ADE8000040012508F0E8FE2B46FFF7BCB8474BAA
:10ADF8001B7813F001017FF42EAE731C3B60307892
:10AE080001250AF0EFFE2B46FFF7ADB83346721C5A
:10AE18003A60394A13F8021BD1703B603C4A737898
:10AE28005371F31C3B60354BB278DA7001252B4621
:10AE3800FFF799B83846F6F781FA3846F6F77EFAFA
:10AE48003846F6F77BFA3846F6F784FA3B68314D10
:10AE58001946581C2A68386011F8020B82F82C0031
:10AE68003960597882F83610D91C39609B7882F895
:10AE780037303846F6F76EFA3846F6F76BFA384642
:10AE8800F6F768FA38462E68F6F758FA70873846A3
:10AE98002E68F6F753FA3B687A683087D11A012989
:10AEA8000ADD591C2A6839601B7882F82E3038462A
:10AEB800F6F750FA3B687A68D31A032B09DD38464F
:10AEC8002E68F6F73BFA708638462E68F6F736FA9B
:10AED800B086286886E600BF3E3300204033002055
:10AEE80064330020EA3A0020CC490020D81F002013
:10AEF800C0510020805400209C410020AC4100201B
:10AF0800A6210020E8300020443E00201B520020EB
:10AF18007C4F0020AC470020983C00200E450020C4
:10AF2800731C3B60B24DDFF8EC82337888F805304B
:10AF380038462E68F6F702FA308438462E68F6F757
:10AF4800FDF97A683B68F083D11A072915DD384680
:10AF5800F6F7F4F9A8F80A003846F6F7EFF9A8F872
:10AF68000C0038462E68F6F7E9F9708438462E68E2
:10AF7800F6F7E4F93B687A68B084D11A03290BDD47
:10AF88003846F6F7DBF9A8F80E003846F6F7D6F992
:10AF98003B687A68A8F81000D21A002A05DD591C07
:10AFA8002A6839601B7882F82630F9F7A1F81FF073
:10AFB80083FD904B1B68002B00F053832868012504
:10AFC8001CF0D2FD2B46FEF7CEBF3346721C3A600A
:10AFD800DFF8408213F8022B88F802203B60864A8B
:10AFE80073781370F31C3B60844DB3782B71331D59
:10AFF8003B60F378092BA8BF09233846AB70F6F7F6
:10B008009DF93B687A682880D11A012905DD384600
:10B01800F6F794F93B687A68E8819A4207D05A1C97
:10B028003A601B78003318BF012388F80730F9F716
:10B038005FF83B687A689A423EF43DAF5A1C3A6022
:10B048001B78EB7001252B46FEF78DBF731C3B6008
:10B0580033780E2B3FF6FFACB21C3A6070780328A9
:10B068003FF6F9AC6649062202FB03F28B18F51C81
:10B0780058713D60B0788854321D3A60F2785A7041
:10B08800721D3A6032799A70B21D3A607279DA703C
:10B09800F21D3A60B2791A7101252B46FEF763BF9B
:10B0A800731C3B60574B32785A7501252B46FEF7C7
:10B0B8005ABF721C3A6035781F2D3FF6CCAC052B71
:10B0C8007FF4C9AC3846F6F721F94F4B43F8250011
:10B0D8001BF04EFDFEF7EFBE4B4D05F1400638461E
:10B0E800F6F72CF93B68A5F88000591C1A46396018
:10B0F80012F8021B85F882103A605B7885F8833075
:10B108000435AE42EBD1FEF7D6BE731C3B603578F2
:10B118000191132D3FF69FACB31C3B60707825F06E
:10B1280025F900283FF497AC384B027803F825201E
:10B13800F21C3A6003EB8505B2786A70321D3A60FA
:10B14800F278AA70721D3A603279EA7003F1500001
:10B15800019902E00433834207D01A78002AF9D112
:10B168009D78DA789542F5D20121294B81F00101C9
:10B17800012519702B46FEF7F6BE731C214D3B6066
:10B1880033782B723846F6F7D9F8A8833846F6F79D
:10B19800D5F828833846F6F7D1F83A686883531CFF
:10B1A8003B601278EA747A68D31A032B00F32C8276
:10B1B8003B68D11A05290EDD5A1C3A601B78EB72E0
:10B1C8003846F6F7A3F83B68E8605A1C3A601B78E3
:10B1D8002B743B687A68D21A002A7EF76CAE5A1C28
:10B1E8003A601B7885F8213001252B46FEF7BBBE57
:10B1F800AC470020D03B0020904100201C59002083
:10B20800503E00201460002048480020D834002018
:10B218004C1C002080540020731C3B60CB493078C4
:10B228000870D21A002A7EF746AEB31C3B607378CA
:10B23800003318BF012301254B702B46FEF793BE40
:10B24800C349102B4FF0000228BF10230A604A6040
:10B258008A60CA600A74002B3EF42DAE3A68013940
:10B26800134401323A6012F8010C01F8010F9A42B6
:10B27800F7D1FEF720BE3846F6F760F8B54E3060D5
:10B288003846F6F75BF870603846F6F757F8012548
:10B29800B0602B46FEF767BEAF4E002333603846DA
:10B2A800F6F734F833680125034333602B46FEF77D
:10B2B8005ABEAA4B1B68002B3EF4FDAD17F0CAFC22
:10B2C800FF283EF4F8AD3846F6F738F83F2840F244
:10B2D800EB81A34E002535703B687A68B080D21A9E
:10B2E800012A7EF7E8AD1A46591C396012F8021B8C
:10B2F800B1700CA83A6000225D7800F8242D17F090
:10B308007BFC9DF80C30AB423EF4D5AD284617F0D7
:10B3180097FCFEF7D0BD934B1B78012B3EF6CBADC7
:10B32800731C31463B60DFF8688211F8023B88F8ED
:10B338000230F31CD21A3960012A70783B6040F35E
:10B348009B813846F5F7FAFF0125A8F800002B463F
:10B35800FEF709BE731C3B607C4B3278DFF8F8813E
:10B368001A700023C8F800303846F5F7CFFF3A685E
:10B37800D8F800307C49774D0343501CC8F800309A
:10B38800386013780B723846F5F7D8FF28603846CE
:10B39800F5F7D4FF68603846F5F7D0FFA86038465F
:10B3A800F5F7CCFF3846F5F7C9FFFEF784BD731CE7
:10B3B8003B6096F80080B8F1110F3FF64CABB31C18
:10B3C8003B606A4D737805F818303846F5F7B6FFD4
:10B3D80040F6CA039842A8BF184640F2EE239842A6
:10B3E80005EB4801B8BF18460125A0F2EE222B460E
:10B3F800192092FBF0F24A70FEF7B5BD3346721C75
:10B408005B4D3A6013F8022B2A713B6073786B71BD
:10B418003846F5F793FF3B6828805A1C3A601B783A
:10B42800AB713846F5F78AFF3B6868805A1C3A606A
:10B438001B78EB7101252B46FEF795BD3346711C31
:10B4480039604C4913F8020B88703B60707848707B
:10B4580093423EF430ADF31C3B60474BB2781A720E
:10B4680001252B46FEF77FBD0722B3FBF2F2C2EBA4
:10B47800C2015B1A7FF4EFAAD2B202F1FF395FFA78
:10B4880089F9002A3EF417ADDFF8F0A009F10109A7
:10B498009846731C3B6096F90010384B002593F9C9
:10B4A80002208A4203F1080300F085800135062D49
:10B4B800F5D1FFF7D0BA324B06F1080201363E60EB
:10B4C80016F8011C03F8011FB242F7D1FEF7F3BCCE
:10B4D800731C3B6033780A2B5CD03846F5F73AFF8B
:10B4E8003846F5F737FF3846F5F734FFFEF7E3BC83
:10B4F8005A1C19463A60204811F8022B027039602C
:10B508005B784370042A06D9FF2A3EF45CAF2268B0
:10B518000021FEF7F0BC1B490978994203D8022A9A
:10B52800F5D1FF2BF3D1236801255A1922601D702C
:10B53800002E3EF4C0AC144B33602B46FEF713BD0F
:10B548003846F5F7FBFE114EFEF7ECBFE83B00204E
:10B5580078410020982E00208C5E00202052002088
:10B5680024520020705E002014600020F035002076
:10B57800DC510020BC410020D81F00204060002082
:10B58800136000200E450020752801088C4100201A
:10B59800725E0020B31C3B604D4B72781A70F21C2F
:10B5A8003A60B2785A70321D3A60F2789A70012582
:10B5B8002B46FEF7D8BC0AEBC50B38468BF80210B1
:10B5C800F5F7BCFE3B682AF835001A46591C396065
:10B5D80012F8021B8BF803103A605A788BF8042093
:10B5E800DA1C3A609A788BF806201E1D3E6008F136
:10B5F8000108DB788BF80530C1457FF44AAFFEF7C8
:10B608005ABC4A46FEF725BF3846F5F797FEA88488
:10B618003846F5F793FE3B687A68E884D11A03291F
:10B628007FF7C7AD1A46591C396012F8021BA97773
:10B638003A605B7885F820303846F5F77FFE3B683E
:10B648007A686884B5E5234A1368012523F4004322
:10B6580013602B46FEF787BC042A7EF42CACFFF758
:10B6680019BB1D481D491E4A1E4B036001250B606E
:10B6780013602B46FEF777BC1B4BB1781A8801255F
:10B6880012FB00F22B4692FBF1F2A8F80020FEF71D
:10B698006ABC00F07F00032828BF002001250AF0BB
:10B6A800CBFD2B46FEF75FBCC50800F0070301354C
:10B6B8000133EDB20D4E28461946737018F090F913
:10B6C80009E601251CF06EFC2B46FEF74CBC00BFBA
:10B6D8003D5D0020A4470020FC4F00205050002072
:10B6E800B8500020F5030008CA3F0020245200206B
:10B6F8002DE9F04F2DED0E8BDFF8F4B093B0DBF8A9
:10B708000420049058469047002800F08E82BBF829
:10B71800A87000218BF85110002F6DD1BBF93A00A9
:10B72800DBF82450DBF82810BBF93860DBF8204040
:10B73800BBF93C20DFF8BCA0401B521A341BCBF8E5
:10B7480030009BF85210CBF82C400BF12C00CBF8B2
:10B75800342013F081F9DAF80020940041F152877F
:10B76800DBED0C5A1F4CDBED0B7A1F4994ED406A58
:10B77800D4ED416A94ED427AD4F80C2109681B4B48
:10B788000293B8EEE58ADBED0D5AF8EEE77AF8EEAB
:10B79800E58A013277EE867A38EE268A78EE878A4D
:10B7A8008A42C4ED407A84ED418AC4ED428AC4F8E5
:10B7B8000C2101F0588393F800E0BEF1140F03F058
:10B7C80004800023D4F814510393062D01F2A584B4
:10B7D800DFE815F0391726178F156C16100CD616DA
:10B7E800F11500BF002000207837002060450020B8
:10B7F800945400201C570020DE4BDF481A6805933C
:10B808004FF47A75B5FBF2F2C2EB421502EB8502F2
:10B81800D500DA4BDFF8C88344780293ADB2AF4263
:10B828001E78B8F9060003F0EA80DBF87C30BBF933
:10B838003810DBF8602003F1010E07EE901A0A4475
:10B84800BEF1010FCBF87CE0CBF86020F8EEE77A88
:10B8580003F0E280DBED1B5ADBED1D6A07EE10EA10
:10B8680037EEE56AB8EEC75A012F86EE057A37EE4D
:10B87800257A77EEC77A8BED1C7AE7EE866A8BED30
:10B888001B7AF0EE667ACBED1E6ACBED1D6A03F0EB
:10B898005584DBF89030BBF93A10DBF8642003F1EB
:10B8A800010E07EE901A0A44BEF1010FCBF890E0A2
:10B8B800CBF86420F8EEE77A03F0C980DBED205A74
:10B8C800DBED226A07EE10EA37EEE56AB8EEC75AF2
:10B8D800012F86EE057A37EE257A77EEC77A8BED5B
:10B8E800217AE7EE866A8BED207AF0EE667ACBED68
:10B8F800236ACBED226A03F04984DBF8A430BBF954
:10B908003C10DBF8682003F1010E07EE901A0A4498
:10B91800BEF1010FCBF8A4E0CBF86820F8EEE77A87
:10B9280003F0B080DBED255ADBED276A07EE10EA5D
:10B9380037EEE56AB8EEC75A012F86EE057A37EE7C
:10B94800257A77EEC77A8BED267AE6EE276A8BEDB5
:10B95800257AF0EE667ACBED286ACBED276A03F0FC
:10B96800E083874CA8F80600BBF8A820029B013AA0
:10B978001E78ABF8A82005990022072E4A608A6035
:10B98800CA6040F05981F9F70DFF029BDFF8508239
:10B998001E78049BC01A94F82831A8F80000069372
:10B9A800002B40F04F81744A5279002A01F08881B7
:10B9B800744A1278013AD2B2072E84F8282102F08C
:10B9C800608200230793704BD4F83421D3F800A089
:10B9D800684B0593049B9FED6D6AD4ED4C9A6C49B6
:10B9E800C4F834319A1A07EE902AF8EE677AB7EE5F
:10B9F800007AC6EE278A0025664BDFF8E891DFF863
:10BA0800E881654F03932E46D1ED006A94ED4BDA39
:10BA18009FED629ADFED62AA9FED62CA9FED62AA6E
:10BA2800DFED62BA9FED62BA77EE69CA6CEEA6CA1C
:10BA3800F4EEC7CAF1EE10FA88BFF0EE47CA5D4BC4
:10BA480099ED008A2B44D3ED007AF5EE407AF1EEB9
:10BA580010FA17D0584B2B4493ED007A78EE476ACA
:10BA6800B0EEE66AF4EEC67AF1EE10FA08D5F5EE15
:10BA7800C06AF1EE10FACCBF37EE878A37EE678AD4
:10BA880083ED008A4D4B1A88910739D0022E37D0A2
:10BA98009AF82E104A4B07EE901A2B4493ED007A31
:10BAA8004B42F8EEE76A07EE903A26EE877AF8EE10
:10BAB800E77AB4EEE77AF1EE10FA0AD407EE901AB4
:10BAC800F8EE677AF4EEC77AF1EE10FA88BFF0EE76
:10BAD800477A3C4B3C4903EB460331F91600B3F96E
:10BAE8000C30C31A07EE103AB8EEC77AD307E7EE60
:10BAF800497A41F18180354B93ED008A27EE888A97
:10BB0800059B94F868212B4493ED01EA78EE4EDA10
:10BB1800002A00F0F7802E4BD4F86C2104991B689A
:10BB28008A1A9A4240F3EE809AF84830022B02F0C3
:10BB3800F781022E04F08584264B1B68980700F1D4
:10BB48009780254B87ED00CA1B689342C0F2CA80D4
:10BB5800F7EE007AF4EEE79AF1EE10FA40F1D280AF
:10BB680005991E4BD1ED017A93ED007AF0EEE77A54
:10BB78003CE000BF0C5700208054002060450020A6
:10BB88000020002090410020AC4700200024744988
:10BB98000C510020503B00205C3B0020CDCCCC3D1C
:10BBA800AE47813F000000000000C8420000344357
:10BBB800610BB63B0051002044210020A84700201B
:10BBC800502100209C41002058470020E8500020C8
:10BBD800145100204C470020105100201C51002017
:10BBE8006445002038210020683B0020F4EEC77A25
:10BBF800F1EE10FA40F18680D1ED027AF0EEE77AA4
:10BC0800B4EEE77AF1EE10FA7CDDD1ED037AF0EECE
:10BC1800E77AB4EEE77AF1EE10FA73DD0F4B1B68A2
:10BC280099075FD50E490F4B43E00F4B0F4C1E7819
:10BC38000293072E3FF4A7AE94F828310693002B01
:10BC48003FF4B1AE013B84F82831012E01F0B782F0
:10BC580013B0BDEC0E8BBDE8F08F00BF4C47002041
:10BC6800584700209C41002060450020002000200B
:10BC7800D34BD449DFF8C8E331F916C09EED008AEA
:10BC8800DFF8C0E387ED00CA03EB460028EE098A17
:10BC9800B0F90C00A0EB0C0007EE900AF8EEE77A7A
:10BCA800DEF8000027EE888A904278EE4EDABFF67A
:10BCB8004FAFB3F90C20B1F900E0C348AEEB020E68
:10BCC80000688EEAEE72A2EBEE7282421ADAB3F9DB
:10BCD8000E30B1F90220D21A82EAE273A3EBE273C2
:10BCE80098420FDDB94B1A88002384F86831002A7E
:10BCF80043F0E485B64AB74B1178186881F0010122
:10BD0800FAF708FCB44B2B4493ED000A039B2DEE85
:10BD1800000A022E20EE2D0AA3EC010A039304F078
:10BD2800B883AE4BD7ED006A93ED007AAC4BD3EDF8
:10BD3800007AAC4B93ED006AAB4B67EE277A2B4445
:10BD480027EEAC7AD3ED007A67EE277AF0EE665AE2
:10BD5800EDEEA75AB1EE467AB4EEE57AF1EE10FAB6
:10BD680008DCB4EEE56AF1EE10FA8CBFB0EE657A45
:10BD7800B0EE467A94ED4C6AF7EE007AB4EEE76AD4
:10BD8800F1EE10FAACBF0123002343B1F0EEE66AEE
:10BD9800F0EEC77AF4EEE67AF1EE10FA01D587ED07
:10BDA800007A022E04F04683904A914B52F82600FE
:10BDB8001B68B0EE4E0A98478E4A8F4B52F8260001
:10BDC8001B6898479AF8373023B18C4B1B88002B97
:10BDD80000F07987B0EE4C8A894B38EE400A2B4444
:10BDE80093ED008A83ED000A9AF8483030EE480A4D
:10BDF80020EE288A002B33D0824B1B7813F00103E6
:10BE080000F0C686F7EE007AF4EEE79AF1EE10FA43
:10BE180094F86831C1F27485002B00F0F987D4F8E2
:10BE28006C31049AD31A784A12689A4218DD774B13
:10BE3800D3ED007AF0EEEDDAF4EEE7DAF1EE10FA8F
:10BE480042F17F80614B1A88002384F86831002A08
:10BE580000F0AA866E494A6912B10A6813604B74E9
:10BE68006C4B94F878212B4493ED000A2DEE000AD0
:10BE780020EE088A88ED008A32B9039B87ED00CA54
:10BE880003ED01CA88ED00CA0136032E09F1040941
:10BE980008F1040807F1040705F104057FF4CFADA4
:10BEA800029B1A78072A01F04185012A01F0D687FA
:10BEB8000023039394F88021002A41F08D81DFF854
:10BEC80088A1554BDAF800201968D20491F82C00A3
:10BED80000F11487DFF87491504AB9F81A3092EDDE
:10BEE800006A4F4A4F4ED2ED005AD6ED036A4E4AC9
:10BEF80084ED646A07EE103A4C4B92ED005AD3ED8C
:10BF0800007AD3ED013AD3ED024A84ED626AB8EEC5
:10BF1800C77A35EEC64A012236EEC77A84ED614A01
:10BF2800C4ED655A84F89821C7EE055A0A8D534224
:10BF380006EE103A3E4BDFED3F6A93ED005A3E4B5A
:10BF480093ED004AB7EE007AF4EEC75A35EE045A7C
:10BF5800F1EE10FA88BFF0EE475A35EE275AB8EEE0
:10BF6800C66AF4EEE65AF1EE10FA07EE902AB4EE3D
:10BF7800C65AB8BFF0EE665AF1EE10FAC4ED685A28
:10BF8800B8EE677A01F13A83B4EEC75AF1EE10FAC7
:10BF980088BFB0EE475A264BDFED286AD3ED017A09
:10BFA800254B93ED014A77EE847A25EE265A77EEF3
:10BFB800A37AB4EEE76AF1EE10FA52DC48E000BF6B
:10BFC8009C41002058470020185100206864002038
:10BFD8006A6400206C640020BC500020F84F0020E8
:10BFE8000400002030510020C850002000500020DC
:10BFF800FC4F00205450002050500020A84700203B
:10C00800702100201B5200201451002020510020D4
:10C0180070640020D4500020AC470020F43F00207A
:10C028007041002080450020C85100205C3B002062
:10C03800503B002000000000683B00206F12833A4C
:10C04800E8500020105100201C57002014600020E8
:10C05800B4EEE77AF1EE10FA8CBFB0EE676AB0EE94
:10C06800476AED4B4A8DD3ED027A9FEDEC7A534245
:10C0780004EE103A74EEA77AB8EEC44A26EE076AC0
:10C08800F4EEC47AF1EE10FA0AD407EE102AB8EEEC
:10C09800474AB4EEE74AF1EE10FA88BFB0EE674AB5
:10C0A800DF4ADFEDDE7A527824EE274A0AB9B1EE8C
:10C0B800444A002841F07686B7EE003AD94E3278E5
:10C0C800002A02F0A786D849DFEDD87AD1ED024AD6
:10C0D800D1ED016A91ED037A66EE244AE5EE264A2F
:10C0E800E4EE074A63EE244AF4EEE74AF1EE10FA6A
:10C0F800B4BFF0EE673AF0EE643A98BFF0EE647AB7
:10C10800012ACDED0A4A02F0D88691ED067AD1EDE2
:10C11800052AD1ED076A26EE077AA5EE227AA4EE63
:10C12800267A23EE077AB4EEE77AF1EE10FAB4EE47
:10C13800E37A8CBFF0EE676AF0EE476AF1EE10FA28
:10C1480088BFF0EE676AB4BFF0EE637AF0EE477A24
:10C15800022A8DED0B7A00F0DE8091ED0A7AD1ED9E
:10C16800092AD1ED0B3A26EE077AA5EE227AA4EE3B
:10C17800237A23EE077AB4EEE67AF1EE10FAB4EEFB
:10C18800E77A8CBFF0EE663AF0EE473AF1EE10FA35
:10C1980098BFF0EE636AA8BFF0EE477A032A8DEDE8
:10C1A8000C7A00F0B88091ED0E7AD1ED0D2AD1ED20
:10C1B8000F3A26EE077AA5EE227AA4EE237A23EE2A
:10C1C800077AB4EEE67AF1EE10FAB4EEE77A8CBFAD
:10C1D800F0EE663AF0EE473AF1EE10FA98BFF0EE5C
:10C1E800636AA8BFF0EE477A042A8DED0D7A00F055
:10C1F8009280D1ED123AD1ED112A91ED137A66EEC3
:10C20800233AE5EE223AE4EE073A63EE233AF4EEF7
:10C21800E63AF1EE10FAF4EEE73A8CBFB0EE667A41
:10C22800B0EE637AF1EE10FA98BFF0EE476AA8BF55
:10C23800F0EE637A052ACDED0E3A6CD0D1ED163AC0
:10C24800D1ED152A91ED177A66EE233AE5EE223AFA
:10C25800E4EE073A63EE233AF4EEE63AF1EE10FA2A
:10C26800F4EEE73A8CBFB0EE667AB0EE637AF1EEA0
:10C2780010FA98BFF0EE476AA8BFF0EE637A062A74
:10C28800CDED0F3A47D0D1ED1A3AD1ED192A91EDFB
:10C298001B7A66EE233AE5EE223AE4EE073A63EEBD
:10C2A800233AF4EEE63AF1EE10FAF4EEE73A8CBFF0
:10C2B800B0EE667AB0EE637AF1EE10FA98BFF0EE5F
:10C2C800476AA8BFF0EE637A072ACDED103A22D06C
:10C2D80091ED1E7AD1ED1D2AD1ED1F3A26EE077A8F
:10C2E800A5EE227AA3EE847A27EE037AB4EEE67AF4
:10C2F800F1EE10FAB4EEE77A8CBFB0EE666AB0EEF3
:10C30800476AF1EE10FA8DED117A98BFF0EE466AA1
:10C31800A8BFF0EE477A77EEE67AF7EE006AF4EE19
:10C32800E67AF1EE10FAC4ED4C7A43F3F08586EE26
:10C33800A77A022ADDED0B7A67EE244A67EE877A40
:10C34800CDED0A4ACDED0B7A2DD0DDED0C7A67EEF6
:10C35800877A032ACDED0C7A25D0DDED0D7A67EECC
:10C36800877A042ACDED0D7A1DD0DDED0E7A67EEC1
:10C37800877A052ACDED0E7A15D0DDED0F7A67EEB6
:10C38800877A062ACDED0F7A0DD0DDED107A67EEAB
:10C39800877A072ACDED107A05D0DDED117A27EEE0
:10C3A800877A8DED117A2249096811F0805801F0D9
:10C3B8005A82F6EE005AC4ED685A002A02F04D85FA
:10C3C8001C4B94ED656A1C491C4F1D78DFF874E01E
:10C3D80094F9983194ED645AB7F90670C878DAF888
:10C3E8000010DEED004A0597BDEEC66A07EE103A6A
:10C3F800B9F81A70124B079716EE10EABDEEC56A27
:10C4080005F0010C01F4805701F0100501F48001DA
:10C4180008911B7818E000BF503B00206F12833A48
:10C42800E83B00200E4500203851002000000000A5
:10C43800644100201B520020D44900208E8800202F
:10C448004059002034510020D4ED616AD4ED627A5D
:10C45800B8EEC77A16EE101A002840F03787002D7C
:10C4680041F06F83D54D9DED0A5A95ED006AD44889
:10C4780025EE866AA5EE076AB0EE675AA6EE265A3A
:10C48800BDEEC56A16EE108A16EE107AF045A8BF02
:10C4980077464145C8BF0F4606EE107AB8EEC66A21
:10C4A800012A80ED006A00F0DC8095ED046A9DEDBC
:10C4B8000B5A25EE866AA5EE076AB0EE675AA6EE15
:10C4C800265ABDEEC56A16EE108A16EE107AF045A9
:10C4D800A8BF77464145C8BF0F4606EE107AB8EEAA
:10C4E800C66A022A80ED016A00F0BB8095ED086AF1
:10C4F8009DED0C5A25EE866AA5EE076AB0EE675ADE
:10C50800A6EE265ABDEEC56A16EE108A16EE107A09
:10C51800F045A8BF77464145C8BF0F4606EE107ADA
:10C52800B8EEC66A032A80ED026A00F09A8095ED9B
:10C538000C6A9DED0D5A25EE866AA5EE076AB0EEE7
:10C54800675AA6EE265ABDEEC56A16EE108A16EE92
:10C55800107AF045A8BF77464145C8BF0F4606EE9A
:10C56800107AB8EEC66A042A80ED036A79D095ED90
:10C57800106A9DED0E5A25EE866AA5EE076AB0EEA2
:10C58800675AA6EE265ABDEEC56A16EE108A16EE52
:10C59800107AF045A8BF77464145C8BF0F4606EE5A
:10C5A800107AB8EEC66A052A80ED046A59D095ED6E
:10C5B800146A9DED0F5A25EE866AA5EE076AB0EE5D
:10C5C800675AA6EE265ABDEEC56A16EE108A16EE12
:10C5D800107AF045A8BF77464145C8BF0F4606EE1A
:10C5E800107AB8EEC66A062A80ED056A39D095ED4C
:10C5F800186A9DED105A25EE866AA5EE076AB0EE18
:10C60800675AA6EE265ABDEEC56A16EE108A16EED1
:10C61800107AF045A8BF77464145C8BF0F4606EED9
:10C62800107AB8EEC66A072A80ED066A19D095ED29
:10C638001C6A9DED115A65EE865AE7EE055AE6EE3C
:10C64800A57AFDEEE77A17EE905AAE45A8BFAE463A
:10C65800A942D8BF714607EE901AF8EEE77AC0ED06
:10C66800077ABCF1000F00F03E87564A1268002A8C
:10C6780040F04687544A127892B1307868B1504FEA
:10C68800DFF868810025E8B2D8F80030B7EC010A75
:10C698009847307801358542F5DB4C4A1268904757
:10C6A800029B1A78072A01F030810025DAF8002069
:10C6B800560500F1BF87464B1B68180700F1C8876D
:10C6C800444B1B78BBB1444AB9F81A30B2F906207A
:10C6D8009A4210DC414B1B78012B01F0E783192BA0
:10C6E80001F0E4830E2B06D0082B04D03C4E002327
:10C6F800B360C4F8403194F8AA6126B1394B1B885D
:10C708009F0741F0958394F8B021002A40F0FB87F9
:10C7180099F81E70002F00F03384022F01F0778300
:10C72800032F41F0708399F82030C3EB431103EBDA
:10C738008101C90089B299F81F300233DBB2002A9F
:10C7480000F08685002900F0838527480768B1FB3B
:10C75800F7F10FB2A4F8E071002B03F0BF8007EEE9
:10C76800907AF8EEE77AF7EE006A86EEA77A1C4E22
:10C77800012BD4ED7D6AD6ED007A77EEE67A67EE86
:10C78800877AC4ED797A3DD0D6ED017AD4ED7E6A08
:10C7980077EEE67A022B67EE877AC4ED7A7A31D0A3
:10C7A800D6ED027AD4ED7F6A77EEE67A032B67EE50
:10C7B800877AC4ED7B7A25D01AE000BF3851002073
:10C7C800B03B0020DC300020685C00203C59002091
:10C7D8004C4700204C1C00208E880020E83B00209D
:10C7E80080450020A8470020D03B00203459002075
:10C7F800D6ED037AD4ED806A77EEE67A67EE877A2B
:10C80800C4ED7C7A02990978092903F0A381002FE5
:10C8180040F3BC839BB394ED7D7AD4ED797A77EEBF
:10C82800877A012BC4ED7D7AC6ED007A21D094ED8C
:10C838007E7AD4ED7A7A77EE877A022BC4ED7E7A07
:10C84800C6ED017A15D094ED7F7AD4ED7B7A77EE38
:10C85800877A032BC4ED7F7AC6ED027A09D0D4ED2E
:10C86800807A94ED7C7A77EE877AC4ED807AC6ED8B
:10C87800037A013B022BB8BF0223DBB20693069B67
:10C88800002A18BF02239E46CC4BDFEDCD6A1A68FA
:10C89800029B91781878137807EE903AF8EEE77AC9
:10C8A800B0EE007A67EEA67AF4EEC77AF1EE10FAE7
:10C8B80040F38F86DFEDC36A37EEC77AB0EE676A5A
:10C8C800A7EE266AF0EE466A96ED007A9FEDBE6AFC
:10C8D80027EE066AF0EEC65A84ED546AC4ED575A3C
:10C8E80099B107EE101AB8EEC75A9FEDB57A66EE01
:10C8F800064A25EE075AB7EE007A37EE457A64EE17
:10C90800A54AA4EE857A26EE076A9FEDB07A537998
:10C9180026EE877A27EE067ACBB1DFEDA96A9FED7E
:10C92800AC6A65EEA65A06EE903AF8EEE66A66EE4E
:10C93800A56AF4EEC66AF1EE10FA01F31D82F7EE6D
:10C94800005A75EEE66A85EEA66A27EE067A0C2886
:10C958009FEDA08ADFEDA06A00F08C87B4EEC87A5C
:10C96800F1EE10FA98BFB0EE478AB4EEE68AF1EE1F
:10C9780010FAB8BFB0EE668A84ED4E8ABEF1000F99
:10C9880000F0DD80B0EE007AF4EEC77AF1EE10FA2E
:10C9980005DD37EEC77ADFED8B6AE7EE267A96ED8E
:10C9A800017ADFED896A27EE267AF0EEC75A84ED20
:10C9B800557AC4ED585A99B106EE901A9FED806ADF
:10C9C800F8EEE66A27EE075A66EE866AB7EE006A60
:10C9D80036EE666A25EE255AA5EE266A27EE067A11
:10C9E800DFED7A6A937967EEA67A67EE877AABB15C
:10C9F80007EE103AB8EEC77A9FED716ADFED746AF8
:10CA080027EE257A27EE067AB4EEE67AF1EE10FAEA
:10CA180041F3A481DFED716A67EEA67A0C2800F075
:10CA28004787DFED6C6A9FED6C7AF4EEE67AF1EEFB
:10CA380010FA88BFF0EE667AF4EEC77AF1EE10FAD3
:10CA4800B8BFF0EE477ABEF1010FC4ED4F7A76DD3C
:10CA58005378DFED5B6A07EE903AF8EEE77AB0EECE
:10CA6800007A67EEA67A537AF4EEC77AF1EE10FAF6
:10CA780005DD37EEC77ADFED536AE7EE267A96EDE5
:10CA8800027ADFED516A27EE267AF0EEC75A84ED76
:10CA9800567AC4ED595A9BB106EE903A9FED486A12
:10CAA800F8EEE66A27EE075A66EE866AB7EE006A7F
:10CAB80036EE666A25EE255AA5EE266A27EE067A30
:10CAC800DFED426AD37967EEA67A67EE877AFBB123
:10CAD80007EE103AB8EEC77A9FED396ADFED3C6A87
:10CAE80027EE257A27EE067AB4EEE67AF1EE10FA0A
:10CAF80001F33081B5EEC07AF1EE10FA02F17283DB
:10CB0800B7EE006A36EE477AC6EE076A67EEA67A8F
:10CB18000C2800F0ED86DFED2F6A9FED2F7AF4EEFA
:10CB2800E67AF1EE10FA88BFF0EE667AF4EEC77A8C
:10CB3800F1EE10FAB8BFF0EE477AC4ED507A092842
:10CB480000F0848699F82160002E40F03986002391
:10CB580084F8B03124F0D6F8002840F05383204BF5
:10CB68001B7823B91F4B9B78002B41F05C810498FC
:10CB780009F0E2FA029B1E78072E7FF466A8F8F700
:10CB880011FE194B029A401B1678D880FFF75DB842
:10CB980094F86821002A3FF463A9144A84F868319C
:10CBA8001288002A7FF456A9114A124B1178186886
:10CBB80081F00101F9F7AEFCFFF752B9B047002048
:10CBC8000AD7233CD7A368416F12033B00004843B0
:10CBD800A4707D3F00C0F94400C0F9C40000C842F9
:10CBE8002F420020725E0020644500206864002007
:10CBF8006A6400206C64002094ED577AB1F9000053
:10CC0800D4ED586AB1F902E0E24AF4EEC76A80EA64
:10CC1800E0738EEAEE71A3EBE073F1EE10FAA1EB8C
:10CC2800EE71B8BFF0EE476A8B42B8BF0B4607EE0D
:10CC3800103A1378B8EEC77A27EE097A002B40F03D
:10CC4800B880D54B93ED006AB4EEEA6AF1EE10FABB
:10CC580041F1E480F7EE005A75EEC65A3BEEC77A0A
:10CC680065EE8B5ACD4BA7EE256A93ED007A26EE3A
:10CC7800076AB5EEC06AF1EE10FA40F2F085CAEE26
:10CC8800065AB7EE007AB0EE476AA6EEE56AF0EE0D
:10CC9800466AF4EEC76AF1EE10FA88BFF0EE476A0A
:10CCA800F5EEC06AF1EE10FAB8BFF0EE4C6ABC4B74
:10CCB80093ED007A67EE877AA7EEA68AFEF720BF83
:10CCC8000122FEF779BEB74BB74A2B4493ED007AA1
:10CCD800D2ED007AB54B67EE277AF7EE006AF4EEEC
:10CCE800E67AF1EE10FA93ED007A88BFF0EE667AF4
:10CCF80067EE877A27EE888AFFF76EB8AC4BDFF8C5
:10CD0800EC921A78AB4ED3075CBFB9F81820A4F898
:10CD18008C21A94AD6ED037A128807EE102AB8EEBC
:10CD2800C77AF4EEC77AF1EE10FA42F24380A34DC7
:10CD38002B8807EE103AB8EEC77AF4EEC77AF1EE10
:10CD480010FAC1F2BF809E4A9E4D92ED006AD5ED61
:10CD5800006A94F99821C4ED646A76EE665A012A4D
:10CD6800C4ED626AC4ED615A84ED656A01F04186DA
:10CD7800049BC4F89C31002537EEC77AFCEEE77AAD
:10CD8800914E84ED687A17EE902AA4F88C2101223E
:10CD980096ED005A84F898218C4A954241F2F7871B
:10CDA8008B4BD3ED007AD3ED013AD3ED024AFFF76E
:10CDB800BBB87A4B93ED005AB5EEC05AF1EE10FAB3
:10CDC80040F34D85834BD3ED004AF5EEC04AF1EEB2
:10CDD80010FA40F3448534EEC77A66EECA5A87EEF5
:10CDE800246AC5EE856AB7EE007AB4EEC76AF1EE3A
:10CDF80010FA88BFB0EE476AB5EEC06AF1EE10FAD5
:10CE080076EE876AB8BFB0EE4C6A66EE266A40E7EF
:10CE1800714AD2ED007AB0EEC87AB4EEE77AF1EE54
:10CE280010FA7FF71DA86D4AD2ED007AB0EEED7AC0
:10CE3800B4EEE77AF1EE10FA7FF712A8684AD9ED56
:10CE4800007A92ED007AF0EEE77AF4EEC77AF1EE26
:10CE580010FA7FF505A801220499C4F86C1184F82A
:10CE68006821FEF7E0BF07EE102A1978DFF8808105
:10CE7800C4F80C71B8EEC77AF7EE006A132986EE8B
:10CE8800879AB8F90400B4F810619BED070A01F01D
:10CE98003C85544A544992ED001AD2ED053A92ED78
:10CEA800122A92ED173AD2ED091AD2ED0E4A92EDF6
:10CEB800016A92ED064A92ED0A7AD2ED0F5AD2ED46
:10CEC800132AD2ED186A92ED045AD2ED030A67EEDE
:10CED800897A69EE288A29EE088AE1EE273A01EB79
:10CEE80086070025A2EE283AC4F80051C4F8045178
:10CEF800E1EE884AA6EE274AE7EE085A92ED167A3E
:10CF080092ED0D6A92ED021AD2ED0C1AC7ED003AB5
:10CF1800E2EEA86A25EE635A27EE437A92ED0B2AD1
:10CF2800D2ED152AC7ED204AA0EEE34A26EE646A40
:10CF3800D2ED143A82ED054AA1EE275AF0EE477A6F
:10CF4800E1EEE45AA2EE086AE2EEC36AE3EEA87ADA
:10CF580082ED065AC2ED0E5A82ED0F6A87ED403A0D
:10CF6800C2ED176AC2ED187AC4F80851721C02F0B3
:10CF78001F02A4F81021A8F80400029BFEF71BBCAE
:10CF8800A4F8E071002A3FF4E5AD0A4E4FF0020E16
:10CF98007AE400BFF4500020FC500020F05000203C
:10CFA800EC5000205C210020E4500020E0500020DC
:10CFB8001B52002080450020CC510020CE5100207B
:10CFC80070410020B8510020D45100208FD00300B8
:10CFD8005C3B0020F8500020245100202051002004
:10CFE80028510020083A00209C37002014600020B7
:10CFF800644500209C4A1178D4F818719B4B9FED2A
:10D008009C7AFE009A1982ED007A002979D0994815
:10D01800B0EE476AF0EE476A0022F0EC017A01327E
:10D0280067EEA77A05EE902AB4EEE77AF1EE10FAE9
:10D03800F8EEE55AB8BFB0EE677A8A4276EEA76A8C
:10D04800A7EEA56AE9D1F5EEC06A9A19F1EE10FAD1
:10D0580082ED007A55DDC6EE265A874A8749098847
:10D06800F7EE007A75EEE75AD2ED007A65EEA77A08
:10D07800FDEEE77A17EE902A812A42F3C6808A42AB
:10D08800A8BF0A4607EE902AF8EEE77A7C4AF0191C
:10D0980002EB800292ED057AD2ED003A92ED066A33
:10D0A80092ED014AD2ED046AD2ED034A92ED025A9A
:10D0B800A3EEA77AA4EE276A66EEC76AA7EE646AAB
:10D0C800BDEEC77AE5EE276A17EE100A812882EDD1
:10D0D800056AC2ED066A42F395808142A8BF0146FF
:10D0E80007EE901AF8EEE77AFCEEE77ACDED057ACE
:10D0F800BDF8142099198A801FB9BEF1130F02F0E8
:10D108001487BEF1150F41F046811E44DFF8908167
:10D11800B28828F81720D4F814515A4A013582FBEE
:10D1280005325119EA17C2EBA102C2EBC202AD1ACD
:10D13800C4F814515448D4F81C11049B534D026888
:10D148002D78C4F81C31591A0A440260002D40F0A9
:10D15800DB8107EE901A4E4EDFF864914D4FB8EE22
:10D16800E78A06F5F07506F51378F6EC017A9BED7B
:10D17800070ADBF80832F8EEE77A284627EE800A35
:10D188009847A5F1E000DBF828319847A5F1700031
:10D19800DBF898319847D6F8EC00DBF8AC309847C4
:10D1A800D7ED007AA9EC010AE0EE087A2435A84503
:10D1B800E7EC017AD9D1029B1E78FEF73ABD364BCF
:10D1C800364A19681288364BC96919805A8013B0D3
:10D1D800BDEC0E8BBDE8F08F324B334E1A7812F04F
:10D1E800010F327840F0DC83002A00F0D5859200E8
:10D1F8002E492F48DFF8CCA0DFF8CC9028F020FB90
:10D20800FFF733BA2B4C23F039FC6378022B00F07C
:10D218003D86032B7FF4A3AC41F2B813E35C002BEB
:10D2280041F06E8341F2A403E35C002B41F0638379
:10D2380041F2E803E35C002B41F0588341F22C13E0
:10D24800E35C002B3FF48BAC1B4817F047FE86E4E9
:10D25800B4F8E071013F3FB2002FA4F8E0717FF706
:10D2680091AE164EFFF7D6BA7E370020743A0020EA
:10D278000000000000200020803700207C370020BC
:10D288009C39002093244992BC4F00207437002019
:10D29800C0540020C04F00208C4F002018320020BE
:10D2A800644500201B5200200E450020E830002075
:10D2B800B03B0020946A0020C07B002080450020FD
:10D2C800105700201C57002014600020002D00F08B
:10D2D8002787BCF1000F42F00B83CC4D002B42F0A6
:10D2E8009F8195ED006A9DED0A5AC94825EE866A28
:10D2F800FDEEE44AA5EE076AB0EE675AA6EE265A96
:10D3080014EE901ABDEEC56A16EE10CA16EE107A23
:10D31800F445A8BF77466145C8BF0F4606EE107AA8
:10D32800B8EEC66A012A80ED006A00F0DF8095ED4C
:10D33800046A9DED0B5A25EE866AA5EE076AB0EEE3
:10D34800675AA6EE265ABDEEC56A16EE10CA16EE44
:10D35800107AF445A8BF77468C45B8BF0F4606EE4D
:10D36800107AB8EEC66A022A80ED016A00F0BE8023
:10D3780095ED086A9DED0C5A25EE866AA5EE076ABA
:10D38800B0EE675AA6EE265ABDEEC56A16EE10CA6A
:10D3980016EE107AF445A8BF77468C45B8BF0F46FD
:10D3A80006EE107AB8EEC66A032A80ED026A00F02B
:10D3B8009D8095ED0C6A9DED0D5A25EE866AA5EEC9
:10D3C800076AB0EE675AA6EE265ABDEEC56A16EE93
:10D3D80010CA16EE107AF445A8BF77468C45B8BF38
:10D3E8000F4606EE107AB8EEC66A042A80ED036A84
:10D3F8007CD095ED106A9DED0E5A25EE866AA5EE55
:10D40800076AB0EE675AA6EE265ABDEEC56A16EE52
:10D4180010CA16EE107AF445A8BF77468C45B8BFF7
:10D428000F4606EE107AB8EEC66A052A80ED046A41
:10D438005CD095ED146A9DED0F5A25EE866AA5EE2F
:10D44800076AB0EE675AA6EE265ABDEEC56A16EE12
:10D4580010CA16EE107AF445A8BF77468C45B8BFB7
:10D468000F4606EE107AB8EEC66A062A80ED056AFF
:10D478003CD095ED186A9DED105A25EE866AA5EE0A
:10D48800076AB0EE675AA6EE265ABDEEC56A16EED2
:10D4980010CA16EE107AF445A8BF77468C45B8BF77
:10D4A8000F4606EE107AB8EEC66A072A80ED066ABD
:10D4B8001CD095ED1C6A9DED115A65EE865AE7EE73
:10D4C800055AE6EEA57AFDEEE77A17EE905AAE45D4
:10D4D800A8BFAE46A942D8BF714607EE901AF8EE2B
:10D4E800E77AC0ED077A002A3FF4BFA892004949BD
:10D4F800474828F0A5F9484A1268002A3FF4BAA814
:10D508000BF060F8FFF7B6B807EE901A434D444B9E
:10D51800DFF81881DFF818910394F8EEE78A05F52B
:10D52800B87600271C46CDF81880029BDBED077AF9
:10D538001B78172B56D095ED007AB8EEC78A082BC2
:10D5480028EE278A07D1B0EE480A059328F0B8FAE2
:10D55800059BA8F80000DAF8002090000BD5002FF2
:10D5680002F0F387B0EE480ADBF8083206F17000E3
:10D578009847B0EE408AB0EE480ADBF82831A6F1A9
:10D5880070009847DBF8983130469847029B1B7823
:10D59800032BB0EE408A20D0D5F8F000DBF8AC3091
:10D5A800B0EE480A9847D9ED007AA4EC010AE0EEFB
:10D5B800287A0137032F06F1240608F1020805F13D
:10D5C8000405E9EC017AB0D1029B039C1E78FEF7B2
:10D5D80030BBF0EE676AFFF777B928F071FAA8F860
:10D5E8000000D9E795ED007A0BEB4702B8EEC78A41
:10D5F800128FA8F8002028EE278AACE7B0EE465A2A
:10D60800FEF7C9BC074B0293074C93E5385100203D
:10D61800B03B0020E8300020DC300020C05400205F
:10D62800105700206045002000200020644500209D
:10D63800C04F0020DBF80830002B3FF43CA8C64957
:10D64800A1F14C009847C54B1B6818077FF538A80F
:10D65800C34ED6ED027AB2EE0E7AF0EEE76AF4EE39
:10D66800C76AF1EE10FA41D5BE4B1B8859073DD564
:10D67800BD4BBE49B3F90430B4F8A62181FB0301C0
:10D68800DB17C3EBA1039B1A9BB219B211F1B30FBD
:10D69800BCBF03F5B47319B2B329C4BFA1F5B47301
:10D6A80019B2B34BB34A1B791278002B4FF6FF73AC
:10D6B80018BF012312077FF503A8AF4A126811FBB0
:10D6C80003F3117EAD4A9BB211FB03F382FB0312F5
:10D6D8001A44DB17C3EB221307EE103AB8EEC77AE9
:10D6E80077EEC77AC6ED027AFEF7EABF9E4B9F4AED
:10D6F800B3F9043082FB0312DB17C3EBA203A4F8CF
:10D70800A631FEF7DDBF9E499E4BD1F8EC101B6891
:10D7180044F620608142A8BF0146B1F57A7FB8BFC0
:10D728004FF47A7189B213F0100FA4F8B211DAF835
:10D73800003000F0C283DB0441F15D858E4BD3F8E5
:10D7480000E0BEF832707F08854E8F48D4F8B431B7
:10D75800D6ED037AA0FB01018809642191FBF0F161
:10D768001429BDEEE77A04EB4306A8BF1421013360
:10D778009942C4F8B43117EE10CADCBF0023C4F8CC
:10D78800B43104EB4303A6F8B8C1B3F9B83107EED6
:10D79800103AB8EEC77A77EEC77AFDEEE77ACDEDA4
:10D7A800037ABDF90C1081EAE173A3EBE173BB4284
:10D7B80001F3F18675494FF07E530B60FEF7A8BF61
:10D7C8001E217048F4F7D8F800283FF4C0A9654B2B
:10D7D8001B885A063FF5BBA994F80432B34242F0BD
:10D7E800DB816A4BD4ED827AD3ED016A94ED505A0D
:10D7F800DFED675A9FED676A27EEC57A67EE887A8C
:10D80800A6EE887AE5EE267AB4EEE57AF1EE10FA1D
:10D8180088BFB0EE657AB4EEC67AF1EE10FAF4EE8F
:10D82800E57AB8BFB0EE467AF1EE10FA88BFF0EEAE
:10D83800657AF4EEC67AF1EE10FAB8BFF0EE467AE1
:10D8480084ED4E7AC4ED507AFFF781B9FDEEC87ABF
:10D85800514A17EE903A9780D380FFF773B9DFEDFE
:10D868004F6AFFF724BADAF800104F023EF5A1AD6F
:10D87800FEF7A3BDB4EEC87AF1EE10FA98BFB0EE89
:10D88800478ABDEEC77AB4EEE68ADFF80CC1F1EE3E
:10D8980010FA17EE103AB8BFB0EE668A84ED4E8AD9
:10D8A800ACF80030BEF1000F7FF46CA8FFF74AB95E
:10D8B8009FED377ADFED376A3749F4EEC77AF1EE34
:10D8C80010FA98BFB0EE677AFDEEE77AB4EEE67A22
:10D8D800F1EE10FA17EE903AB8BFB0EE667ABEF1E4
:10D8E800010F84ED4F7A4B803FF7B2A8FFF72AB9B2
:10D8F800BDEEE77A284B17EE102A9A80FFF70BB98E
:10D90800002B3EF4ADAAFEF78ABAF7F74BFF029B4D
:10D9180021491A78039B072AA0EB030088807EF42C
:10D92800C4AEF7F73FFF0546FEF7C0BEF7F73AFF6C
:10D93800029BDFF864801A78079B012AA0EB03009A
:10D94800A8F8020000F08C82072A7EF4B1AAF7F743
:10D9580029FF0390FEF7AEBAE05400204C470020A0
:10D9680080450020A8470020584700206766666663
:10D9780094410020F43B0020AC4700208988888827
:10D98800E002002064410020D34D62100400002012
:10D9980000C0F94400C0F9C464450020000000003C
:10D9A800002A00F0F981D4ED583A94ED574AD4EDA5
:10D9B800627AF34994ED617A91ED005AD4ED555AA3
:10D9C80094ED546AEF4DF048F4EEC43AF3EE046A6D
:10D9D800F1EE10FA77EEA64A00F1C28295ED026ADE
:10D9E80026EE656AB0EE674AA6EE074AB4EEE44A48
:10D9F80034EE666AF1EE10FA48BFB0EE456A012AC5
:10DA080080ED006A00F0C88195ED066A26EE656A29
:10DA1800B0EE674AA6EE074AB4EEE44A34EE666A08
:10DA2800F1EE10FA48BFB0EE456A022A80ED016AAD
:10DA380000F0B28195ED0A6A26EE656AB0EE674A93
:10DA4800A6EE074AB4EEE44A34EE666AF1EE10FA3E
:10DA580048BFB0EE456A032A80ED026A00F09C8157
:10DA680095ED0E6A26EE656AB0EE674AA6EE074A9D
:10DA7800B4EEE44A34EE666AF1EE10FA48BFB0EE4E
:10DA8800456A042A80ED036A00F0868195ED126AE2
:10DA980026EE656AB0EE674AA6EE074AB4EEE44A97
:10DAA80034EE666AF1EE10FA48BFB0EE456A052A10
:10DAB80080ED046A00F0708195ED166A26EE656ABD
:10DAC800B0EE674AA6EE074AB4EEE44A74EE666A18
:10DAD800F1EE10FA48BFF0EE456A062AC0ED056A75
:10DAE80000F05A81D5ED1A6A66EEE56AB0EE674A2B
:10DAF800A6EE874AB3EE046AB4EEE44A74EE466AC8
:10DB0800F1EE10FA48BFF0EE456A072AC0ED066A42
:10DB180000F04281D5ED1E6ADFF874A2DFF8749236
:10DB280066EEE55AE5EE877AF4EEE47A77EEC67AA1
:10DB3800F1EE10FA48BFF0EE457AC0ED077AFEF72D
:10DB480094BD904D9DED0A5A95ED006ABCF1000F09
:10DB580041F0E48125EE866A8B48A5EE076AB0EEAF
:10DB6800675AA6EE265ABDEEC56A16EE10CA16EE1C
:10DB7800107AF445A8BF77466145C8BF0F4606EE40
:10DB8800107AB8EEC66A012A80ED006A3FF4AEAC9E
:10DB980095ED046A9DED0B5A25EE866AA5EE076A97
:10DBA800B0EE675AA6EE265ABDEEC56A16EE10CA42
:10DBB80016EE107AF445A8BF77466145C8BF0F46F0
:10DBC80006EE107AB8EEC66A022A80ED016A3FF4C2
:10DBD8008DAC95ED086A9DED0C5A25EE866AA5EE8A
:10DBE800076AB0EE675AA6EE265ABDEEC56A16EE6B
:10DBF80010CA16EE107AF445A8BF77466145C8BF2B
:10DC08000F4606EE107AB8EEC66A032A80ED026A5D
:10DC18003FF46CAC95ED0C6A9DED0D5A25EE866AC5
:10DC2800A5EE076AB0EE675AA6EE265ABDEEC56A9B
:10DC380016EE10CA16EE107AF445A8BF774661456D
:10DC4800C8BF0F4606EE107AB8EEC66A042A80ED01
:10DC5800036A3FF44BAC95ED106A9DED0E5A25EE24
:10DC6800866AA5EE076AB0EE675AA6EE265ABDEE9A
:10DC7800C56A16EE10CA16EE107AF445A8BF7746A4
:10DC88006145C8BF0F4606EE107AB8EEC66A052A87
:10DC980080ED046A3FF42AAC95ED146A9DED0F5AA5
:10DCA80025EE866AA5EE076AB0EE675AA6EE265AF2
:10DCB800BDEEC56A16EE10CA16EE107AF445A8BF76
:10DCC80077466145C8BF0F4606EE107AB8EEC66AB9
:10DCD800062A80ED056A3FF409AC95ED186A9DEDBA
:10DCE800105A25EE866AA5EE076AB0EE675AA6EEC8
:10DCF800265ABDEEC56A16EE10CA16EE107AF4451D
:10DD0800A8BF77466145C8BF0F4606EE107AB8EE41
:10DD1800C66A072A80ED066A3FF4E8AB95ED1C6AEF
:10DD28009DED115A65EE865AE7EE055AE6EEA57A9C
:10DD3800FDEEE77A17EE905AAE45A8BFAE46A94267
:10DD4800C8BF8E4607EE90EAF8EEE77AC0ED077A8C
:10DD5800FFF7C9BBDFED0D6AFEF7D8BEB5EEC07A96
:10DD6800F1EE10FA01F13A82B7EE006A36EE477A20
:10DD7800C6EE076AFEF750BE9FED046AFEF7E5BDE2
:10DD88003451002038510020B03B00200000C84228
:10DD98001C57002014600020DFF878A3DFF8789380
:10DDA800FEF763BCC8494A79002A3EF485A9C74AE8
:10DDB8001278002A3EF480A90B78C549DFEDC54AE0
:10DDC80007EE903A0B88B8EE677A07EE902A06EECF
:10DDD800903AF8EEE77AF8EE666A67EE277AB7EED9
:10DDE800007A87EEA63AB4EEE43AF1EE10FA88BF6C
:10DDF800B0EE643AB4EEC73AF1EE10FAB8BFB0EE3E
:10DE0800473AFEF75BB9B44B5988FEF794BCB4F8AF
:10DE1800B21101F57A7189B2FEF78DBCAF4B93ED63
:10DE2800006AFEF726BF049813F064F8FEF79FBE59
:10DE3800AB4B9FEDAC7AD3ED087AF4EEC77AF1EEEE
:10DE480010FA00F2F7849FEDA87AA84ED6ED037A6F
:10DE580077EE877AC6ED037AFEF755BCDFF8BC8209
:10DE6800F7F7A0FCA249D4F87C2109680390821A2C
:10DE7800511AC4F87C01A8F80420A8F80610FEF787
:10DE880019B8F7F78FFC0790FDF79DBDA3784FF001
:10DE9800010A072B3EF663AEDFE813F05606560775
:10DEA8003F074B076E06280732075206914B9B7BAC
:10DEB800002B3EF41BACFEF71EBCD8003FF53BAC74
:10DEC800FEF726BCB4F88C51954240F2FE8494F8D3
:10DED800A451002D40F0C787874A884E92ED007AFA
:10DEE800D6ED007A94F99821C4ED647A77EE676AE2
:10DEF800012AC4ED627AC4ED616A84ED657A02F0A4
:10DF08000E80049BC4F89C317D4A9FED777A92ED90
:10DF1800005A84ED687A012284F89821FEF73CBF04
:10DF2800784B1B88002B40F0F385774A774B1178A4
:10DF38001868F8F7EFFAD4F86C21049B9A1AFDF7E1
:10DF4800F8BD734BD9ED007A93ED007AF0EEE77ADD
:10DF5800F4EEC77AF1EE10FA7DF782AFFDF772BFE3
:10DF6800D5ED015A65EEC65AB0EE674AA5EE874A66
:10DF7800B4EEE44A74EE665AF1EE10FA48BFF0EED9
:10DF8800455A012AC0ED005A3FF406AFD5ED055AAF
:10DF980065EEC65AB0EE674AA5EE874AB4EEE44A83
:10DFA80074EE665AF1EE10FA48BFF0EE455A022AAE
:10DFB800C0ED015A3FF4F0AED5ED095A65EEC65AE8
:10DFC800B0EE674AA5EE874AB4EEE44A74EE665AA4
:10DFD800F1EE10FA48BFF0EE455A032AC0ED025A96
:10DFE8003FF4DAAED5ED0D5A65EEC65AB0EE674A83
:10DFF800A5EE874AB4EEE44A74EE665AF1EE10FADA
:10E0080048BFF0EE455A042AC0ED035A3FF4C4AEA7
:10E01800D5ED115A65EEC65AB0EE674AA5EE874AA5
:10E02800B4EEE44A74EE665AF1EE10FA48BFF0EE28
:10E03800455A052AC0ED045A3FF4AEAED5ED155A3F
:10E0480065EEC65AB0EE674AA5EE874AB4EEE44AD2
:10E0580074EE666AF1EE10FA48BFF0EE456A062AD9
:10E06800C0ED056A3FF498AED5ED196A66EEC66A4A
:10E07800B0EE674AA6EE874AF3EE045AB4EEE44AD5
:10E0880074EE656AF1EE10FA48BFF0EE456A072AA9
:10E09800C0ED066A3FF480AED5ED1D6ADFF874A0C6
:10E0A800DFF8749026EEC66AE6EE077AF4EEE47AB4
:10E0B80077EEE57AF1EE10FAB8BFF0EE457AC0EDEA
:10E0C800077AFEF7D2BA00BF3C4700207E45002001
:10E0D80084440020713DAA3FE0420020F050002017
:10E0E800944F00208FC2753C00000000804500203E
:10E0F800D03B00208052002070410020B851002001
:10E10800D4510020686400206A6400206C640020F8
:10E11800285100201C57002014600020644500206E
:10E12800D94D002B41F09E8095ED006A9DED0A5A6D
:10E13800D64825EE866AFDEEE44AA5EE076AB0EEFB
:10E14800675AA6EE265A14EE901ABDEEC56A16EE68
:10E15800108A16EE107AF045A8BF77464145C8BF29
:10E168000F4606EE107AB8EEC66A012A80ED006AFC
:10E178003EF477AA95ED046A9DED0B5A25EE866A62
:10E18800A5EE076AB0EE675AA6EE265ABDEEC56A36
:10E1980016EE108A16EE107AF045A8BF7746884525
:10E1A800B8BF0F4606EE107AB8EEC66A022A80EDAE
:10E1B800016A3EF456AA95ED086A9DED0C5A25EEC3
:10E1C800866AA5EE076AB0EE675AA6EE265ABDEE35
:10E1D800C56A16EE108A16EE107AF045A8BF774683
:10E1E8008845B8BF0F4606EE107AB8EEC66A032A0D
:10E1F80080ED026A3EF435AA95ED0C6A9DED0D5A44
:10E2080025EE866AA5EE076AB0EE675AA6EE265A8C
:10E21800BDEEC56A16EE108A16EE107AF045A8BF54
:10E2280077468845B8BF0F4606EE107AB8EEC66A3C
:10E23800042A80ED036A3EF414AA95ED106A9DED58
:10E248000E5A25EE866AA5EE076AB0EE675AA6EE64
:10E25800265ABDEEC56A16EE108A16EE107AF045FB
:10E26800A8BF77468845B8BF0F4606EE107AB8EEC5
:10E27800C66A052A80ED046A3EF4F3A995ED146A8E
:10E288009DED0F5A25EE866AA5EE076AB0EE675A2D
:10E29800A6EE265ABDEEC56A16EE108A16EE107A5C
:10E2A800F045A8BF77468845B8BF0F4606EE107AF6
:10E2B800B8EEC66A062A80ED056A3EF4D2A995ED45
:10E2C800186A9DED105A25EE866AA5EE076AB0EE2B
:10E2D800675AA6EE265ABDEEC56A16EE108A16EEE5
:10E2E800107AF045A8BF77468845B8BF0F46FEF7B5
:10E2F80096B9674ED4ED017A94ED006A3188726957
:10E3080077EEA77AF0EE006AB0EE677AA6EE267A84
:10E318004E1E04EBC601D6EE267A08391032F6EE08
:10E32800003A27EE237A67EEA37A84ED207AC4EDCB
:10E33800217A584C274604F1800091ED027A91ED3C
:10E34800036AD7ED036AD7ED027A52ED014A12ED5E
:10E35800025A37EE674A76EEC65A77EE277AE4EE27
:10E36800845A013EA1F10801E5EE047A07F1080795
:10E3780002F1080236EE267A00F10800E4EE877A08
:10E38800E5EE475A67EEA37A25EEA37AC0ED007A48
:10E3980080ED017AD1D1BEF1140F7EF4BEAEF7F74D
:10E3A80001FA039BDFF80081C01AA8F80200D4F82C
:10E3B8001451FEF7B2BED4F81831B4F810C1364A79
:10E3C800CCF120095FFA89F90CEB431702EB8707B8
:10E3D8005FEA990201F0BA85013216012F483049E7
:10E3E80007EB060807F1100212ED024A12ED035A74
:10E3F80012ED016A12ED047A50ED024A50ED035A0B
:10E4080050ED016A50ED047A64EE244A65EE255A0F
:10E4180066EE266A67EE277A1032904541ED024A89
:10E4280041ED035A41ED016A41ED047A00F1100013
:10E4380001F11001D8D11B48A6F110010F4400EBDF
:10E448000108214419F0030209D0B7EC017AF8EC6D
:10E45800017A67EE277A013AE1EC017AF5D1BCF14D
:10E46800000F41F04280BEF1140F7EF456AEF7F76C
:10E4780099F9039BDFF83080D4F81451C01AA8F832
:10E488000200FEF74ABE00BF38510020B03B002012
:10E4980084370020002000209C3700202C390020E1
:10E4A800102000201C39002064450020DFF860930C
:10E4B80099F800108F0801F0D686CD4E07F10108B3
:10E4C8004FEA481806EB080C06F12002A6F1700086
:10E4D80012ED076A52ED056A12ED037A52ED017AE0
:10E4E80052ED025A12ED084A52ED064A12ED045A4C
:10E4F80026EE066A66EEA66A27EE077A67EEA77A20
:10E50800A4EE046A20329445E4EEA46A00F11000F7
:10E51800A5EE057AE5EEA57AF1EEC65AB1EEE66A01
:10E52800F1EEC76AB1EEE77A40ED085A00ED076AE6
:10E5380040ED066A00ED057ACAD1A8F120023244FE
:10E5480004EB071711F0030018BF08320FD052ED83
:10E55800017A12ED027A67EEA77A0138E7EE077AB8
:10E5680002F10802B1EEE77AA7EC017AEFD1BEF129
:10E57800140F01F03F850135C4F81451FEF73CBD76
:10E58800D4F818519B499C489C4BEA001144154407
:10E598008A88196800EE102A643AC82AA8BFC822D7
:10E5A800782AB8BF782207EE902AB8EEC07AF8EE3B
:10E5B800E77A00EB850577EE670A77EE876A67EEFC
:10E5C800877A20EEA67AB8EE400AC7EE870A284670
:10E5D800D5F81490D5F81880EF692E6A1FF058FE08
:10E5E800029BC5F8149093F800E0C5F81880BEF1B6
:10E5F800140FEF612E6201F01085D4F81821804BBA
:10E60800D4F81451013283FB0213A3EBE27303EB3A
:10E618004303D31A0135C4F81831C4F81451CCE6B1
:10E62800784E7948B268B18926F004F9029B93F8CC
:10E6380000E0BEF1140F01F0FD84D4F81451013547
:10E64800C4F8145156E66F4E318873684FEA510981
:10E658004FEA89005FEAD10C04EB000204EB810564
:10E6680000F0A18000F110010CF1010C674F02EBE2
:10E678000C1C2944103203F1100E05F1100050ED66
:10E68800032A50ED043A17ED043A17ED032A50ED2A
:10E69800026A10ED016A17ED021A57ED010A11ED31
:10E6A800044A11ED035A52ED044A52ED035A12ED91
:10E6B800027A52ED017A51ED021A11ED010A73EE58
:10E6C800238A32EE228A47ED048A07ED038A71EE27
:10E6D800268A30EE868A47ED028A07ED018A74EEB3
:10E6E800848A35EE858A42ED048A02ED038A77EE44
:10E6F800218A37EE808A42ED028A02ED018A73EEA2
:10E70800633A75EE655A1EED035A32EE623A74EEBC
:10E71800644A25EE638A1EED044A23EE052A64EE58
:10E72800652AA3EE048A1032944524EE843AA3EEB7
:10E73800842A07F110070EF1100EA5EE853A00F1B4
:10E74800100001F11001E4EE852A00ED078A00EDC2
:10E75800082A01ED073A41ED082A5EED055A1EED3B
:10E76800065A71EE666A30EEC66A31EEC77A70EE06
:10E77800677A26EE253A65EEE63A25EE674A67EEB1
:10E78800054AE6EE053AA6EE853AA7EE254AE7EEF3
:10E79800A54A00ED063A40ED053A01ED064A41ED7D
:10E7A800054A7FF46CAF1FFA89F91A46494616489C
:10E7B8001FF010FA7268494628461FF00BFA029BB0
:10E7C8001A78142A7FF4F3ADE9E5F6F7EBFF029B1C
:10E7D800039093F800E0BEF1140F05BFDFF8348012
:10E7E800D4F81451D4F81451A8F80050FCF7EDBF30
:10E7F80080200020743A0020A05600200C570020EA
:10E808005655555584370020002000201020002040
:10E818007E37002064450020306E99BC2716983D4D
:10E82800A40DC93F843459BEDB0F4940D06D393A35
:10E8380000000000F0EEE76AB7EE005A35EE665ABF
:10E848001FED0B4A5FED0B5A1FED0A6A1FED0C7A9C
:10E8580094ED6B0AF1EEC54AE6EE845AF5EEC07AFD
:10E86800A6EEA56AF1EE10FAA6EE867A48BF5FED2D
:10E87800127A27EE247A48BF37EEC77A27EE000AC5
:10E8880027F01EF9B0F5617F00F3A08607EE900A25
:10E89800F8EEE76A5FED1B7A66EEA76A07EE906A04
:10E8A800BDEEE67AF8EEE77A17EE103A2033402B01
:10E8B80041F287841FED220A27F002F900B207EE21
:10E8C800900AB8EEE77AFFF7C0BAC84A02F15005D5
:10E8D80003E00432954200F0C6821378262BF8D163
:10E8E8009678D3789E42F4D2FFF7F1BAC04816F072
:10E8F800F5FAFEF7A3BCBF4816F0F0FAFEF798BC8D
:10E90800BD4816F0EBFAFEF78DBCBC4DBC4F95ED3B
:10E91800004A95ED057AD5ED014A95ED066AD5EDE3
:10E92800046A95ED035AD5ED025A67EE897A07EB2A
:10E938008602A4EE277AA4EEA76A66EEC76AA5EE59
:10E94800476AE5EEA76A20EE070A85ED056AC5ED78
:10E95800066A82ED007A29EE088A27F0B1F869EE96
:10E96800288AD5ED0E5AD5ED176A95ED091AD5ED19
:10E97800121A95ED0F5A95ED187A95ED0A2AD5EDEC
:10E98800132A95ED0D6AD5ED167A95ED0C3AD5ED6D
:10E998000B3A95ED154AD5ED144AE1EE085A0022D6
:10E9A80007EB8601E8EEA16A00B2C4F80021A2EEE6
:10E9B800085AC4F80421C4F80821A8EEA27A26EE61
:10E9C800656A67EEE67AA3EE655AA3EE886AA6EE54
:10E9D800C47AE8EEA47A85ED0E5AC1ED205A85ED89
:10E9E8000F6AC1ED406A85ED177AC5ED187AFEF712
:10E9F800BDBAD4F89C51049B5D1BFEF7BDB9BBF9A9
:10EA08003820CBF8201007EE902A0121F8EEE77A9B
:10EA1800CBF86020CBF87C100022012FCBED1C7ABC
:10EA2800CBED1B7ACBF8742001F06982AF427CF4FD
:10EA380030AFBBF93A20CBF8642007EE902A0021CA
:10EA48000122F8EEE77ACBF82410CBF890200022C8
:10EA5800012FCBED217ACBED207ACBF8882001F07D
:10EA68005282AF427CF449AFBBF93C20CBF8682016
:10EA780007EE902A00210122F8EEE77ACBF8281059
:10EA8800CBF8A4200022012FCBED267ACBED257AF6
:10EA9800CBF89C207CF465AF9FED5A8A032E49D0B1
:10EAA8004CB107EE904AF8EEE77AF4EEC87AF1EE48
:10EAB80010FA01F1DD83544A544C1168DBF86820E0
:10EAC800A8F8060094F8200102EB550292FBF5F530
:10EAD8000022CBF828508A620A63CA6228B14C4ADD
:10EAE800126832F480637CF43FAF4A4A126812F429
:10EAF800003241F0FC8148481146835C012B02F149
:10EB08000C0200F0908301311829F6D1FCF72CBFD4
:10EB180042494B69002B3DF40CA84148414B008801
:10EB280093FBF0F00B684FF0010E186081F811E0CC
:10EB3800FCF7FFBFB0EE480A26F0C2FF00B2AFE70D
:10EB480003236370FEF70BB800230AAE314618465C
:10EB5800092221F06FFD01287EF401A80A9B93F891
:10EB6800FE21552A01F0F78141F2B4120221012356
:10EB7800A1546370FDF7F3BF2278237D2A4FDFF895
:10EB8800B490032A14BF4FF480784FF08008002B0C
:10EB980067D0012BFBD1254B6268196838680023C0
:10EBA8004FEA412E4FF0FF31B1FBFEF112EB010BA2
:10EBB80043F1000C0021614500F1020008BF5845EF
:10EBC80038BF83465A461A49022021F073FE0328AB
:10EBD80001F2B98101A353F820F000BF67CB000808
:10EBE80041EC000867CB000841EC0008D83400204D
:10EBF8007C7B0020387B00204C7C0020083A0020D9
:10EC08009C370020000000008C4F002000200020CE
:10EC1800A4470020443E0020A48303087064002019
:10EC28008864002020A107009C7C0020A47C002090
:10EC38009C6A0020986A00206268A3682669991A6D
:10EC4800B14284BFE260216103281FD00133B3FBC6
:10EC5800F8F208FB12320AB143449B1A002263609F
:10EC680022753A6849460232002021F023FE032823
:10EC780001F2698101A353F820F000BF67CB0008B7
:10EC88008BED000867CB000895EC00082369062285
:10EC9800652BA27034D92278032A14BF6FF0FF02C3
:10ECA8006FF07F02A3F1650303EA020303F1010396
:10ECB80014BF4FF4807280229A42236120D23A68AE
:10ECC800E768023203EB0708904581F0A183844A84
:10ECD8006760D16FC4F80880490203FB01F305217E
:10ECE800176042F81C3C42F8183CA170A2687D49A4
:10ECF800012024F00DFF012841F01B830623A37097
:10ED08000021794824F024FB012841F01283A378DC
:10ED18000133DBB2A370FFF7BCB8744B0093032038
:10ED2800A0703023052272496F4825F0C5F8FDF719
:10ED380016BF41F27013E35C002B3DF410AF6A4834
:10ED480016F0CCF8FDF70BBF0AAE41F2FC173146BE
:10ED5800E0590023092221F06DFC01287DF4FFAE63
:10ED680000230A9A2370B2F80B30B3F5007F01F044
:10ED7800EA8241F2B41203210123A1546370FDF722
:10ED8800EEBE636884F814A00133A36003E7DFEDE7
:10ED9800597A594B94ED687AC3ED007AC3ED017A3C
:10EDA800C3ED027A554BF0EE674AF0EE673A196800
:10EDB800FDF7BAB8524A534DD2ED006A524A95ED62
:10EDC800006A1278C4ED646A84ED656A002A00F06E
:10EDD8000D8276EE665A94F99821C4ED615A013293
:10EDE800C4ED626A00F07485049BC4F89C31002568
:10EDF80037EE677AFCEEE77A444E84ED687A17EED0
:10EE0800902AA4F88C21FF2296ED005A84F89821C4
:10EE1800FDF7C2BF3E49DFED3F7A0968C4ED4C7A81
:10EE280011F0805840F0C683DAF8001011F4800819
:10EE380000F0EF814FF00008B6EE007A67EE877AAF
:10EE4800F4EEE57AF1EE10FAC8BFF0EE675A40F337
:10EE5800B183C4ED685AFDF7B0BA2F4B1D7805F0A1
:10EE6800010CFDF7FEBB264A264DD2ED007A264A54
:10EE780095ED007A1278C4ED647A84ED657A002AFB
:10EE880000F02E8377EE676A94F99821C4ED616AE1
:10EE98000132C4ED627A00F05786049BC4F89C31B5
:10EEA80000259FED147A194E84ED687AFF2296EDBD
:10EEB800005A84F89821FDF76FBF73EEE77AB7EE32
:10EEC800007AF4EEC77AF1EE10FAC4ED4C7A41F309
:10EED8001E8084EEA77A8DED0A7AFDF764BA00BF2A
:10EEE800287C0020986A0020047C0020B1300308A8
:10EEF800F0960308000000005C3B0020AC470020AF
:10EF0800F43F0020BC51002040590020D05100207F
:10EF180064410020000000801B520020002F00F0F8
:10EF2800CD8625EE866ACC48A5EE076AB0EE675A0C
:10EF3800A6EE265ABDEEC56A16EE10CA16EE107A6F
:10EF4800F445A8BF77466145C8BF0F4606EE107A5C
:10EF5800B8EEC66A012A80ED006A3DF486AB95EDED
:10EF6800046A9DED0B5A25EE866AA5EE076AB0EE97
:10EF7800675AA6EE265ABDEEC56A16EE10CA16EEF8
:10EF8800107AF445A8BF77466145C8BF0F4606EE1C
:10EF9800107AB8EEC66A022A80ED016A3DF465ABC4
:10EFA80095ED086A9DED0C5A25EE866AA5EE076A6E
:10EFB800B0EE675AA6EE265ABDEEC56A16EE10CA1E
:10EFC80016EE107AF445A8BF77466145C8BF0F46CC
:10EFD80006EE107AB8EEC66A032A80ED026A3DF49E
:10EFE80044AB95ED0C6A9DED0D5A25EE866AA5EEAB
:10EFF800076AB0EE675AA6EE265ABDEEC56A16EE47
:10F0080010CA16EE107AF445A8BF77466145C8BF06
:10F018000F4606EE107AB8EEC66A042A80ED036A37
:10F028003DF423AB95ED106A9DED0E5A25EE866AE8
:10F03800A5EE076AB0EE675AA6EE265ABDEEC56A77
:10F0480016EE10CA16EE107AF445A8BF7746614549
:10F05800C8BF0F4606EE107AB8EEC66A052A80EDDC
:10F06800046A3DF402AB95ED146A9DED0F5A25EE46
:10F07800866AA5EE076AB0EE675AA6EE265ABDEE76
:10F08800C56A16EE10CA16EE107AF445A8BF774680
:10F098006145C8BF0F4606EE107AB8EEC66A062A62
:10F0A80080ED056A3DF4E1AA95ED186A9DED105AC8
:10F0B80025EE866AA5EE076AB0EE675AA6EE265ACE
:10F0C800BDEEC56A16EE10CA16EE107AF445A8BF52
:10F0D80077466145C8BF0F4606EE107AB8EEC66A95
:10F0E800072A80ED066A3DF4C0AA95ED1C6A9DEDDD
:10F0F800115A65EE865AE5EE075AE6EEA57AFDEE58
:10F10800E77A17EE902A9645A8BF96469142D8BF4F
:10F11800714607EE901AF8EEE77AC0ED077AFDF728
:10F12800A4BABEF1010F7FF7B7AC07EE103AB8EEFC
:10F13800C77AC7EE876AB1EEE68AAFE4BEF1010F7F
:10F1480040F3DD8607EE103AB8EEC77AC7EE876A55
:10F15800B1EEE68A032E13D04CB107EE904AF8EED2
:10F16800E77AF4EEC87AF1EE10FA01F18180DBF863
:10F17800602002EB550292FBF5F2CBF8202055E413
:10F18800B0EE480A26F09CFC00B2E5E7BEF1010F9C
:10F1980040F3B98607EE103AB8EEC77AC7EE876A29
:10F1A800B1EEE68A032E13D04CB107EE904AF8EE82
:10F1B800E77AF4EEC87AF1EE10FA01F15980DBF83B
:10F1C800642002EB550292FBF5F2CBF8242048E4C8
:10F1D800B0EE480A26F074FC00B2E5E7F7EE006AE4
:10F1E800FDF71ABCF7EE006AFDF790BC76EEC65A3A
:10F1F800F0EE466AEFE5194BD3F800E0BEF932703D
:10F20800FEF7A2BA8222FDF775BFDFED157AFDF78A
:10F218003DBFB6EE007AF4EEC75AF1EE10FA3FF7AA
:10F228000BAEFDF7CAB8D4F824614A003EB15518B0
:10F2380000EB850576786D78B542BCF495AB0A4449
:10F2480000EB82000022C4F82401A4F80C22C4F8C0
:10F258001022FCF789BB00BFB03B0020AC47002060
:10F268000000024395ED006A9DED0A4AE44825EE48
:10F27800866AFDEEE43AA4EE076AB0EE674AA6EEA7
:10F28800264A13EE901AB4EEC45AF1EE10FAB0EE14
:10F29800446A88BFB0EE646ABDEEC66A16EE108A8C
:10F2A80016EE107AF045A8BF77464145C8BF0F460D
:10F2B80006EE107AB8EEC66A012A80ED006A3DF4BF
:10F2C800D0A995ED046A9DED0B4A25EE866AA4EE59
:10F2D800076AB0EE674AA6EE264AB4EEC45AF1EEC3
:10F2E80010FAB0EE446A88BFB0EE646ABDEEC66A32
:10F2F80016EE108A16EE107AF045A8BF77468845B4
:10F30800B8BF0F4606EE107AB8EEC66A022A80ED3C
:10F31800016A3DF4A6A995ED086A9DED0C4A25EE13
:10F32800866AA4EE076AB0EE674AA6EE264AB4EEED
:10F33800C45AF1EE10FAB0EE446A88BFB0EE646ABF
:10F34800BDEEC66A16EE108A16EE107AF045A8BF12
:10F3580077468845B8BF0F4606EE107AB8EEC66AFB
:10F36800032A80ED026A3DF47CA995ED0C6A9DEDB7
:10F378000D4A25EE866AA4EE076AB0EE674AA6EE45
:10F38800264AB4EEC45AF1EE10FAB0EE446A88BFC9
:10F39800B0EE646ABDEEC66A16EE108A16EE107AF2
:10F3A800F045A8BF77468845B8BF0F4606EE107AE5
:10F3B800B8EEC66A042A80ED036A3DF452A995EDB9
:10F3C800106A9DED0E4A25EE866AA4EE076AB0EE35
:10F3D800674AA6EE264AB4EEC45AF1EE10FAB0EE29
:10F3E800446A88BFB0EE646ABDEEC66A16EE108A3B
:10F3F80016EE107AF045A8BF77468845B8BF0F4685
:10F4080006EE107AB8EEC66A052A80ED046A3DF465
:10F4180028A995ED146A9DED0F4A25EE866AA4EE9B
:10F42800076AB0EE674AA6EE264AB4EEC45AF1EE71
:10F4380010FAB0EE446A88BFB0EE646ABDEEC66AE0
:10F4480016EE108A16EE107AF045A8BF7746884562
:10F45800B8BF0F4606EE107AB8EEC66A062A80EDE7
:10F46800056A3DF4FEA895ED186A9DED104A25EE53
:10F47800866AA4EE076AB0EE674AA6EE264AB4EE9C
:10F48800C45AF1EE10FAB0EE446A88BFB0EE646A6E
:10F49800BDEEC66A16EE108A16EE107AF045A8BFC1
:10F4A80077468845B8BF0F4606EE107AB8EEC66AAA
:10F4B800072A80ED066A3DF4D4A895ED1C6A9DEDF7
:10F4C800114A65EE865AE7EE045AE6EEA57AB4EEDE
:10F4D800E75AF1EE10FAC8BFF0EE647AFDF7B1B85A
:10F4E80077EEC76AF0EE477ACEE4464A4FEA8906D5
:10F4F8005FEA9C0900EB060802EBC313264400F000
:10F50800118709F101094FEA091903EB090703F10A
:10F51800100208F1100006F1100112ED024A12ED76
:10F52800035A12ED016A12ED047A50ED024A50EDC9
:10F53800035A50ED016A50ED047A64EE244A65EEF0
:10F54800255A66EE266A67EE277A1032974241ED11
:10F55800024A41ED035A41ED016A41ED047A00F196
:10F56800100001F11001D8D1A9F110094B4408EBA2
:10F5780009004E441CF0030C3EF475AFB3EC017A5D
:10F58800F0EC017A67EE277ABCF1010CE6EC017A1F
:10F59800F4D1FEF768BFBEF834309FED1B7A07EE52
:10F5A800903AF8EEE77A194B67EE877AC3ED007A5E
:10F5B800FDF7AEB8B7EE007A77EE677AF4EEE75A61
:10F5C800F1EE10FA88BFF0EE675A42E407EE906A4F
:10F5D800DFED0F6AF8EEE77A66EEA65A9FED0D5A50
:10F5E8009FED0D6A9FED0D7AA5EE856A26EEA55A68
:10F5F800A5EE867AE5EE076A26EEA70AFFF75CB95C
:10F60800B03B00209C3700206F12833A0400002092
:10F6180084F9223F92E741B99730083C15A82ABEE1
:10F6280095ED006A9DED0A4AAE4825EE866AFDEE24
:10F63800E43AA4EE076AB0EE674AA6EE264A13EE4D
:10F64800907AB4EEC45AF1EE10FAB0EE446A88BF6C
:10F65800B0EE646ABDEEC66A16EE10CA16EE101A4F
:10F66800F445A8BF71466745C8BF394606EE101A6B
:10F67800B8EEC66A012A80ED006A3DF437AF95ED11
:10F68800046A9DED0B4A25EE866AA4EE076AB0EE81
:10F69800674AA6EE264AB4EEC45AF1EE10FAB0EE66
:10F6A800446A88BFB0EE646ABDEEC66A16EE10CA38
:10F6B80016EE101AF445A8BF7146BC45B8BF3946C6
:10F6C80006EE101AB8EEC66A022A80ED016A3DF409
:10F6D8000DAF95ED086A9DED0C4A25EE866AA4EEFD
:10F6E800076AB0EE674AA6EE264AB4EEC45AF1EEAF
:10F6F80010FAB0EE446A88BFB0EE646ABDEEC66A1E
:10F7080016EE10CA16EE101AF445A8BF7146BC458D
:10F71800B8BF394606EE101AB8EEC66A032A80ED5D
:10F72800026A3DF4E3AE95ED0C6A9DED0D4A25EEB7
:10F73800866AA4EE076AB0EE674AA6EE264AB4EED9
:10F74800C45AF1EE10FAB0EE446A88BFB0EE646AAB
:10F75800BDEEC66A16EE10CA16EE101AF445A8BF1A
:10F768007146BC45B8BF394606EE101AB8EEC66AEF
:10F77800042A80ED036A3DF4B9AE95ED106A9DED5B
:10F788000E4A25EE866AA4EE076AB0EE674AA6EE30
:10F79800264AB4EEC45AF1EE10FAB0EE446A88BFB5
:10F7A800B0EE646ABDEEC66A16EE10CA16EE101AFE
:10F7B800F445A8BF7146BC45B8BF394606EE101AD5
:10F7C800B8EEC66A052A80ED046A3DF48FAE95ED61
:10F7D800146A9DED0F4A25EE866AA4EE076AB0EE1C
:10F7E800674AA6EE264AB4EEC45AF1EE10FAB0EE15
:10F7F800446A88BFB0EE646ABDEEC66A16EE10CAE7
:10F8080016EE101AF445A8BF7146BC45B8BF394674
:10F8180006EE101AB8EEC66A062A80ED056A3DF4AF
:10F8280065AE95ED186A9DED104A25EE866AA4EE40
:10F83800076AB0EE674AA6EE264AB4EEC45AF1EE5D
:10F8480010FAB0EE446A88BFB0EE646ABDEEC66ACC
:10F8580016EE10CA16EE101AF445A8BF7146BC453C
:10F86800B8BF394606EE101AB8EEC66A072A80ED08
:10F87800066A3DF43BAE95ED1C6A9DED114A65EEB6
:10F88800865AE7EE045AE6EEA57AB4EEE75AF1EEA8
:10F8980010FAC8BFF0EE647AFDEEE77A17EE901A18
:10F8A8008E45A8BF8E468F42D8BF774607EE907A1E
:10F8B800F8EEE77AC0ED077AFDF715BE0A494A69FE
:10F8C800002A3CF41FAA0A6813604B74FCF71ABAA2
:10F8D800D4F89C51049B5D1BFFF78ABA034EFCF7D2
:10F8E80091BF00BFB03B002070640020804500201D
:10F8F800002F00F0AC83E04D9DED0A4A95ED006ABB
:10F9080025EE866AA4EE076AB0EE674AA6EE264A96
:10F91800B0EE446A33B1B4EE445AF1EE10FAC8BFFF
:10F92800B0EE646AFDEEE44ABDEEC66A14EE907A63
:10F9380016EE101A8F4214EE90CA00F3EF84714548
:10F94800A8BF714606EE101ACC48B8EEC66A012A5E
:10F9580080ED006A3CF489AE95ED046ADDED0B4A52
:10F9680025EE866AA4EE876AF0EE674AE6EE264A36
:10F97800B0EE646A002B00F0BB84B4EEE45AF1EEFA
:10F9880010FA40F3B58439467145A8BF714606EEB2
:10F99800101AB8EEC66A022A80ED016A3CF465AE18
:10F9A80095ED086ADDED0C4A25EE866AA4EE876AB5
:10F9B800F0EE674AE6EE264AB0EE646A002B00F0E5
:10F9C8008D84B4EEE45AF1EE10FA40F38784394698
:10F9D8007145A8BF714606EE101AB8EEC66A032A2A
:10F9E80080ED026A3CF441AE95ED0C6ADDED0D4AFE
:10F9F80025EE866AA4EE876AF0EE674AE6EE264AA6
:10FA0800B0EE646A002B00F05F84B4EEE45AF1EEC5
:10FA180010FA40F3598439467145A8BF714606EE7D
:10FA2800101AB8EEC66A042A80ED036A3CF41DAECB
:10FA380095ED106ADDED0E4A25EE866AA4EE876A1A
:10FA4800F0EE674AE6EE264AB0EE646A002B00F054
:10FA58003184B4EEE45AF1EE10FA40F32B843946BF
:10FA68007145A8BF714606EE101AB8EEC66A052A97
:10FA780080ED046A3CF4F9AD95ED146ADDED0F4AAA
:10FA880025EE866AA4EE876AF0EE674AE6EE264A15
:10FA9800B0EE646A002B00F00384B4EEE45AF1EE91
:10FAA80010FA40F3FD8339467145A8BF714606EE4A
:10FAB800101AB8EEC66A062A80ED056A3CF4D5AD80
:10FAC80095ED186ADDED104A25EE866AA4EE876A80
:10FAD800F0EE674AE6EE264AB0EE646A002B00F0C4
:10FAE800D683B4EEE45AF1EE10FA40F3D0833946E7
:10FAF8007145A8BF714606EE101AB8EEC66A072A05
:10FB080080ED066A3CF4B1AD95ED1C6ADDED114A55
:10FB180065EE865AE4EE875AE5EEA67A002B00F0E9
:10FB2800AE83F4EEC57AF1EE10FA40F1A8833A46B6
:10FB38007245A8BF7246944607EE90CAF8EEE77A77
:10FB4800C0ED077AFCF791BDD4F89C51049B5D1B6E
:10FB5800FFF7A7B996ED000A0593039225F0B0FFC9
:10FB68004749DFF850E1D1F8EC10DFF84CC1039AAF
:10FB7800ACF800008EFB013EC917C1EBAE1107EED1
:10FB8800901AF8EEE77A059BFDEEE77A17EE901AE1
:10FB9800ACF80210FCF73BBE07EE906ADFED396A5D
:10FBA8009FED397A84F80462F8EEE77A67EEA67A70
:10FBB80077EE876ABDEEE66A16EE103A2033402BE0
:10FBC80040F2B582DFED316A314BBDEEE77AC3ED25
:10FBD800016A17EE103A2033402B00F2EF829FEDB6
:10FBE8002D7AF4EEC77AF1EE10FA40F31984DFEDBE
:10FBF8002A5A9FED2A6A01E0F0EE477AF4EEC67AB7
:10FC0800F1EE10FA37EEE57AF6DCDFED257AB4EEA0
:10FC1800E77AF1EE10FA40F10A84DFED1F5A9FED02
:10FC2800216A01E0B0EE677AB4EEC67AF1EE10FA16
:10FC380077EE257AF6D49FED147AF4EEC77AF1EED2
:10FC480010FA40F304839FED137A77EE677A67EE34
:10FC5800A75A9FED155A9FED156A9FED157AA5EEE7
:10FC6800856A27EEA55AA5EE867AE5EE077AC4EDF1
:10FC7800827AFDF7BBBD00BF38510020B03B0020A1
:10FC8800E002002035FA8E3CDB0FC93F000000007F
:10FC980004000020DB0F4940DB0FC940E4CB1641CC
:10FCA800DB0F49C0E4CB16C192E741B99730083C55
:10FCB80015A82ABED34D62106445002025EE866A39
:10FCC800A5EE076AB0EE675AA6EE265ABDEEC56ADB
:10FCD80016EE100A814200F38B817045A8BF70466A
:10FCE80006EE100AB8EEC66AB8F1000F00F0B38449
:10FCF800DE48012A80ED006A3CF4B7AC95ED046A51
:10FD08009DED0B5A25EE866AA5EE076AB0EE675A96
:10FD1800A6EE265ABDEEC56A16EE107AB94200F371
:10FD280065817745A8BF774606EE107AB8EEC66AB1
:10FD3800B8F1000F00F08384022A80ED016A3CF4D8
:10FD480094AC95ED086A9DED0C5A25EE866AA5EEF1
:10FD5800076AB0EE675AA6EE265ABDEEC56A16EED9
:10FD6800107AB94200F340817745A8BF774606EE7E
:10FD7800107AB8EEC66AB8F1000F00F05484032A6E
:10FD880080ED026A3CF471AC95ED0C6A9DED0D5A5C
:10FD980025EE866AA5EE076AB0EE675AA6EE265AE1
:10FDA800BDEEC56A16EE107AB94200F31B8177459D
:10FDB800A8BF774606EE107AB8EEC66AB8F1000F0B
:10FDC80000F02584042A80ED036A3CF44EAC95EDDE
:10FDD800106A9DED0E5A25EE866AA5EE076AB0EE0A
:10FDE800675AA6EE265ABDEEC56A16EE107AB942D3
:10FDF80000F3F6807745A8BF774606EE107AB8EE8E
:10FE0800C66AB8F1000F00F0BB83052A80ED046ACA
:10FE18003CF42BAC95ED146A9DED0F5A25EE866ADD
:10FE2800A5EE076AB0EE675AA6EE265ABDEEC56A79
:10FE380016EE107AB94200F3D1807745A8BF77460D
:10FE480006EE107AB8EEC66AB8F1000F00F07283B9
:10FE5800062A80ED056A3CF408AC95ED186A9DED1C
:10FE6800105A25EE866AA5EE076AB0EE675AA6EE26
:10FE7800265ABDEEC56A16EE107AB94200F3CB8059
:10FE88007745A8BF774606EE107AB8EEC66AB8F18D
:10FE9800000F00F08083072A80ED066A3CF4E5AB8A
:10FEA80095ED1C6A9DED115A65EE865AE7EE055AE6
:10FEB800E6EEA57AFDEEE77A17EE902A914203DC8A
:10FEC8007245A8BF7246114607EE901AF8EEE77A17
:10FED800B8F1000F7FF434AE089B002B7FF430AEEE
:10FEE800059B079A9342B8BFF0EE647A28E6604A09
:10FEF8001278032A00F019820022FEF7FCBD9FED5C
:10FF0800668AFFF727B99FED648AFFF74BB959490D
:10FF1800096811F080587EF48FAFFEF785BFD4F8DA
:10FF28009C51049B5D1BFDF7EFBF9FED530ADFF863
:10FF3800588125EE800A25F0C3FDD4F81451A8F89D
:10FF48000600FDF7EAB8237DFEF721BE4B484C4971
:10FF58008046FEF777BA93F8FF21AA2A7EF404AE0A
:10FF6800D3F8C61149B193F8C221A2F10B000128B8
:10FF78002DD902F0F702062A29D0D3F8D61149B1B3
:10FF880093F8D221A2F10B00012820D902F0F70240
:10FF9800062A1CD0D3F8E61149B193F8E221A2F160
:10FFA8000B00012813D902F0F702062A0FD0D3F864
:10FFB800F61100293EF4D8AD93F8F231A3F10B0203
:10FFC800012A04D903F0F703062B7EF4CDAD41F2E4
:10FFD800FC120123A150A370FEF7B7BE0F462FE70E
:10FFE8000F460AE70F46E5E60F46C0E60F469BE6D2
:08FFF800084675E6F5F7D6FB9B
:020000040801F1
:10000000029BDFF88C8093F800E0039B99F80010C6
:10001000D4F81451C01AA8F80400FEF7B0BA0F467D
:1000200035E7F5F7C3FB029BDFF8648093F800E047
:10003000039BC01AA8F80200FEF7E3BAF5F7B6FB77
:10004000029BDFF84C8093F800E0039BC01AA8F8ED
:100050000200FEF7F6BA0AA9BDEEE46A01EB8202DD
:1000600094460A48034D09941A4616EE107A434600
:100070002CE000BFB03B0020CF49002064410020AD
:100080000000C8421C390020002000203851002008
:100090006445002092E741B99730083C15A82ABE74
:1000A00000000000E4CB1641DB0FC940E4CB16C1D1
:1000B000DB0FC93FDB0F4940DB0FC9BFDB0F49C076
:1000C0006145A5EC016A00F1100031D090ED006AA5
:1000D000B1EC014A25EE866AA7EE046AB0EE674AE3
:1000E000A6EE864AB0EE446A32B1B4EE445AF1EE5E
:1000F00010FAC8BFB0EE646ABDEEC66A16EE108A8A
:10010000474506EE107A04DCF045A8BFF04606EE3F
:10011000108AB8EEC66A002BD2D1089C002CCFD131
:10012000059CA046079CA045B8BFB0EE646AC7E72F
:10013000099CFCF79EBAF4EEC77AF1EE10FA40F390
:1001400077815FED275A1FED296A01E0F0EE476ADB
:10015000F4EEC66AF1EE10FA36EEE57AF6DC5FED03
:10016000296AB4EEE67AF1EE10FA40F15A815FEDB9
:10017000325A1FED326A01E0B0EE667AB4EEC67A0A
:10018000F1EE10FA77EE256AF6D41FED377AF4EE29
:10019000C76AF1EE10FA40F3B9801FED3A7A77EEB4
:1001A000666A66EEA65A1FED455A1FED456A1FEDB9
:1001B000457AA5EE856A26EEA55AA5EE867AE5EE85
:1001C000076A05E55FED4A7A55E51FED467AF4EEDC
:1001D000C76AF1EE10FA40F31B825FED4D5A1FED36
:1001E0004F6A01E0F0EE476AF4EEC66AF1EE10FAEB
:1001F00036EEE57AF6DC5FED4F6AB4EEE67AF1EEC4
:1002000010FA40F1D7815FED585A1FED586A01E0AE
:10021000B0EE667AB4EEC67AF1EE10FA77EE256AA1
:10022000F6D41FED5D7AF4EEC76AF1EE10FA05DD43
:100230001FED607A77EE666AFFF7D2B91FED627A3A
:10024000F4EEC76AF1EE10FA44BF1FED647A77EE60
:10025000666AFFF7C5B91FED687AF4EEC77AF1EE6A
:1002600010FA44BF1FED6B7A77EE677AF3E4D34F51
:1002700007F18002FEF76AB9A8F80600ABF8A850AB
:10028000CE4CFBF77CBBFDEEE77A17EE902ABA4224
:10029000FFF656AC50E4BDEEC66A16EE101AB9422F
:1002A000BFF62AAC39462AE4BDEEC66A16EE101A2D
:1002B000B942BFF6FDAB3946FFF7FDBBBDEEC66ADE
:1002C00016EE101AB942BFF6CFAB3946FFF7CFBBD7
:1002D000BDEEC66A16EE101AB942BFF6A1AB39469A
:1002E000FFF7A1BBBDEEC66A16EE101AB942BFF603
:1002F00073AB3946FFF773BBBDEEC66A16EE101A34
:10030000B942BFF645AB3946FFF745BB9FEDAC7A26
:10031000F4EEC76AF1EE10FA44BF9FEDAA7A77EEC9
:10032000666A3EE714EE901AFFF710BB4046FFF7EF
:1003300025B91FF02BFEFBF71BBB02287CF413AC86
:1003400041F2B4120123A3546370FCF70CBC137C7C
:10035000022B7EF412AD92F8FE31552B7EF40DADDA
:1003600092F8FF31AA2B7EF408ADD689E759964B57
:1003700037441F6092F80DE041F210210EF1FF3377
:100380007F2B44F801E03EF6F8ACCEF100033EEAE4
:1003900003037EF4F2AC4FEA4E2341F21821013BF5
:1003A0006350D08A00B9506A884941F20423E05072
:1003B000B2F811305B0103F2FF135B120B60B2F86D
:1003C000131001B9116A40001E440644891B41F212
:1003D000082C40F6F476B1FBFEF1B14244F80C1063
:1003E00040F2A8804FF6F476B14240F29F8003219C
:1003F0002170D26A76493B44184441F20C2641F2FE
:100400001C230978A051E25009B925F03BF9A378E3
:100410000133A370FCF7A7BB22F068FE2369FEF747
:100420005ABCF0EE476AB0E6B0EE677AFFF7F1BB70
:10043000B0EE667A93E6F0EE477A00E494F878310D
:10044000002B7BF431ADFBF71CBDDFED627AB4EE1F
:10045000E7EAF1EE10FA66DCDFED5F7AB4EEE7EA88
:10046000F1EE10FA5FD45D4BD3ED007AB1EE677A0E
:10047000F4EEC7DAF1EE10FA52D4F4EEE7DAF1EE68
:1004800010FA88BFF0EE67DA554B87ED00CA1B689B
:100490009342BBF661ABFBF7C5BB524A524B1068A7
:1004A0001B689847514BD7ED006A93ED007A504B8B
:1004B000D3ED007A4F4B83ED020A4F4B67EE277A5C
:1004C0002B4427EEAC7AD3ED007A4C4B67EE277ABB
:1004D000F0EE665AEDEEA75A93ED006AB1EE467A59
:1004E000B4EEE57AF1EE10FA08DCF4EEC65AF1EE5D
:1004F00010FA8CBFB0EE467AB0EE657A404B1B78AE
:10050000012B02D0192B7BF439ACDFED3E7AF4EEEF
:10051000E7DAF1EE10FACCBF01230023FBF739BC78
:10052000F0EE47DAB0E7DFED38DAADE7022222700D
:1005300000225FE701232370FEF71FBC089B002BFE
:100540007FF48AAC059B079FBB42B8BFB0EE646ADC
:1005500082E4132B05D1B0EE480A25F0B5FA069BCC
:100560001880B0EE480ADBF8083228489847029B0A
:100570001B78132BB0EE408A7DF401A825F0A4FA75
:10058000069B5880FCF7FBBF089B002B7FF441AC17
:10059000059B079FBB42B8BFB0EE646A39E4089B75
:1005A000002B7FF47CAC059B079FBB42B8BFB0EE2D
:1005B000646A74E4F0EE476A33E600BF002000206E
:1005C000DB0FC9BFDB0F49C0947C0020B47C002046
:1005D000747C002000C0F84400C0F8C42C510020F6
:1005E00010510020A4500020B8500020F84F0020E7
:1005F00004000020503B0020C85000203051002053
:10060000443000200000964200000000A056002068
:10061000B0EE667AEFE5089B002B7FF4D7AB059B25
:10062000079FBB42B8BFB0EE646AFFF7CFBB089B21
:10063000002B7FF4A8AB059B079FBB42B8BFB0EE71
:10064000646AFFF7A0BB089B002B7FF479AB059B86
:10065000079FBB42B8BFB0EE646AFFF771BB089B4F
:10066000002B7FF449AB059B07988342B8BFB0EEDF
:10067000646AFFF741BB00BF2DE9F04F2DED028BFF
:1006800095B0064615F056FFB74B1D7825B115B04D
:10069000BDEC028BBDE8F08FDFF834B3DBF800303F
:1006A0005805F4D5B14F3A68002A00F02681B04CC5
:1006B000D4F8283103F5F43348339E42C0F01D814D
:1006C000DFF8108394F82C11D8F80030C4F82861B2
:1006D000013184F82C11990701F1D68113F0140F20
:1006E00041F07B8113F0080F94F82C3140F07881B1
:1006F000580701F0B580282B9E4B039301F0A88288
:100700005E2090479C4B1B78002B6BD0984C9B4AEB
:10071000D4F83031F31A934201F20080DFF8B8A226
:100720009AF80080B8F1000F33D1DFF86092D9F861
:100730000000F5F7BFFAC0B201280ED90228904F89
:1007400041F03D833B78002B41F00D85D4F83831E2
:10075000F31AB3F57A6F81F096858A480268002A09
:1007600040D09AF80030BBB9874BD9F800001B681D
:100770009B781E3B012B4FF0020141F202850430B1
:1007800013F0ACFE012200238AF8002084F84431E3
:1007900026E07C4802682AB3D4F8403140F6B731ED
:1007A000F31A8B421ED994F83C31002B01F0FE82E3
:1007B000013BDBB284F83C31002B01F0D08112F810
:1007C000011B94F84471026094F845316F48CA19CE
:1007D0000133006884F8442184F84531F5F76EFA56
:1007E000C4F840616A4A039B12781B68012A03F12E
:1007F00001030C9300F0DF86664B1B786BB1664FEC
:100800003B6853B1039B5A4CD3F80090D4F858314D
:10081000A9EB0303632B00F28586DFF8C08198F80B
:100820000090B9F1020F01F07681554F97F87430BE
:10083000032B00F0D487594B1B7873B1584D2B68AC
:100840005BB14B4CF4F7B2FFD4F86431049044F63A
:100850001F62C31A934200F20581524B1B78002B92
:100860004ED1514B1B7843B1414CD4F8B43203F50F
:100870000043E8339E4280F018874C4B1B78002BD6
:100880003FF405AF3A4E4A4C4A4D06F2BD27206868
:10089000F5F710FA00283FF4FAAE2068F5F702FAEF
:1008A0002B7880465A1E33B120682A70F5F702FA79
:1008B0000028F2D1EBE603223946781E26F0A7F88D
:1008C00096F8BC3296F8BD2286F8BF8283F47F4347
:1008D00083F0FF039B1A1FFA88F89BB2B8EB132F23
:1008E000D5D196F8BE22DBB29A42D0D1781E13F051
:1008F00023F92B7818442870C9E71E4B039301E7AE
:100900002D4C2278002A40F04D862C4F3C78002C4C
:1009100040F093802A4D2878002841F0AF83144C92
:10092000284DD4F8AC122A78274B93FBF2F30B44F2
:100930009E4296D394F8B032244AC4F8AC62D75C95
:10094000FB0701F1BE84B90701F12E857A0701F199
:10095000208494F8B0322978013393FBF1F201FB43
:10096000123384F8B0327CE72F420020C8470020C1
:100970001822002090640020764A00203F0D0300DA
:100980000C000020C0470020BC470020B8470020D2
:10099000774A0020844A0020E07C00208C4A002016
:1009A000904A0020D04A0020E14A0020964A0020C8
:1009B0009C4A0020A04A0020684A0020D94A002012
:1009C000D84A0020E04A0020A0860100DC4A00202E
:1009D0001C5700204C470020C44700205E340020F4
:1009E00013F0030A7FF484AE5E2090473B68142026
:1009F0009847184B184AB3F9043082FB03124FEAA8
:100A0000E379C9EBA2090FFA89F95FFA89F013F0CB
:100A1000F5FDC9F3072013F0F1FD3B685E20984710
:100A20003B681C209847504613F0E8FD504613F0F1
:100A3000E5FD94F82C313A685AE6084D286E0028F6
:100A400041F0E1808146064B87F80090C3F8AC6224
:100A500007E700BF5847002067666666E84A00203F
:100A60001822002094F86A31002B41F08080DC4B82
:100A70001A6802F00803002B48F603414AF60B40BF
:100A80004BF60F4349F6074804BF0346884612F069
:100A9000040F4FF0190118BF9846920684F86A11A6
:100AA00003D548F4804848F0200805F0DDFBC8F382
:100AB0000909002841F07685CA4B9F79002F41F043
:100AC000708664204FF0FF3A4FF0000CADF83E7096
:100AD000ADF83CC0CDF842C0CDF846C0CDF84AC014
:100AE000CDF83080CDF83480CDF83890ADF840A006
:100AF0008DF84E000CAF0FCFDFF800E384F805C08F
:100B0000AEE80F0097E80F00AEE807002EF8023BB2
:100B100071464FF0010C1B0CFE271F20C82201F864
:100B20001E39A770A27184F807C0E07094F87A01AA
:100B3000207180F0F10383EA0313DAB2130983F022
:100B4000E70343EA022383EAC2031BB283EA0312E8
:100B5000D2B2C3F3072383EA121343EA022383EAE0
:100B6000C2031BB283F0C80282EA0212D2B2C3F3FC
:100B7000072383EA121343EA022383EAC2031BB268
:100B800083EA0C0787EA0717FFB2C3F3072282EA5A
:100B9000171242EA072200EB0C0382EAC7070EEBAA
:100BA0000C0084F87A31278011F8013B7B4083EAFE
:100BB0000313DBB21A0982EA172242EA032282EA0D
:100BC000C3031BB29FB281422780EDD183F07C0327
:100BD00083EA0313DBB24FEA131E8EEA172E8EEA66
:100BE000032E8EEAC30E0FFA8EFE1FFA8EF9DFF87F
:100BF00010C2A4F800905FFA8EFE4FEA192984F81B
:100C0000289084F827E00CF5D17804F1220ADCF86A
:100C10000000DCF80410DCF80820DCF80C30474653
:100C20000FC70CF1100CD445B846F0D1DCF8000029
:100C300038606D4F9CF8043088F8043007F12708BD
:100C400084F8C9E184F8CA9117F8011F2868F5F7FC
:100C500035F8B845F8D194F86B31002B40F08C870B
:100C60006249039A097812680A2084F86B01002906
:100C700001F07D815E4F01293888089041F2B185ED
:100C80000229B7F802E001F0A384B888079003298D
:100C900001F0A085F8880690042901F095850529C2
:100CA000388901F08C850629B7F80A9001F0838510
:100CB0000729B7F80C8001F07B85FB89059394F830
:100CC0007A110C920B4683F0300282EA0212D2B201
:100CD00017094849099387F07A0747EA02270988E4
:100CE000237187EAC202444FC1EB012187FB013A1D
:100CF000089B4FF0000C63F30F0C079B6EF31F4C27
:100D00004FF0000E63F30F0E069BCDF834C012B205
:100D10008A440027C91763F31F4EC1EB6A2A059B5B
:100D2000CDF838E082EA021160F30F070020C9B263
:100D300068F30F00C2F3072269F31F4782EA11121A
:100D400063F31F404FF000090F978DF845A01090F6
:100D50008DF8449042EA01220DF1300C82EAC1077D
:100D6000BCE80F003FB287F0C80888EA0818DFF82F
:100D70008CE084F805905FFA88F8C7F30727AEE89F
:100D80000F0087EA181747EA08239CE8030083EA64
:100D9000C8031BB283F023024EF8040B82EA02124E
:100DA000D2B2C3F30723099F83EA1213704643EAC2
:100DB000022383EAC20207F1010C20F814194FF054
:100DC00023081621FE27C82384F87AC1228084F8DC
:100DD00007800EF1020EA770E170A371114611E0B9
:100DE0004C4700203C470020BB230020E04200206D
:100DF0008E880020CC49002003082080202200207B
:100E00001A22002010F8013B4B4083EA0313DBB2A7
:100E10001A0982EA112242EA032282EAC3031BB2C0
:100E200099B270452180EDD183F0F40383EA031376
:100E3000DBB24FEA131E8EEA112E8EEA032E8EEAE3
:100E4000C30E0FFA8EFE1FFA8EF8D44FA4F800805E
:100E50004FEA182C5FFA8EFE84F81EE084F81FC05B
:100E60007968BA683868FB6807F5D178A8E80F0098
:100E700038697969BA6904F2A317A8E8070004F28F
:100E8000C11884F8C1C184F8C0E117F8011F2868AF
:100E9000F4F714FFB845F8D194F87271002F40F0C0
:100EA0007486BF4B94F87AE1B3F90010B3F90220CD
:100EB000B3F904309FEDBB6A677107EE103A039BEC
:100EC0001B680C938EF06A0383EA031306EE901AF4
:100ED000D9B20B0983F0D50343EA012383EAC103A6
:100EE0001BB283EA03115242C9B207EE902AC3F340
:100EF000072383EA111343EA0123F8EEE77AF8EEB9
:100F0000E66AB8EEC77A83EAC1031BB267EE867A57
:100F100066EE866A27EE067A002083F0C808CDEDDB
:100F20000E7ACDED0D6A8DED0F7A10901190129022
:100F300088EA081C0DF130095FFA8CFCC3F307281E
:100F4000B9E80F0088EA1C1848EA0C2888EACC089F
:100F5000DFF86CC20FFA88F8ACE80F0088F01E07C3
:100F600099E8070087EA0717FFB2C8F3072383EA67
:100F7000171343EA07238CE8070083EAC7071C20FE
:100F8000C8214FF005094FF01E08FE230EF10102A3
:100F9000E07084F8729184F80780A3700CF10C0063
:100FA000A171ACF1100184F804E0278084F87A2163
:100FB00011F8013B7B4083EA0313DBB21A0982EA92
:100FC000172242EA032282EAC3031BB29FB2814284
:100FD0002780EDD183F0270383EA0313DBB24FEAC6
:100FE000131E8EEA172E8EEA032E8EEAC30E0FFA18
:100FF0008EFE1FFA8EF9DFF8A4C1A4F800905FFA04
:101000008EFE4FEA192984F8259084F824E00CF527
:10101000D17804F1220ADCF80000DCF80410DCF8D6
:101020000820DCF80C3047460FC70CF1100CD445F3
:10103000B846F0D15C4FBCF80030A8F8003007F19A
:10104000240884F8C6E184F8C79117F8011F2868BE
:10105000F4F734FEB845F8D194F873310393002BBC
:1010600040F08F85514B1B68052213F0140F84F854
:10107000732140F0AA86DFED4E7A94F87A81484BCE
:101080004C4AB3F90410B2F906204B4F4B48CDED52
:101090000E7A88F0220383EA03135FFA83FE4FEA95
:1010A0001E1383F0590343EA0E2383EACE03B2F5FD
:1010B000FA6F1BB2A8BF4FF4FA6283EA031E5FFA0D
:1010C0008EFEB2F57A7FC3F3072383EA1E13B8BFFF
:1010D0004FF47A724FF0640C43EA0E23A2F57A7251
:1010E0000CFB02F283EACE0387FB02C780FB01C040
:1010F0000FFA83FED217C9174FF0000AC2EBA712EE
:10110000C1EBA0018EF0C8070DF13009ADF8422007
:10111000ADF84010CDF830A0CDF834A0CDF83CA00B
:10112000CC4687EA0717BCE80F00FFB2CEF3072EC4
:101130008EEA171E4EEA072E8EEAC707DFF880E018
:10114000DCF800C084F80480AEE80F003FB287F0FE
:101150004A0383EA0313DBB2C7F3072181EA1311C1
:10116000724641EA032108F1010881EAC303142011
:1011700042F810C9FE274FF04A0C002184F87A810A
:101180004FF0C808E07023800EF1040E84F807C009
:10119000A770617184F80680184613E01A220020B7
:1011A0005847002088C3E43ABB2300204C47002066
:1011B000000000008E880020D34D621067666666CE
:1011C0002022002012F8011B414081EA0111C9B21E
:1011D0000B0983EA102343EA012383EAC10109B220
:1011E00088B272452080EDD181F0140181EA0111AD
:1011F000C9B24FEA111E8EEA102E8EEA012E8EEA37
:10120000C10E0FFA8EFE1FFA8EFC4FEA1C2ABF4B4E
:10121000BE4884F81DA05FFA8EFE84F81CE0BB4F28
:1012200059689A680068DB68A4F800C007F5D17CAB
:10123000ACE80F0038697969B7F81880ACE80300AA
:1012400004F2A317ACF8008084F8BFA1B84684F874
:10125000BEE104F2BF1A18F8011F2868F4F72EFD4A
:10126000C245F8D1AA4BAB4A1B781278013B12F069
:101270000100DBB214BFC0214021172B03D8A64ABE
:1012800013441B7B0393A54B1A8893071ABF0023B3
:1012900041F01001012312F4027F18BF022312F063
:1012A000100F18BF062312F0200F18BF10230028BC
:1012B00040F0D9874FF0030C94F87AA10C938AF090
:1012C000460383EA0313DAB2130983F0920343EA75
:1012D000022383EAC2031BB283EA0310C0B2C3F342
:1012E000072282EA101242EA002282EAC00212B207
:1012F00082F0C80E8EEA0E1E00235FFA8EFE9DF865
:101300000C808DF834800320C2F307228DF837C09B
:1013100082EA1E128DF835308DF836108DF83800BF
:1013200042EA0E2C99E807008CEACE0E0FFA8EFEE8
:10133000DFF8EC81E3718EEA0E1CA8E803005FFA87
:101340008CFCCEF3072E8EEA1C1E4EEA0C2181EA9D
:10135000CC0C94F808E088F800200FFA8CFC8EEA98
:101360000C0E8EEA0E1E5FFA8EFECCF3072282EA86
:101370001E1242EA0E22607AA17A94F80BC06371C1
:1013800082EACE0E0FFA8EFE80EA0E0080EA00128C
:10139000D2B2CEF3072080EA121040EA022080EA9F
:1013A000C20000B2414081EA0111C9B2C0F3072274
:1013B00082EA111242EA012282EAC10212B28CEAE6
:1013C000020C8CEA0C1C5FFA8CFCC2F3072282EA46
:1013D0001C1242EA0C2294F80CE0607BA17B94F88A
:1013E000109084F804A082EACC0212B28EEA020EB7
:1013F0008EEA0E1E5FFA8EFEC2F3072282EA1E12EA
:1014000042EA0E2282EACE0212B2504080EA001076
:10141000C0B2C2F3072282EA101242EA002282EA34
:10142000C00212B2514081EA0111C9B2C2F30722CF
:1014300082EA111242EA012282EAC102E17B13B27E
:1014400081EA030282EA0212D2B2C3F3072383EADB
:10145000121343EA022383EAC2031BB289EA03029E
:1014600082EA0212D2B2C3F3072383EA121343EAD9
:10147000022383EAC2031BB283F0320282EA021221
:10148000D2B2C3F3072383EA121343EA022383EAA7
:10149000C2031BB29AB24FF0FE0C0AF10101DBB29B
:1014A00022804FF0090EC82084F802C04FEA122CA7
:1014B000A8F10E0284F803E0A07184F87A1184F890
:1014C00012C00393637458F80E0C5168926838F890
:1014D00002AC9DF80C3008F5CA7EAEE8070008F5AE
:1014E000D2788EF80290AEF800A084F8B4C184F8E7
:1014F000B33117F8011F2868F4F7E0FBB845F8D1BD
:10150000049BC4F86431FFF7A8B900BF1A22002079
:10151000E83B00201B520020FC6C0308A847002079
:1015200020220020DFF82CA3DFF82C83412012F0CA
:1015300033FDBAF9023088FB0320DB17C3EBA000B0
:1015400080B212F00FFDBAF9003088FB0320DB17E0
:10155000C3EBA00080B212F005FDBAF9043088FB9D
:101560000320DB17C3EBA00080B212F0FBFCA64BFC
:1015700038681978F4F7A2FB94F85C3113F001088D
:1015800000F05684A14AC4F858910133DBB2A2FBA3
:101590000312D20802EB8202A3EB420384F85C310F
:1015A000FFF73BB99A4B9B491868F4F753FB0023AC
:1015B0002370FFF7AAB9984F386800283FF41CA998
:1015C0004FF0000A2B46DFF89482944C049655465F
:1015D0009A46F4F76FFBF8B1F5B94FF001092E46C2
:1015E0003868F4F75FFB83B27E2B00F0A98298F88D
:1015F0000120002A4BD194F84811C1B11B2B84F86B
:10160000482100F077820D2B47D0386888F8019088
:10161000F4F750FB0028E3D15346AA4650460CAAE3
:101620007F49049E1D4612F0CFFCFFF7E5B87D2BE5
:1016300000F0938494F84C2122B180F02003DBB2B7
:1016400084F84C1194F84721062A10D8B4F84A11AE
:1016500038681944A4F84A11A118013281F85031B0
:1016600084F84721F4F726FB0028B9D1D4E7B4F871
:101670004A2188F8019013449BB21A0A52FA83F364
:10168000FF2BA4F84A31386802D1664DA1E73868CB
:10169000F4F710FB0028A3D1BEE73868A4F84A216C
:1016A000F4F708FB00289BD1B6E794F8B832C4F8E9
:1016B000B462012B40F27E8394F8B9225A499818FB
:1016C00001EB8001013202F001024F6A84F8B92275
:1016D000BFB1564D0D950DF15009123DA52349F8A6
:1016E000205D802284F8103115233146484684F865
:1016F000112184F81231B847002840F0E18294F8B3
:10170000B8324B4A013382FB0312A2EBE37202EBC5
:1017100042029B1A84F8B832FFF7AFB8454A464BED
:1017200092F80BC0039A1B88D4F83401126843491D
:101730005FFA83FE1F0A4FF47A73121A03FB0CF34D
:1017400000209A4281F81EE0CF7781F814E04F75AF
:101750008870087180F01B83394BDFF8F4E01B6858
:10176000384A3948176800689268C4F830618EFBBF
:10177000038CDB17C3EB6C13DFF8DCC08EFB008E31
:101780008CFB07988CFB029CD217C2EBAC0203F5D2
:10179000FA734FEAE07C9BB2CCEB6E1CFF1700F5AE
:1017A000EA4EC7EBA8070EF1300E8B761B0A0CF140
:1017B000780C4FEA2E2E3030CB764FEA27281312C2
:1017C0000F7781F81D8081F8202081F8213081F881
:1017D00024C081F823E081F82200FEF79FBF1B4B55
:1017E00004931868F4F75AFA00283FF424A8049BDD
:1017F00001211868F4F74EFA0222002387F87420BA
:1018000088F80030FFF717B8BC890020CDCCCCCCCD
:10181000D44A0020284A0020B44700201822002083
:101820005E23002068230020FC6C03083D23002079
:10183000565555557045002084440020A44A002088
:101840005047002070440020544700207435002089
:101850001F85EB5158470020676666660C00002024
:101860005E2090473B6802209847CA4BCA4A9B6A51
:10187000323382FB0329DB17C3EB69195FFA89F066
:1018800012F0BCFEC9F3072012F0B8FE3B685E20E0
:1018900098473B6803209847C04B1B78D90740F115
:1018A000A18117F031FCBE4B9FEDBE7AD3ED037AD8
:1018B00067EE877AFCEEE77ACDED037ABDF80C305F
:1018C000002800F05684D8B24FEA132912F096FE91
:1018D000484612F093FEB44B1B78042B73D0B34AE6
:1018E000B4F82E311178DFF8F4A293FBF1F201FB8A
:1018F000123292B2BAF80030A4F82E2112016420FC
:1019000092B200FB03134900B3FBF1F342EA03294F
:101910005E20C3F303221FFA89F93B6849EA0209F2
:1019200098473B68062098475FFA89F012F066FEF8
:101930004FEA192012F062FE9D49B4F82E214B7A2D
:10194000BAF800A00132012BA4F82E2100F066861F
:101950004A7B0AEB8A031FFA83FA002A40F08D843F
:101960003B685E2098473B683A2098478A4BA3FB28
:101970000A394FEA59191FFA89F3D8B2039312F0C2
:101980003DFE039B180A12F039FE3B685E20984723
:101990003B683B209847642303FB19A39BB285480F
:1019A000053380FB0320DB17C3EBA000C0B212F0AD
:1019B00025FE002012F022FEDFF81C9299F8063076
:1019C000002B40F01E84D8F80030180700F1D982AF
:1019D00094F82C313A68FEF78EBE5E2090473B6843
:1019E00030209847744BD3F800905FFA89F012F0DA
:1019F00005FEC9F3072012F001FE94F82C3113F014
:101A000003097FF418A86D49D4F828216C4B8A4249
:101A10001B6840F2BA83002BB8BF5B425E4A1BB220
:101A200082FB0312D917C1EB62124FF0640909FB64
:101A300012390FFA89F913B25FFA89FADAB2C9F3E7
:101A40000729C3F307213B6804915E20039298475E
:101A50003B6810209847039A104612F0CFFD049976
:101A6000084612F0CBFD3B685E2098473B6821207A
:101A70009847504612F0C2FD484612F0BFFDD8F814
:101A800000303A68FEF72EBEDFF854919FED4D8A84
:101A900004944FF0240A5E20904750463B689847D4
:101AA000494BF9EC016A9B8A07EE103AF8EEE66AB8
:101AB000B8EEC77A0AF1010AC6EE877A5FFA8AFAA7
:101AC00067EE887AFDEEE77ACDED037ABDF90C403A
:101AD000E0B212F093FDC4F3072012F08FFDBAF1CB
:101AE000270F01D03A68D6E7049CD8F800303A684E
:101AF000FEF7F4BD3868F4F7DDF800287FF485AD13
:101B0000386884F8469188F80190F4F7D3F80028F3
:101B10007FF466AD80E5F3F749FE2C4B1B68A0EB24
:101B2000030A40F6B8339A4500F25A81284B1B79D4
:101B30003A2B00F07D84002388F80030FEF77BBE4E
:101B4000386884F8466184F8476184F8489188F8D9
:101B50000160F4F7AFF800287FF442AD5CE594F83B
:101B6000441194F845311B484A1CFEF731BE013B35
:101B700084F86A31FFF76FB8013B84F86B31FFF7E7
:101B80008BB9013B84F87331BAE4013F84F8727178
:101B9000FFF762BA743B00201F85EB511B520020F7
:101BA00080450020CDCC4C3ECF4900207E45002012
:101BB0007045002067666666544700203F4B4C0026
:101BC0005047002000007A44604700206434002021
:101BD0004C340020B84700203C47002084440020BB
:101BE00090470020844A854BB2F80890A3FB09393E
:101BF0004FEA99095FFA89F012F000FD4FEA1920C7
